:020000040800F2
:1080000090AC00209D810008A5810008CDA8000843
:10801000A9810008AB810008AD81000800000000C4
:10802000000000000000000000000000AF81000818
:10803000B181000800000000B3810008B58100088C
:10804000B7810008B7810008B7810008B781000830
:10805000B7810008B7810008B7810008B781000820
:10806000B7810008B7810008B7810008B781000810
:10807000B7810008B78100084F96000853960008A2
:10808000B781000857960008B7810008B78100083B
:10809000B7810008B7810008B7810008B7810008E0
:1080A000B7810008B7810008B7810008B7810008D0
:1080B00005680108B7810008B7810008B78100088A
:1080C000B7810008B7810008B7810008B7810008B0
:1080D000B7810008AD6F0108B16F0108B56F0108E5
:1080E0001F9A0008B7810008B7810008B78100080F
:1080F000B7810008B7810008B78100085B960008C7
:10810000B7810008B7810008B7810008B78100086F
:10811000A56F0108A96F0108B7810008B7810008A1
:10812000B7810008B7810008B7810008B78100084F
:10813000B7810008B7810008B7810008B78100083F
:10814000B7810008B7810008B7810008B78100082F
:10815000B78100085F96000863960008B96F0108B0
:10816000B7810008B7810008B7810008B78100080F
:10817000B7810008B7810008B7810008B7810008FF
:10818000B7810008B7810008DFF80CD000F0C4FB0D
:1081900000480047A18C010890AC002006488047A9
:1081A00006480047FEE7FEE7FEE7FEE7FEE7FEE7DC
:1081B000FEE7FEE7FEE7FEE7A96701088981000800
:1081C0002DE9F05F0546002092469B46884606460C
:1081D000814640241BE0284641464746224600F09F
:1081E00020F853465A46C01A914110D311461846FA
:1081F000224600F04EFA2D1A67EB01084F46224640
:108200000120002100F045FA17EB00094E41201E25
:10821000A4F10104DFDC484631462A464346BDE866
:10822000F09F202A04DB203A21FA02F00021704757
:1082300021FA02F3D040C2F12002914008431946CE
:10824000704740EA01039B0703D009E008C9121FE9
:1082500008C0042AFAD203E011F8013B00F8013B00
:10826000521EF9D27047421E12F8013F002BFBD17B
:1082700011F8013B02F8013B002BF9D17047421C79
:1082800010F8011B0029FBD1801A704730B5054654
:108290000020034600E05B1C934205D2EC5CC85C06
:1082A000201A01D1002CF6D130BD2DE9FE4F8046B9
:1082B00081EA0300C00F0C46009021F0004123F03A
:1082C0000045B8EB0200A94105D240462146904640
:1082D0001C460B46024623F00040104347D0270DB2
:1082E000C7F30A00C3F30A510290401A01904028D4
:1082F0006BDAC3F3130040F4801B0098924620B160
:108300000023D2EB030A63EB0B0B01985946C0F133
:108310004002504600F0BDF906460D46504659460B
:10832000019A00F0C5F910EB08006141002487EACA
:10833000115284EAE7731A4340D0009A62B3019A5B
:10834000012A4FEA075215DC001B61EB02014FF0D6
:10835000004202EA0752CDE90042001C41F58011BB
:1083600032462B4600F04AFA03B0BDE8F08F404693
:108370002146F9E7001B61EB0201001C41F5801367
:1083800000185B412018A2F5001747EB030140EAF3
:10839000D570B6196D4111E06D084FEA360645EA11
:1083A000C0754FEA0752001B61EB0201001C41F54A
:1083B000801149084FEA30000019514132462B46DE
:1083C00003B0BDE8F04F00F00ABA00980122400067
:1083D0000023D0EB020263EBE073009821464FEAE2
:1083E000E074B8EB000061EB0401E9E783F00043BF
:1083F0005BE781F0004158E72DE9FE4F81EA030475
:1084000004F0004421F0004100944FF0000B23F0F1
:10841000004350EA01045ED052EA03045BD0C3F388
:108420000A54C1F30A552C44A4F2F3340194A0FB7E
:108430000254C1F3130141F48011C3F3130343F455
:10844000801301FB024400FB034E840A970A44EAAE
:10845000815447EA8357A4FB076802958D0A05FB00
:1084600007854FEA932C04FB0C542705029D4FEA25
:10847000065847EA1637B5EB08056EEB070C870E72
:10848000920E47EA811742EA8312A7FB0201B6EB7C
:108490000B0164EB00042B0D43EA0C335E1844EB34
:1084A0001C50DA465146E7FB0201C5F313044FEABC
:1084B0000B3343EA14534FEA0432019C43EA0603A8
:1084C000A4F10C040294009CCDE900B400F096F9EC
:1084D00003B0BDE8F08F00200146F9E72DE9F04D2B
:1084E00081EA030404F0004B21F0004514464FF0EC
:1084F000000A23F0004150EA050220D054EA0102AC
:108500001DD0C5F30A570246C5F31303C1F3130088
:10851000C1F30A5640F4801543F48013A7EB060814
:10852000101BD64608F2FD3873EB050002D308F1A4
:10853000010801E092185B41B8F1000F03DA002056
:108540000146BDE8F08D00204FF4801106468446B8
:108550000EE0171B73EB050705D3121B63EB050336
:1085600006434CEA010C49084FEA300092185B417F
:1085700050EA0107EDD152EA030012D082EA04006A
:1085800083EA0501084305D0101BAB4106D2012246
:10859000002306E000224FF0004302E06FF00102EA
:1085A00053101AEB06004CEB085110EB0A0041EB9C
:1085B0000B01BDE8F04D00F012B90EB540F23341A9
:1085C00002910021CDE900110A460B4600F016F990
:1085D00003B000BD0EB540F2334202920022CDE955
:1085E0000022134600F00AF903B000BD70B5C1F3D4
:1085F0000A5201F000450024C1F3130140F2FF3399
:1086000041F480119A4201DA002070BD40F23343F8
:108610009A42A2F2334203DC5242FFF702FE00E02C
:1086200090402C43F1D0404270BDC1F30A52C1F3D7
:10863000130140F2FF3341F480119A4202DA002024
:108640000146704740F233439A42A2F2334202DCC1
:108650005242FFF7E6BD00F01CB801F0004330B411
:1086600021F0004150EA010206D00A0DA2F5607225
:10867000C1F31301002A02DC30BC00207047440F14
:1086800044EAC104C100E01830BC00EBC25000F065
:108690006FB8202A04DB203A00FA02F1002070476C
:1086A0009140C2F1200320FA03F319439040704730
:1086B000202A06DBCB17203A41FA02F043EAE073A6
:1086C00006E041FA02F3D040C2F120029140084393
:1086D000194670470FB4002300B589B00CA900916A
:1086E0000B996FF00042CB601E4B06931E4B079315
:1086F0000423CDE901321D4A089202466B46002050
:1087000000F0A2F909B05DF814FB70B586B006461A
:108710004FF0FF300091CDE90101002015460C46D5
:1087200004903246694604A8FFF7D4FF0346049834
:10873000211825B108B10A4600E022462A60002827
:108740000DD0002B02DD0098884208D0081B009451
:10875000CDE901043246694604A8FFF7BBFF06B025
:1087600070BD0000818C00089F8C00083D890008C6
:108770000029A8BF7047401C490008BF20F0010035
:10878000704710B4B0FA80FC00FA0CF050EA010413
:1087900004BF10BC704749B1CCF1200421FA04F4A5
:1087A00011FA0CF118BF012121430843A3EB0C017E
:1087B000CB1D4FEA00614FEA102042BF002010BCE1
:1087C000704700EBC35010440029A4BF10BC704791
:1087D000401C490008BF20F0010010BC704710B5D4
:1087E000141E73F1000408DA401C41F100019218D4
:1087F0005B411A4301D120F0010010BD2DE9F04D7D
:1088000092469B4611B1B1FA81F202E0B0FA80F2D1
:1088100020329046FFF73DFF04460F4640EA0A002B
:1088200041EA0B0153465A46084313D0114653EA16
:10883000010019D0C8F140025046FFF7F2FC05468E
:108840000E46504659464246FFF723FF084305D0DF
:10885000012004E020463946BDE8F08D00200543A4
:1088600046EAE0762C4337430A986305E40AA0EB16
:1088700008000022FD0A44EA47540A3002D50020CD
:108880000146E9E7010510196941DDE908450019CC
:108890006941BDE8F04DA2E770B521F00043034304
:1088A0000CD0C1F30A550024D5EB040564EB040396
:1088B000D617AD1AB34102DB0020014670BD201867
:1088C00041EB025170BD0EB5C10F80EAE070084463
:1088D000CA07002140F233438DE80E000A460B46DA
:1088E000FFF78CFF03B000BD30B5041E71F100042A
:1088F00004DB4FF00044404264EB0101141E73F1AD
:10890000000405DB1C464FF00043524263EB0403B6
:10891000994208BF904230BD064C074D06E0E06822
:1089200040F0010394E8070098471034AC42F6D3B6
:10893000FFF72EFC30B5010850B50108C0B24FF466
:10894000F05100F027BA00002DE9FF4F087881B000
:108950009946FF2805D0491C2D2804D00024002367
:1089600008E000230BE00124F9E703EB830300EBAD
:108970004303491C0878FF28F7D104B15B4200206B
:108980000090147801462D2C01D02B2C04D1521CC0
:108990002D2C12D00024009400251678FF2E0ED026
:1089A0000A24A0FB04C801FB0481002700FB071177
:1089B000521C16EB0C006941EFE70124EBE79944E8
:1089C00050EA01020ED00024AA4D2646DFF8A88204
:1089D000FFF700FE82468B46B9F1000009DAC9F1C3
:1089E00000071BE001980021C0E9001105B0BDE8B7
:1089F000F08F074612E0F80707D022462B46304694
:108A00004146FFF7F9FC0646884622462B461046AB
:108A10001946FFF7F1FC04460D467F10002FEAD1FE
:108A2000B9F1000F324643465046594602DAFFF785
:108A300055FD01E0FFF7E0FC009A0AB181F000412A
:108A4000019AC2E90001D1E72DE9FF4F1F468DB021
:108A5000D7E901464FF0FF382E2045464FF0000978
:108A60000B90B9696D1C0E988847396A8246884711
:108A70000028F6D1BAF1FF3F0AD024F4D064002ECA
:108A800011DDBAF12B0F08D0BAF12D0F0BD102E096
:108A9000404611B0ABE744F48064B9696D1C0E9890
:108AA00088478246761E6946600501D52D2000E084
:108AB0002B208DF8000001F1010B0DF1200809E0D9
:108AC000B9696D1C0E98884782460F9844F400746B
:108AD000761E0560002E02DDBAF1300FF0D00B9942
:108AE0008A453ED144F0800406E00F99681CA9F144
:108AF000010944F400740860B9696D1C761E0E9873
:108B0000884782463028F0D02BE00B998A4505D162
:108B1000200603D444F08004761E18E050460FF07F
:108B200023FD08B30DF11301761E44F400748B4548
:108B300008D2AAF130000BF8010B200607D5A9F1E5
:108B4000010003E0200602D409F101008146A005DE
:108B500002D50F99681C0860B9696D1C0E9888478A
:108B60008246002ED1DC53E0002E51DDBAF1650FB4
:108B700002D0BAF1450F4BD1A00549D5B9696D1C9A
:108B800024F44074761E0E9888478246002E0CDD31
:108B90002B2804D0BAF12D0F07D144F48074B969A1
:108BA0006D1C0E9888478246761EE00501D52D2162
:108BB00000E02B2108F8011BCDF82C8021E00DF1FD
:108BC0002901761E44F4007488450CD2AAF13000C5
:108BD00010F0FF0088F8000002D10B99884509D9F0
:108BE00008F1010806E0E00501D5244801E042F261
:108BF0000F708146B9696D1C0E98884782460F98A0
:108C00000560002E04DD50460FF0AEFC0028D6D1E2
:108C1000F9690E988847FF208BF8000088F800005B
:108C20000020069007904B466A4608A906A8FFF761
:108C30008BFEA00502D46FF001002AE714F0240F88
:108C40000AD0E00714D1DDE906123868031D3B6045
:108C50000068C0E900120BE0DDE90601FFF7FDFC4A
:108C60000146E00704D13868021D3A6000680160DF
:108C700028460EE7000024400000F03FF1D8FFFF37
:108C8000426842B1016811F8013B23B1521EC0E9AC
:108C90000012184670470121C160881E7047426863
:108CA0005AB1C368016843B983688B4205D0491E35
:108CB000521CC0E90012002070474FF0FF3070478F
:108CC0002DE9F04D00231A461B1A8A4103DB0020D0
:108CD0000146BDE8F08DC1F30A52C1F3130141F41E
:108CE00080154FF0000BD10702D100186D41521EC4
:108CF0000027044640F2FF11384601EB620A3E4667
:108D00008046024600204FF48011FFF78AFAC2190C
:108D10007141BB1846EB0100B4EB030C75EB000C82
:108D200004D3E41A65EB000517460E46241908F132
:108D300001006D4180463428E3DDF91946EB060059
:108D4000091BA84103D24FF0FF32134601E0002275
:108D500013461BEB070046EB0A51BDE8F04DFFF749
:108D60003EBD000030B5041E71F1000404DB4FF07D
:108D70000044404264EB0101141E73F1000405DB62
:108D80001C464FF00043524263EB04038B4208BF82
:108D9000824230BD7F2801D9002208E0064A02EB5A
:108DA0005002C007127800D1120902F00F02012010
:108DB0009040084070470000F0B4010870B58C186E
:108DC00010F8015B15F0070301D110F8013B2A11DF
:108DD00006D110F8012B03E010F8016B01F8016BCC
:108DE0005B1EF9D12B0705D40023521E0DD401F8C8
:108DF000013BFAE710F8013BCB1A921C03E013F891
:108E0000015B01F8015B521EF9D5A142D8D30020C5
:108E100070BD027803E010F8013B1A44D2B2491E3B
:108E200089B2F8D21046704770B5ADF5287D00269E
:108E30000D46ADF89462ADF8986200EB40012D4804
:108E400000EBC104608AA84251D9ADF898624AE0AB
:108E5000A089228A284481B2274800F0B1F8ADF8F1
:108E600094626A46208A0BE0BDF894326168C95C5E
:108E7000BDF89432D154BDF89412491CADF8941247
:108E8000BDF894128842EFD8401E81B21046FFF719
:108E9000C0FF1A498870228A0DF1FF31515C81426E
:108EA00019D1ADF894620CE0BDF894126068BDF879
:108EB0009422405CA1688854BDF89402401CADF82F
:108EC0009402208ABDF89412401E8842ECDC0120F6
:108ED0000DF5287D70BD64200FF084FDBDF898026B
:108EE000401CADF89802BDF898020628B0D30020C7
:108EF000EEE70000F8930108FC6500201E1000203A
:108F0000F0B50D46064600EB46011C48002200EB7A
:108F1000C104ADF5257D608AA8422BD9694606E0DB
:108F2000A0686368805C98548854521C92B2208A6E
:108F3000401E9042F4DC208A401E81B26846FFF752
:108F400068FF228A0DF1FF3100275054A089228A40
:108F5000284481B2684600F02FF929463046FFF7D1
:108F600063FF012807D064200FF03CFD7F1CBFB2D7
:108F7000062FEBD300200DF5257DF0BDF8930108F9
:108F800038B50025ADF800500CF070F80A4C207090
:108F900000F088F820780949242807D0272808D02D
:108FA000282802D1022081F8650038BD81F865507B
:108FB00038BD0120F7E700001E100020D41000206B
:108FC0002DE9F041064615460C46012080F3108835
:108FD000254F0020B8800CF029F8000609D40120A4
:108FE0000FF000FDB888401C80B2B880C828F2D3CA
:108FF00035E0B888C82832D21C4F1021384601F01D
:10900000C6F90821384601F0C4F9E82000F030F82C
:10901000C4F3871000F02CF8A006000E00F028F82A
:10902000002000F025F80024002000F021F8641C46
:10903000A4B2042CF8D3002405E0FF2000F018F8B7
:109040003055641CA4B2AC42F7D31021384601F06D
:10905000A0F9002080F310880120BDE8F0810020F5
:1090600080F31088F9E700001E1000200000024085
:1090700070B50B4C0546022120460CF0F1F8002893
:10908000F9D0294620460CF0F4F8012120460CF0D6
:10909000E7F80028F9D020460CF0E9F8C0B270BD1E
:1090A0000030014010B5012080F310881A4C0020D8
:1090B000A0800BF0BBFF000609D401200FF092FC4A
:1090C000A088401C80B2A080C828F2D320E0A088ED
:1090D000C8281DD2114C1021204601F058F9082152
:1090E000204601F056F93D20FFF7C2FF2A20FFF786
:1090F000BFFF8020FFF7BCFFA720FFF7B9FF1021BB
:10910000204601F046F9002080F31088012010BDB0
:10911000002080F3108810BD1E10002000000240C7
:109120002DE9F04106460D46012080F31088204CC1
:109130000020A0800BF07AFF000609D401200FF078
:1091400051FCA088401C82B2A280C82AF2D32AE037
:10915000A088C82827D2174F1021384601F017F9E8
:109160000821384601F015F98420FFF781FF00201F
:10917000FFF77EFF0020FFF77BFF0020FFF778FF5F
:10918000002404E0305DFFF773FF641CA4B2AC421E
:10919000F8D31021384601F0FCF8002080F3108845
:1091A0000120BDE8F081002080F31088F9E700007D
:1091B0001E1000200000024070B50D46012181F311
:1091C00010881146FFF7ACFF002832D01B4C00205E
:1091D000A0800BF02BFF000609D401200FF002FC49
:1091E000A088401C80B2A080C828F2D322E0A088CA
:1091F000C8281FD2124C1021204601F0C8F80821BF
:10920000204601F0C6F88320FFF732FFC5F3871030
:10921000FFF72EFFA806000EFFF72AFF0020FFF73A
:1092200027FF1021204601F0B4F8002080F31088B9
:10923000012070BD002080F3108870BD1E1000203A
:109240000000024010B500231A4604E010F8014B5C
:109250006340521CD2B28A42F8D3184610BD0000B7
:1092600010B5044639200FF0ABFDE0B20FF0C8FD99
:10927000C4F307200FF0C4FDC4F307400FF0C0FD96
:10928000200E0FF0BDFD4FF48051034801F081F82E
:10929000BDE810400DF082BF000402402DE9F0410E
:1092A000054614460E463A200FF08AFDF0B20FF044
:1092B000A7FD300A0FF0A4FD104F4FF48056314641
:1092C000384601F066F8B0463E460DF067FF1D28AF
:1092D00011D1284600F0A4F807463B200FF070FD9E
:1092E0004146304601F055F83D44002CEDD0208831
:1092F00038442080E9E7BDE8F08100000004024026
:109300002DE9F041054614460E463C200FF058FD6D
:10931000F0B20FF075FD300A0FF072FD114F4FF4EF
:1093200080563146384601F034F80CB100202080D8
:10933000B0463E460DF032FF1E2811D1284600F0FF
:1093400017F907463D200FF03BFD4146304601F03E
:1093500020F83D44002CEDD0208838442080E9E7F7
:10936000BDE8F0810004024010B50BF0A7FD08B184
:1093700000F028F8BDE81040302000F09FB801460A
:10938000362000F089B810B508B100F0A5F8BDE8A6
:109390001040342000F092B810B5044600F09CF85C
:1093A00020785C2801D02F2803D10021642000F010
:1093B000FBF8BDE81040322000F080B8682000F0D3
:1093C0004BB8000010B522200FF0FAFC0FF0EEFCB5
:1093D00004464FF48051024800F0DBFF204610BDE8
:1093E000000402402DE9F0410FF0E0FC06460FF0CA
:1093F000DDFC05460FF0DAFC04460FF0D7FC07460B
:109400004FF48051054800F0C4FF46EA052040EAC9
:10941000044040EA0760BDE8F0810000000402401B
:1094200070B5054627200FF0CBFC0FF0BFFC0446BB
:10943000260007D00FF0BAFC641E05F8010B14F0EB
:10944000FF04F7D14FF48051024800F0A2FF3046EC
:1094500070BD00000004024010B504460C200FF05F
:10946000AFFC20460FF0CCFCBDE81040FFF7BABFC0
:1094700010B504460A200FF0A3FC20460FF0C0FCF4
:109480000FF094FC04464FF48051024800F081FF35
:10949000204610BD0004024010B50C460FF090FCB1
:1094A00020460FF0ADFC4FF48051034800F071FFEF
:1094B000BDE810400DF072BE0004024010B50FF080
:1094C0007FFC4FF48051034800F063FFBDE810407B
:1094D0000DF064BE0004024070B5054601200FF097
:1094E0006FFC0FF063FC432828D22B20FFF7C0FF4E
:1094F000102823D22F200FF063FC00200FF080FCF7
:109500003220FFF7DBFF142818D1CF20FFF7B0FF80
:10951000040013D04C20FFF79FFF00EB04214C20E8
:1095200000F042F85020FFF797FF00EB0421502095
:1095300000F03AF80021702000F036F82F200FF0EC
:109540003FFC2C7806E015F8014F5C2C01D02F2C45
:1095500000D1002420460FF053FC002CF3D1BDE8CD
:1095600070404FF48051014800F013BF00040240E6
:1095700070B505462D200FF023FC0FF017FC0446B4
:10958000260007D028780FF03BFC641E6D1C14F0F9
:10959000FF04F7D14FF48051024800F0FAFE304644
:1095A00070BD00000004024070B505460C460D2059
:1095B0000FF006FC28460FF023FCE0B20FF020FC71
:1095C000C4F307200FF01CFCC4F307400FF018FC95
:1095D000200E0FF015FCBDE870404FF4805101489B
:1095E00000F0D7BE0004024070B5094DFF221346BB
:1095F00005F5807605E010F8014B54402A5D5A408D
:10960000335D491E89B2F6D242EA032070BD0000E4
:109610008891010870B500221346154605E010F840
:10962000014BA2186B41491E89B20029F7D1100CD9
:1096300040EA034092B2801845EB13414FEA0142E1
:1096400042EA104108186FEA000080B270BD07F0CE
:1096500093BC07F031BC07F0FFBB07F05DBC00F026
:10966000CBBF0AF039BD0000074A904201D207483B
:1096700001E005481038064A8B0001EA020101D5D5
:10968000C160704781607047106402400060024012
:109690007D0F7D0F0029016802D041F0010101E03A
:1096A00021F00101016070472DE9F043016821F0CC
:1096B000010101600021016041608160C1600161C0
:1096C000212141613C493C4A3D251039904202D15B
:1096D0008D60BDE8F083384A4FF4746618329042CA
:1096E00001D18E60F5E7344A4FF47417303290425E
:1096F00001D18F60EDE7304A4FF0746C48329042F0
:1097000002D1C1F808C0E4E72B4B2C4A60339842E1
:1097100001D1CA60DDE7284C294B7834A04201D141
:10972000CB60D6E7DFF89080264C08F190084045E2
:1097300001D1CC60CDE7DFF880804FF03D5908F1D2
:10974000A808404502D1C1F80C90C2E71E49DFF8D5
:1097500078800839404501D10D60BAE71A4D1835B7
:10976000A84201D10E60B4E7174D3035A84201D1AF
:109770000F60AEE7144D4835A84202D1C1F800C0D1
:10978000A7E7114D10496035091FA84201D10A60B1
:109790009FE70D4A7832904201D10B6099E70A4A5F
:1097A0009032904201D10C6093E7074AA832904270
:1097B0008FD1C1F800908CE7106002403D0000207E
:1097C000400F002000003D20106402400B0607D52A
:1097D000436912B143F0800301E023F08003436149
:1097E000802908D0002A026801F01E0101D00A4336
:1097F00000E08A430260704730B50368124ACC68C3
:1098000013400A682243D1E905452C432243CC6921
:1098100022430C6A22434C6A22438C6A22434C6BDB
:1098200022438C6B22431A430260426922F00703F1
:10983000D1E90B2422431A4342610A6942604A6813
:1098400082608968C16030BD3F801CF02DE9FC4119
:10985000012120200BF03AFB01268DF80460002541
:109860008DF8065003208DF805001A4C302700971C
:109870008DF807506946204600F036FD302120461D
:1098800000F087FD144C84F8F05484F8F25484F806
:10989000F16484F8F3644FF4FA70C4F8F80400F04B
:1098A0001DF894F86802802812D16565232084F899
:1098B0006D02052084F86C0284F86B72142084F821
:1098C0006A02202084F8690284F8685200F048F89F
:1098D000BDE8FC8100140240D41000207CB50FF0DC
:1098E00043F9D0200FF010F90FF072F900200FF0BB
:1098F0000BF90FF06DF90FF037F9D1200FF004F9E3
:109900000FF066F900246D4601E0062C01D201201B
:1099100000E000200FF0C8F82855641CE4B2072CC2
:10992000F3D30FF03BF90D489DF8061080F86D1247
:109930009DF8051080F86C129DF8041080F86B12E9
:109940009DF8021080F86A129DF8011080F86912E3
:109950009DF8001080F868127CBD0000D410002033
:109960007CB51B48002490F868128DF8001090F820
:1099700069128DF8011090F86A128DF80210012119
:109980008DF8031090F86B128DF8041090F86C129B
:109990008DF8051090F86D028DF806000FF0E4F8D0
:1099A000D0200FF0B1F80FF013F900200FF0ACF851
:1099B0000FF00EF96D46285D0FF0A6F80FF008F9CC
:1099C000641CE4B2072CF6D30FF0E8F87CBD00006D
:1099D000D410002070B5094D0022134605F580769D
:1099E00005E010F8014B54402A5D5A40335D491E92
:1099F00089B2F6D242EA032070BD000088910108C6
:109A0000072A00D9072240EA002021B1012901D10B
:109A1000D040C0B270479040C0F3072070477047F5
:109A2000072A00D9072240EA002029B1012902D1E2
:109A30009040C0F307207047D040C0B2704700008C
:109A400070B5ADF5327D00260D46ADF8BC62ADF8BF
:109A5000C06200EB4001324800EBC104608AA842BA
:109A60005CD9ADF8C06255E0012264212D4800F0B8
:109A7000A9F92C4800788DF80000382842D1228AB4
:109A8000E06802FB0501274800F09CF9ADF8BC62D4
:109A90006A46208A0BE0BDF8BC326168C95CBDF83B
:109AA000BC32D154BDF8BC12491CADF8BC12BDF893
:109AB000BC128842EFD8401E81B2104600F044FA32
:109AC000228A0DF1FF31515C81421BD1ADF8BC629D
:109AD0000EE0BDF8BC226168895CA26800FB05202D
:109AE000BDF8BC221154BDF8BC02401CADF8BC024C
:109AF000208ABDF8BC12401E8842EADC01200DF528
:109B0000327D70BD64200EF06DFFBDF8C002401CB8
:109B1000ADF8C002BDF8C0020628A5D30020EEE7CC
:109B20000490010820410020F0B50E46074600EBE6
:109B300047012648ADF5317D002500EBC1048DF8C5
:109B4000BC52608AB0423DD900210846FFF778FF39
:109B5000012837D1694609E0A268401E00FB0620B3
:109B60006268285C505548556D1CADB2208AA842E9
:109B7000F2D80025208AE16800FB0611401E82B25F
:109B8000134800F09DF9208A401E81B2684600F01B
:109B9000DBF98DF8BC02208AE168012201447043A0
:109BA000401E0144AFA800F08BF931463846FFF75C
:109BB00047FF012807D064200EF014FF6D1CADB2E2
:109BC000062DD7D300200DF5317DF0BD049001089E
:109BD00020410020F0B5ADF5317D2C4D00208DF8F1
:109BE000BC022B4E288000243FE000206F4607E097
:109BF00056F832204968125C0A543A54401C80B22C
:109C0000298801EB410206EBC2010B8A5B1E8342ED
:109C1000EEDC288800EB400006EBC000008A401E06
:109C200081B2384600F090F98DF8BC02288800EB2C
:109C3000400006EBC000C168008A00FB0411401E12
:109C400082B2144800F03CF92888012200EB400061
:109C500006EBC000C168008A01446043401E014415
:109C6000AFA800F02DF9641CA4B2288800EB4000D6
:109C700006EBC000408AA042B7D82888401C80B2BA
:109C800028800728AFD30DF5317DF0BD10000020EE
:109C900004900108204100207CB5012108460BF00A
:109CA00015F901208DF8040002258DF805500024D7
:109CB0008DF806408DF807001820154E0090694673
:109CC000304600F011FB05221146304600F048FBFB
:109CD00005220621304600F043FB052207213046CD
:109CE00000F03EFBA02000908DF8045003208DF87A
:109CF00005008DF806408DF807406946304600F0B3
:109D0000F3FA402000906946304600F0EDFA7CBD41
:109D100000000240F8B5002634460096FFF7BCFF6D
:109D200000F0A0F82248641C8442FCD3214C082196
:109D3000204600F02CFB1021204600F02AFB0620D4
:109D400000F076F80821204600F023FB0821204689
:109D500000F01DFB1021204600F01BFB012000F04D
:109D600067F8002000F064F80821204600F011FB9D
:109D70001148D0F81C0208B9FFF72CFF0F4D2E80B8
:109D80000F4E002405E0C0B22146FFF759FE641CC7
:109D9000A4B2288800EB400106EBC101498AA14228
:109DA000F1D880B2401C80B228800728E9D3F8BDE2
:109DB000FFFF0F000000024000004342100000209F
:109DC000049001082DE9F0410546002416460F468F
:109DD000012080F31088DFF854800821404600F00D
:109DE000D6FA1021404600F0D4FA032000F020F803
:109DF000C7F3074000F01CF8C7F3072000F018F87D
:109E0000F8B200F015F806E0002000F011F8641C2C
:109E100005F8010BA4B2B442F6D30821404600F085
:109E2000B8FA002080F31088BDE8F08100000240FD
:109E300070B50B4C0546022120460BF011FA0028A4
:109E4000F9D0294620460BF014FA012120460BF0E8
:109E500007FA0028F9D020460BF009FAC0B270BD0D
:109E60000030014010B5012186B008030BF06AF8FC
:109E7000124C20460BF0CAF90021ADF8081060150D
:109E8000ADF80A003820ADF80C000720ADF800103E
:109E9000ADF81000ADF804104FF48270ADF8061064
:109EA000ADF80E10ADF80200694620460BF0E3F95C
:109EB000012120460BF0A0F906B010BD0030014092
:109EC0002DE9F0410546002416460F46012080F397
:109ED0001088DFF870800821404600F058FA102101
:109EE000404600F056FA0620FFF7A2FF0821404640
:109EF00000F04FFA0821404600F049FA1021404690
:109F000000F047FA0220FFF793FFC7F30740FFF77F
:109F10008FFFC7F30720FFF78BFFF8B2FFF788FF2B
:109F200005E02878FFF784FF641CA4B26D1CB442DE
:109F3000F7D30821404600F02CFA002080F3108867
:109F4000BDE8F08100000240027803E010F8013B18
:109F50001A44D2B2491E89B2F8D2104670470000A6
:109F600070B51E4A907A012825D1002595721C49AA
:109F70001C480F244E780123F6B14D70D0F82852BA
:109F8000D0F8346245EAC605D0F83062D0F82C0229
:109F9000B60046EA40000543AC43CC708878CC78E4
:109FA000A04208D108710C78A04204D0D07108708A
:109FB000002800D0937170BD4B70D0F82852D0F8B3
:109FC000346245EAC605D0F83062D0F82C02B600FB
:109FD00046EA40000543AC438C70DFE7D410002014
:109FE000C9100020000042422DE9F041ADF57C7D12
:109FF00000273C46ADF8E873FFF7B6F9714D142819
:10A0000007D085F867420EF017FE0DF57C7DBDE8A0
:10A01000F0816D48FFF7C0F96B4E103E1428307088
:10A0200006D042287ED00120FFF7A9F93470ECE772
:10A03000FFF7C4F9C6E90204B046BDF8E803FFF72C
:10A040000FF9FAAA4FF4FA716846FFF727F95FA1F2
:10A0500068460EF055FEB0806E46D0B1E91981F821
:10A06000BC457F1CBFB2282FF8D34746304459A1C6
:10A070000EF046FE78800021001F08E0BA886B18B9
:10A080000A443244D27883F8BC25491C89B2814203
:10A09000F4DB51A168460EF033FE4746A8F80400F1
:10A0A000D0B100216A1882F8E445491C89B22829F8
:10A0B000F8D3304447A10EF023FE78800021093800
:10A0C00008E0BA886B180A443244127A83F8E4250F
:10A0D000491C89B28142F4DB42A168460EF010FEB1
:10A0E000B880D0B100216A1882F80C46491C89B2A8
:10A0F0001429F8D3304437A10EF002FE78800021F5
:10A100000D3808E0BA886B180A443244127B83F891
:10A110000C26491C89B28142F4DB36A168460EF058
:10A12000EFFD00E049E0B88070B395F823160229EE
:10A130000FD00D216A1882F87645491C89B2322960
:10A14000F8D3304423A10EF0DBFD78800021C01F3E
:10A1500024E000216A1882F87645491C89B2322928
:10A16000F8D330441BA10EF0CBFD78800021C01F36
:10A1700008E0BA886B180A443244927983F876254D
:10A18000491C89B28142F4DB0EE0BA886B180A449C
:10A190003244927983F88325491C89B28142F4DBE9
:10A1A00016A11748FEF75FF800210320FFF7BCFC5B
:10A1B0000120FFF7E4F8012027E70348FFF7E3F861
:10A1C00023E70000D41000203810002041504E3DFD
:10A1D000000000003B000000574946494E414D45F4
:10A1E0003D0000005749464950415353574F524490
:10A1F0003D0000005345525645523D000D0A0000F7
:10A200004A1600202F4910B5884206D10121084680
:10A210000AF068FE002101204FE02B49884206D158
:10A22000012102200AF05EFE0021022045E02749BC
:10A23000884206D1012104200AF054FE00210420A6
:10A240003BE02349884206D1012108200AF04AFE5A
:10A250000021082031E01F49884206D10121102049
:10A260000AF040FE0021102027E01B49884206D159
:10A27000012120200AF036FE002120201DE0174990
:10A28000884206D1012140200AF02CFE0021402006
:10A2900013E01349884206D1012180200AF022FEF2
:10A2A0000021802009E00F4988420AD1841501214C
:10A2B00020460AF017FE00212046BDE810400AF0B3
:10A2C00011BE10BD00000240000402400008024020
:10A2D000000C02400010024000140240001802402E
:10A2E000001C024000200240F0B5002201274FF080
:10A2F000030C0B6807FA02F52B40AB422CD1066821
:10A3000053000CFA03F4A64306600E79D0F800E07F
:10A310009E4046EA0E0606600E79012E01D0022EFE
:10A3200012D18668A64386604E79D0F808E09E4038
:10A3300046EA0E0686604668AE43466045688E79FA
:10A340009640B6B235434560C568A543C560CC7933
:10A350009C40C3681C43C460521C102AC9D3F0BD82
:10A360004B07DB0E9A40C90810B500EB8100016A6B
:10A370000F249C40A1430162016A1143016210BD98
:10A380000246002012690A4200D001207047418332
:10A3900070470183704700002DE9F04F7548002594
:10A3A0002DED028B85B001782C4601294FD1002676
:10A3B0008246067000F1020898F80000DFF8B891B4
:10A3C0008B46F52804D098F819004F2874D077E010
:10A3D00098F8020098F8011040EA012465482146E7
:10A3E000801CFFF701F908EB0401497818F80420F4
:10A3F00041EA022181422AD198F803105F4FF129E6
:10A400002AD05F48F2294BD0F32920D180F8486048
:10A4100080F83CB0F52038707E700520B870F320CD
:10A42000F8705920387105215448FFF7DDF8010A0A
:10A430007971B8715348076052490720083908609C
:10A44000504801210C38FFF725F98AF8016005B062
:10A45000BDEC028BBDE8F08F4946481980F8BC6519
:10A460006D1CADB2282DF8D30020241F07E008EBA7
:10A47000000212790B1883F8BC25401C80B2A04260
:10A48000F5DB00210320FFF74FFB0028DFD009F0A8
:10A490007FFFF52038707E700520B870F120BFE78F
:10A4A00080F848B080F83DB0F52038707E70052007
:10A4B000B870F220B4E7FFE798F81A004B281AD0DA
:10A4C0002C4831A1801C0EF01BFC050002D002219B
:10A4D00089F8021008EB0507B87B41280ED0B87B3D
:10A4E0005628B4D1C9F8396689F83D66C9F8396685
:10A4F00089F83D66ABE789F802B0A8E76E462919EE
:10A5000001EB0800007C3055641CA4B2092CF6D382
:10A5100030460CF081FE51EC100BFEF79EF800EE79
:10A52000100A9FED1A8A1A484146C0EE080AC0ED8B
:10A530008D0AB87E4C4689F8380600202A180A444D
:10A54000127F3254401C80B20928F7D368460CF0C1
:10A5500063FE51EC100BFEF780F800EE100AC0EE1F
:10A56000080A10EE900AC4F8390697F8270084F814
:10A570003D066CE712000020D4100020FC030020F0
:10A58000D4400020AC640240524D43000000C84259
:10A59000D414002070B5144C40F2244631462046B5
:10A5A0000CF06FFD00281ED0314620460CF006FD51
:10A5B0000E4D00212846FFF76DF8314620460CF07D
:10A5C000FDFC0B492846FFF74FF82088201D008826
:10A5D000291D4FF47A70086001212846FFF75AF8C8
:10A5E00004490120087070BD001401402864024035
:10A5F000008800101200002010B5104C0E492046B3
:10A60000FFF732F800212046FFF744F80C4C4021B8
:10A6100020460CF02FFD0028F9D0084C0949783C61
:10A620002046FFF721F801212046FFF733F80649BD
:10A630000120487010BD000000802020A06402406E
:10A640000014014000880010120000202DE9F043A2
:10A6500001218FB088050AF039FCDFF88C9048465C
:10A66000FFF722F84020050103900024CDE90545BD
:10A67000C60207940894CDE909461C4F0B944FF08D
:10A680002068CDE900870C940D94694648460E94E5
:10A69000FFF7B2F8012210214846FFF797F8DFF8DC
:10A6A0004890A9F178094846FEF7FEFF4FF47A700A
:10A6B000CDE90340CDE9054507940894CDE9094665
:10A6C0000B480B940C940D94CDF800800E94CDE9BA
:10A6D000017069464846FFF78FF801214846FEF7AA
:10A6E000D9FF0FB0BDE8F083A0640240041401401C
:10A6F000140000207CB5012104200AF0E7FB164E6F
:10A70000082206213046FFF72BFE0822072130469B
:10A71000FFF726FE02218DF8051000258DF8065062
:10A720000124C0208DF8074000908DF80410694680
:10A730003046FFF7D9FD600200908DF804408DF897
:10A74000065003208DF805008DF807406946304615
:10A75000FFF7CAFD7CBD0000000802402DE9F0476C
:10A76000FFF7C8FF4FF4E13000F07AF8FFF76EFF13
:10A7700000F058F8264D002685F8286685F82A66E8
:10A78000012085F8290685F82B0642F21070C5F8DD
:10A790003006214F1F483860DFF87C800E21A8F179
:10A7A0000808C8F80010A8F1040901214846FEF77E
:10A7B00071FF1A4C667060780028FCD04FF4FA7074
:10A7C0000EF010F94FF4165000F04AF8114900202D
:10A7D000134A103101EB000C135C401CC0B28CF822
:10A7E00008300A28F6D300202A1892F8B8250B184A
:10A7F000401CC0B2DA740428F6D339601921C8F8B5
:10A80000001001214846FEF745FF6670BDE8F0875D
:10A81000D4100020E4070020AC64024012000020A5
:10A82000108E010838B545208DF8000002208DF803
:10A83000010001248DF802408DF80340684607F0BE
:10A84000B3F847208DF800008DF8014000208DF806
:10A8500002008DF80340684607F0A6F838BD0000F6
:10A860001FB50446012120200AF06CFB0020ADF842
:10A8700004000094ADF80600ADF80800ADF80C0037
:10A880000C200D4CADF80A00694620460CF030FC57
:10A89000012120460CF095FB012240F22441204684
:10A8A0000CF00EFC102120460CF088FB0122C02188
:10A8B00020460CF090FB1FBD001401400249C879EE
:10A8C0000022CA7170470000D410002002480068BE
:10A8D000C00700D000BEFEE7F0ED00E002494AF6F6
:10A8E000AA200860704700000030004010B50EF04C
:10A8F000A3F9BDE8104064200EF074B82DE9F04FC4
:10A9000083466BA0ADF57D7D002400689A460E4617
:10A910002746FB90ADF8E843042A26D8DFF8949147
:10A9200099F86C1202EBC20505EB0215624A30235E
:10A93000154403EB1111297199F86C1201F00F0104
:10A940003031697199F86B1203EB1111A97199F803
:10A950006B0200F00F003030E871FEF705FD14289F
:10A9600007D089F867720EF067F90DF57D7DBDE8B7
:10A97000F08FDFF84481A8F1240898F8000014282B
:10A980000ED02846FEF708FD88F80000142807D0EE
:10A9900042287DD00120FEF7F2FC88F80070E4E741
:10A9A0004FF47A70864200D90646FEF707FD454609
:10A9B000C5E90207FEF754FC99F86B22484630219E
:10A9C00001EB12128DF8002099F86B2202F00F02B1
:10A9D00030328DF8012099F86A2201EB12128DF8BD
:10A9E000022099F86A2202F00F0230328DF803201B
:10A9F00099F8692201EB12128DF8042090F869226F
:10AA000002F00F0230328DF8052090F8682201EB39
:10AA100012118DF8061090F8680200F00F00303027
:10AA20008DF80700BAF1000F03D0BAF1010F02D080
:10AA300004E0542000E052208DF808003A208DF800
:10AA400009000A23EC4618E00BEB540210780009C9
:10AA5000B0FBF3F1C1EBC10108440CEB0401303051
:10AA60008872107800F00F00B0FBF3F2C2EBC20264
:10AA700010443030A41CC872A4B2B4EB460FE3D328
:10AA800003EB460081B2FAAA6046FEF739FC00E00B
:10AA900009E0FAAA0221FBA8FEF732FC0120FEF72A
:10AAA0006EFC2F7061E72846FEF76DFC5DE7000045
:10AAB0000D0A0000D41000204C1000202DE9F04FAA
:10AAC00000252DED028B99B08DF828508DF85C5043
:10AAD0008DF85450CDE91255CDE900558DF8085048
:10AAE0008DF80C508DF810508DF81450ADF81850AA
:10AAF0009FEDF90AF9488DED090A00F50057253058
:10AB00000124DFF8DCA34FF47A7BD526DFF8D48369
:10AB100007909CE0DFF8C49399F8720918B389F89C
:10AB20007259B7F8F81FDAF88C205046C2F57A72DD
:10AB3000914218D1D0F88C00C0F57A70A7F8F00FC8
:10AB4000E74800218830FEF7A5FDE548E649883052
:10AB5000FEF78AFD88F80040CAF88CB0E048012171
:10AB60008830FEF797FD99F87E0910B389F87E5971
:10AB7000B7F8FA1FDAF844205046C2F57A729142CB
:10AB800017D1406CC0F57A70A7F8F20FD4480021B5
:10AB90004030FEF77FFDD248D4494030FEF764FDD7
:10ABA00088F80140CAF844B0CD4801214030FEF792
:10ABB00071FD99F88A0910B389F88A59B7F8FC1F12
:10ABC000DAF814205046C2F57A72914217D14069E2
:10ABD000C0F57A70A7F8F40FC14800211030FEF7D5
:10ABE00059FDBF48C2491030FEF73EFD88F80240CB
:10ABF000CAF814B0BA4801211030FEF74BFD99F89D
:10AC00009619484619B380F89659B7F8FE1FDAF836
:10AC10002C205046C2F57A72914218D1C06AD146B2
:10AC2000C0F57A70A7F8F60FAD4800212830FEF77E
:10AC300031FDAB48AF492830FEF716FD88F80340D8
:10AC4000C9F82CB0A64801212830FEF723FDA348FF
:10AC500090F8721990F87E29114490F88A2990F89A
:10AC600096091044C1427FF455AF04F00BBE017841
:10AC700019B105708DF8085010E0417819B1457090
:10AC80008DF808400AE0817811B18570022003E058
:10AC9000C17819B1C57003208DF808009DF808002F
:10ACA000DFF8388200EB400101EB001008EB0010E8
:10ACB00090F8161A9DF80800DFF83CB200EB40024D
:10ACC000C2EBC0121BF83200C1280AD19DF808005F
:10ACD00000EB4002C2EBC0120BEBC20080780828E8
:10ACE0000CD0082984F09A85DFE811F0A517280018
:10ACF000AC08641011173B18781BA01E7F4880F821
:10AD000048409DF8080030B1012807D002280FD034
:10AD1000032808D10FE04FF4804101E04FF40051C7
:10AD20007748FFF734FB7748C0F8885204F076BDC7
:10AD30004FF48051F4E74FF40061F1E79DF808000B
:10AD400000EB4001C1EBC0110BEBC10040780021CA
:10AD500005F0B6FF8DF810008DF85450C14619E08B
:10AD60009DF8080000EB400101EB001009EB001119
:10AD70009DF8540001EB001090F8410A9DF8101066
:10AD800088429DF8540002D18DF8100010E0401C5C
:10AD90008DF854009DF8080000EB400101EB001015
:10ADA00009EB001090F8170A9DF854108842D7D884
:10ADB0009DF8080000EB4001C1EBC0100BEBC00098
:10ADC00080780A22B2EB101F9DF8080000EB4002C9
:10ADD000C2EBC0100BEBC000807801D100F00F0077
:10ADE0008DF80C009DF80C0010B910208DF80C00A7
:10ADF0009DF808009DF80C1000EB4002C2EBC01259
:10AE00005F460BEBC20008444078ADF818009DF88F
:10AE1000080000EB4001C1EBC0110BEBC1009DF835
:10AE20000C10491C06F02FFB8DF85C009DF8080003
:10AE300000EB4001C1EBC01107EBC1009DF80C1005
:10AE4000084480789DF85C10884244F0E7849DF8BF
:10AE5000080000EB4001C1EBC01107EBC10138460F
:10AE60004978002904F0DA849DF8081001EB4102CA
:10AE7000C2EBC11100EBC1029DF80C101144CA785D
:10AE80009DF8081001EBC10303EB012109EBC1039D
:10AE90009DF8101001EB411103EB810181F8142F93
:10AEA0009DF8081009EB01129DF81010114481F86B
:10AEB000D059BDF81810CE292DD02DDCB9297DD060
:10AEC00022DC5A29CED0B22904F01E82B529F6D050
:10AED000B629BAD1FEE3000000000000D410002023
:10AEE000006002400F080020008800200080201031
:10AEF00020800010008800106C4E0020D4400020FC
:10AF00000018024000004242C32904F0C381C52951
:10AF10007DD0CA2999D1E4E3E129FCD003F3698605
:10AF2000D52908D0D7299DD0D9298ED17CE2E7290F
:10AF30008BD104F08FBC9DF8081001EB4102C2EBED
:10AF4000C11107EBC100C07889F862009DF80800C4
:10AF500000EB400101EB00109DF8101009EB001010
:10AF600000EB011099F86210A4EBD11290F8421A8C
:10AF700062F3000180F8421A9DF8080000EB4001DE
:10AF800001EB00109DF8101009EB001000EB011010
:10AF900099F862104A0990F8421A62F3410180F868
:10AFA000421A9DF8080000EB400101EB001009EB8C
:10AFB00000119DF8100001EB001000E0E3E390F8B1
:10AFC000420AC0F340019DF8080000EBC00202EB0A
:10AFD000002009EBC0029DF8100000EB401002EBCE
:10AFE000800090F8F00EC0F3400081424BD09DF8F5
:10AFF00008004A4600EBC00101EB002009EBC0014C
:10B000009DF8100000EB401001EB800100E0FDE333
:10B010009DF8080000EB400303EB00109DF8103092
:10B0200009EB001000EB031090F8420A430891F876
:10B03000F00E63F3410081F8F00E9DF8080000EB7C
:10B04000400101EB00109DF8101002EB001000EB26
:10B05000011090F8420A800716D59DF80800D92102
:10B0600000EBC00303EB002009EBC0029DF81000C9
:10B0700000EB401002EB800080F8DC1E9DF8081009
:10B080000220FEF751FD42E09DF8080000EBC001F0
:10B0900001EB002002EBC0019DF8100000EB401016
:10B0A00001EB800080F8E54E9DF80800D92100EB07
:10B0B000C00303EB002002EBC0039DF8100000EB7F
:10B0C000401003EB800080F8DC1E9DF8080000EBC8
:10B0D000400101EB001002EB00119DF8100001EBA4
:10B0E000001191F8420A20F0200381F8423A9DF8BD
:10B0F000080000EBC00101EB002009EBC0019DF846
:10B10000100000EB401001EB800080F8164F9DF816
:10B11000080000EB400101EB001009EB00119DF865
:10B12000100001EB001090F8420A00F001019DF8B8
:10B13000080000EBC00202EB002009EBC0029DF802
:10B14000100000EB401002EB800090F8F00E00F0D1
:10B150000100814203F0A6879DF8080000EBC001C2
:10B1600001EB00209DF8101009EBC00001EB41112C
:10B1700000EB81009DF8081001EB410202EB011188
:10B180009DF8102009EB011101EB021191F8421A10
:10B1900090F8F02E61F3000280F8F02E9DF8080080
:10B1A00000EB400101EB00109DF8101009EB0010BE
:10B1B00000EB011090F8420AC00739D09DF8080052
:10B1C0004F4600EBC00101EB002009EBC0019DF8E8
:10B1D000100000EB401001EB800090F8160F0028E3
:10B1E0009DF8080000EBC00101EB002009EBC00155
:10B1F0009DF8100000EB401001EB80003BD080F880
:10B20000155F9DF8080000EB400101EB001007EB13
:10B2100000119DF8100001EB001191F8420A20F096
:10B22000010281F8422A97F8210638B303F03ABFA9
:10B230009DF8080000EB400101EB00109DF8101094
:10B2400009EB001000EB011090F8421A21F02001E8
:10B2500080F8421A9DF8080000EBC00101EB0020C5
:10B2600009EBC0019DF8100000EB401001EB8000DD
:10B2700080F8155FDAE780F8154FD4E7387D0128AC
:10B28000D4D1786DF98A8842D0D29DF8080000EBBD
:10B29000C00101EB002007EBC0019DF8100000EB9E
:10B2A000401001EB800090F8150F0128BED19DF8E9
:10B2B000080000EBC00101EB002007EBC0019DF886
:10B2C000100000EB401001EB800090F8490F0028BF
:10B2D000ACD19DF8080000EB400101EB001007EB3A
:10B2E00000119DF8100001EB001090F8401A9DF835
:10B2F000080000EBC00202EB002007EBC00080F862
:10B30000D11E9DF80800C32100EBC00202EB002013
:10B3100007EBC0029DF8100000EB401002EB80002C
:10B3200080F8DC1E9DF8080000EB400101EB0010E6
:10B3300007EB00119DF8100001EB0010C0F8445A13
:10B340009DF808100220FEF7EFFB8DF8285017E05B
:10B350009DF8080000EBC00101EB002007EBC001E5
:10B360009DF8100000EB401001EB80019DF82800D3
:10B37000084480F8175F9DF82810491C8DF82810A4
:10B380009DF828001428E3D38DF8285017E09DF885
:10B39000080000EBC00101EB002007EBC0019DF8A5
:10B3A000100000EB401001EB80009DF828100844CD
:10B3B00080F8335F9DF82800401C8DF828009DF828
:10B3C00028000A28E3D331E79DF8080000EBC0010C
:10B3D00001EB002009EBC0019DF8100000EB4010CC
:10B3E00001EB800090F8D80E012844F017829DF8F8
:10B3F000080000EBC00101EB002009EBC00080F861
:10B40000D35E9DF80800022100EBC00202EB002091
:10B4100009EBC0029DF8100000EB401002EB800029
:10B4200080F8D81EB62140E29DF8081001EB4102D9
:10B4300002EB011109EB011191F81C1A00299DF88A
:10B440000C1002D00A29D0D191E00829CDD18DF875
:10B45000285024E09DF8081001EB4102C2EBC11115
:10B460009DF8282000EBC1011144C97801F00F01BB
:10B47000092918D89DF8081001EB4102C2EBC1114F
:10B480009DF8282000EBC1011144C97801F0F001BA
:10B49000902908D89DF82810491C8DF828109DF88F
:10B4A00028100629D6D39DF828100629C4F0B681A5
:10B4B0009DF8081001EB4102C2EBC11100EBC10184
:10B4C000C9780B049DF8081001EB4102C2EBC111D1
:10B4D00000EBC10109799DF8082043EA012102EB44
:10B4E0004203C3EBC21200EBC202527911439DF832
:10B4F000082002EBC20303EB022209EBC2039DF812
:10B50000102002EB421203EB8202C2F8F11E9DF8FA
:10B51000081001EB4102C2EBC11100EBC1018979B6
:10B520000B049DF8081001EB4102C2EBC11100EBC6
:10B53000C101C97943EA01239DF8081001EB4102DA
:10B54000C2EBC11100EBC100007A03439DF8080073
:10B5500000EBC00101EB002009EBC0019DF81000D9
:10B5600000EB401001EB8000C0F8F53E95E08DF84F
:10B57000285024E09DF8081001EB4102C2EBC111F4
:10B580009DF8282000EBC1011144C97801F00F019A
:10B59000092918D89DF8081001EB4102C2EBC1112E
:10B5A0009DF8282000EBC1011144C97801F0F00199
:10B5B000902908D89DF82810491C8DF828109DF86E
:10B5C00028100829D6D39DF828100829C4F0268110
:10B5D0009DF8081001EB4102C2EBC11100EBC10163
:10B5E0008A799DF8081001EB4103C3EBC11100EB10
:10B5F000C101C97842EA01629DF8081001EB4103DC
:10B60000C3EBC11100EBC10109790B049DF80810CF
:10B6100001EB4107C7EBC11100EBC101497943EAD6
:10B6200001210A439DF8081001EBC10303EB01213E
:10B6300009EBC1039DF8101001EB411103EB8101EF
:10B64000C1F8F12E9DF8081001EB4102C2EBC111C7
:10B6500000EBC1018A7A9DF8081001EB4103C3EBAE
:10B66000C11100EBC101C97942EA01629DF80810DD
:10B6700001EB4103C3EBC11100EBC101097A0B04DB
:10B680009DF8081001EB4107C7EBC11100EBC100A9
:10B69000407A43EA002003F0BBBD9DF8080000EBB0
:10B6A000C00101EB002009EBC0019DF8100000EB88
:10B6B000401001EB800090F8D80E03289DF8080098
:10B6C00010D000EB400101EB001009EB00109DF8D9
:10B6D000101000E063E000EB011090F8420A8007D0
:10B6E0002DD51AE000EBC00101EB002009EBC000F2
:10B6F00080F8D35E9DF80800042100EBC00202EB45
:10B70000002009EBC0029DF8100000EB401002EB96
:10B71000800080F8D81EC521C7E09DF8080000EB26
:10B72000C00101EB002009EBC0019DF8100000EB07
:10B73000401001EB800080F8DC6E04F06FB89DF8DB
:10B74000080000EBC00101EB002009EBC0019DF8EF
:10B75000100000EB401001EB800090F8E60E01288D
:10B76000EBD19DF8080000EBC00101EB002009EBD4
:10B77000C0019DF8100000EB401001EB800080F844
:10B78000E65EB6215CE09DF8080000EBC00101EB2D
:10B79000002009EBC00080F8D35EC32185E09DF84E
:10B7A000081001EB410202EB011109EB011191F8C4
:10B7B0001C1A00299DF8081001EB4102C2EBC111CF
:10B7C00000EBC10103F09285C9780A049DF80810C6
:10B7D00001EB4103C3EBC11100EBC101097942EA5E
:10B7E00001229DF8081001EB4103C3EBC11107EBE7
:10B7F000C100407902439DF8080000EBC00101EB55
:10B80000002009EBC0039DF8100000E064E000EBAD
:10B81000401003EB8000C0F80C2F9DF8080000EBEF
:10B82000C00101EB002009EBC0019DF8100000EB06
:10B83000401001EB800090F8D80E022819D0C521E5
:10B840009DF8080000EBC00202EB002009EBC002EB
:10B850009DF8100000EB401002EB800080F8DC1E29
:10B860009DF8080000EBC00101EB002009EBC000CF
:10B870002CE09DF8080000EBC00101EB002009EB73
:10B88000C00080F8D35E9DF80800032100EBC002E1
:10B8900002EB002009EBC0029DF8100000EB401005
:10B8A00002EB800080F8D81ED9219DF8080000EB3B
:10B8B000C00202EB002009EBC0029DF8100000EB73
:10B8C000401002EB800080F8DC1E36E780F8D35E83
:10B8D00033E780F8422A30E79DF8081001EB410277
:10B8E00002EB011109EB011191F81C1A00299DF8D6
:10B8F0000C1002D00E29E8D19CE00C29E5D18DF87E
:10B90000285024E09DF808109DF8283001EB4102F2
:10B91000C2EBC11100EBC102D118C97801F00F01CF
:10B92000092918D89DF8082002EB4203C3EBC21185
:10B9300000EBC1029DF828101144C97801F0F00114
:10B94000902908D89DF82810491C8DF828109DF8DA
:10B9500028100A29D6D39DF828100A29B5D3002229
:10B96000CDE9002229468DF82850BC461FE0DDE9CC
:10B970000002120242EA10620002CDE900029DF8C4
:10B98000080000EB4002C2EBC0109DF828200CEB31
:10B99000C0001044C078DDE90023104341EA0302EF
:10B9A000CDE900029DF82800401C8DF828009DF884
:10B9B00028000528DBD3DDE900239DF8080000EB13
:10B9C000C00707EB002009EBC0079DF8100000EB53
:10B9D000401007EB8000C0F8F92EC0F8FD3E0022B1
:10B9E000CDE900228DF828101FE0DDE900021202E7
:10B9F00042EA10620002CDE900029DF8080000EB67
:10BA00004002C2EBC0109DF828200CEBC00010448F
:10BA1000007ADDE90023104341EA0302CDE9000288
:10BA20009DF82800401C8DF828009DF82800052866
:10BA3000DBD399E08DF8285024E09DF808109DF89C
:10BA4000283001EB4102C2EBC11100EBC102D11859
:10BA5000C97801F00F01092918D89DF8082002EBD8
:10BA60004203C3EBC21100EBC1029DF82810114440
:10BA7000C97801F0F001902908D89DF82810491CD8
:10BA80008DF828109DF828100C29D6D39DF8281081
:10BA90000C29C3F0C3860022CDE9002213462946B3
:10BAA0008DF828501EE0009A1B0243EA126312022E
:10BAB000CDE900239DF8082002EB4203C3EBC2123C
:10BAC0009DF8283000EBC2021A44D278DDE9003735
:10BAD0001A4341EA0703CDE900239DF82820521CB0
:10BAE0008DF828209DF82820062ADCD3DDE90037D0
:10BAF0009DF8082002EBC20A0AEB022209EBC20AF7
:10BB00009DF8102002EB42120AEB8202C2F8F93EC5
:10BB1000C2F8FD7E0023CDE900338DF828101FE028
:10BB2000DDE900231B0243EA12631202CDE9002380
:10BB30009DF8082002EB4203C3EBC2129DF82830A7
:10BB400000EBC2021A44527ADDE900371A4341EA97
:10BB50000703CDE900239DF82820521C8DF82820EA
:10BB60009DF82820062ADBD3DDE900129DF80800A5
:10BB700000EBC00303EB002009EBC0039DF81000AD
:10BB800000EB401003EB8000C0F8011FC0F8052F48
:10BB90009DF8080000EBC00101EB002009EBC0019B
:10BBA0009DF8100000EB401001EB800090F8D81ECB
:10BBB0009DF8080000EBC00202EB002009EBC0007A
:10BBC00090F8D40E81427CD199F821064F46B8B145
:10BBD0009DF8080000EB400101EB00109DF81010EB
:10BBE00009EB001000EB011090F8421A41F0080236
:10BBF00080F8422A9DF808100220FDF795FF88E0A2
:10BC0000C7F835509DF8080000EBC00101EB00209B
:10BC100007EBC0019DF81000102200EB401001EB73
:10BC2000800101F6F9610798FCF70BFB9DF808000D
:10BC300000EBC00101EB002007EBC0019DF81000F4
:10BC400000EB401001EB8000D0F8F11EC7F819108E
:10BC5000D0F8F50EC7F81D009DF8080000EB400174
:10BC600001EB001007EB00119DF8100001EB001034
:10BC700090F8400A3876FE48D0F86812C7F83910B4
:10BC8000B0F86C02A7F83D009DF8080000EBC00179
:10BC900001EB002007EBC0019DF8100000EB401005
:10BCA00001EB8000D0F80C0FC7F821009DF80800C8
:10BCB00000EB400101EB001007EB00119DF81000B4
:10BCC00000E014E001EB0010D0F8440AC7F83F0090
:10BCD000786D81B20220FDF713F900210620FDF7EF
:10BCE00023FF786D401C78650021052085E79DF8CD
:10BCF000080000EB400101EB00109DF8101009EB6B
:10BD0000001000EB011090F8421A41F0040180F895
:10BD1000421A9DF8080000EBC00101EB002009EB7E
:10BD2000C0019DF8100000EB401001EB800080F88E
:10BD3000165F9DF8080000EBC00101EB002009EB45
:10BD4000C0019DF8100000EB401001EB800080F86E
:10BD5000DC6E9DF8080000EBC00101EB002009EB50
:10BD6000C0019DF8100000EB401001EB800090F83E
:10BD7000D80E042843F052859DF8080000EB4001DE
:10BD800001EB00109DF8101009EB001000EB011002
:10BD900090F8421A41F0800280F8422A9DF808008B
:10BDA00000EBC00101EB002009EBC00080F8D34E8E
:10BDB0009DF80800052200EBC00101EB002009EB13
:10BDC000C0039DF8100000EB401003EB800080F8EA
:10BDD000D82EB2E409EBC0019DF8100000EB401032
:10BDE00001EB800090F8DA0EB228F2D19DF808003D
:10BDF00000EBC00101EB002009EBC00080F8D35E2E
:10BE00009DF80800B22100EBC00202EB002009EB14
:10BE1000C0029DF8100000EB401002EB800080F89B
:10BE2000DC1E9DF8080000EBC00101EB002009EBCF
:10BE3000C0019DF8100000EB401001EB800080F87D
:10BE4000DA5E7AE49DF8080000EB4001C1EBC01017
:10BE500059461BF83000042809D09DF8080000EB73
:10BE60004002C2EBC01011F83000152801D1ADF826
:10BE700018009DF80800D94600EB4002C2EBC01044
:10BE800001EBC00042789DF8080000EB4003C3EBD3
:10BE9000C01011F8300042EA0020A0F5805130397E
:10BEA00022D09DF8080000EB4001C1EBC01009EB67
:10BEB000C000494642789DF8080000EB4003C3EB00
:10BEC000C01019F8300042EA0022A2F58050313843
:10BED0000CD09DF8080000EB4002C2EBC01011F836
:10BEE0003000022804D019E0A62015E0A72013E0B6
:10BEF0009DF8080000EB4002C2EBC01001EBC0004F
:10BF000002799DF8080000EB4003C3EBC01009EB79
:10BF1000C000C07842EA0020ADF818009DF8080083
:10BF2000474600EBC00101EB002008EBC00090F891
:10BF3000D21E8DF810109DF8080008EB00119DF836
:10BF40001000084480F8D059BDF8180043F23002C0
:10BF5000811A90427ED009DC04287CD015287BD041
:10BF6000A6280DD0A72843F05984AFE0B1F5C06FE3
:10BF700073D0A1F5C061013970D00429F3D1FBE37E
:10BF80009DF8080000EBC00101EB002007EBC000AA
:10BF900080F8D35E9DF8080000EBC00101EB0020A3
:10BFA00007EBC0019DF8100000EB401001EB800092
:10BFB00090F8D80E032824D09DF8080000EBC001AB
:10BFC00001EB002007EBC0019DF8100000EB4010D2
:10BFD00001EB800090F8D80E082825D09DF80800C5
:10BFE00000EBC00101EB002007EBC0019DF8100041
:10BFF00000EB401001EB800090F8D80E0D2815D012
:10C00000FEE39DF80800042100EBC00202EB0020D3
:10C0100007EBC0029DF8100000EB401002EB80001F
:10C0200080F8D81EA821ECE30921EBE30E21EAE316
:10C030009DF8080000EBC00101EB002007EBC001F8
:10C040009DF8100000EB401001EB800090F8DA0E34
:10C05000A12804E0FAE3B5E0D5E1F6E124E203F03B
:10C06000DD839DF8080000EBC00101EB002001E03A
:10C07000D410002007EBC0019DF8100000EB401029
:10C0800001EB800090F8DA1E9DF8080000EBC0027A
:10C0900002EB002007EBC0029DF8100000EB4010FF
:10C0A00002EB800080F8DC1E9DF80800A12100EB67
:10C0B000C00202EB002008EBC0029DF8100000EB6C
:10C0C000401002EB800080F8DA1E04E49DF80800BE
:10C0D00000EBC00101EB002007EBC00080F8D35E4D
:10C0E0009DF8080000EBC00101EB002007EBC00148
:10C0F0009DF8100000EB401001EB800090F8D80E86
:10C1000005289DF8080000EBC00101EB00200CD0D1
:10C1100007EBC0019DF8100000EB401001EB800020
:10C1200090F8D80E092806D016E007EBC00080F87A
:10C13000D35E062100E00A219DF8080000EBC00252
:10C1400002EB002007EBC0029DF8100000EB40104E
:10C1500002EB800080F8D81E9DF8080000EBC001BB
:10C1600001EB002007EBC0019DF8100000EB401030
:10C1700001EB800090F8DC0EA42821D19DF8080086
:10C1800000EB400101EB00109DF8101007EB0010D0
:10C1900000EB011090F8421A41F0200180F8421A99
:10C1A0009DF8080000EBC00101EB002007EBC00187
:10C1B0009DF8100000EB401001EB800080F8155F47
:10C1C000A12130E79DF8080000EBC00101EB002041
:10C1D00007EBC0019DF8100000EB401001EB800060
:10C1E00090F8D80E012876D09DF8080000EBC00129
:10C1F00001EB002007EBC0019DF8100000EB4010A0
:10C2000001EB800090F8D80E07289DF8080000EB9D
:10C21000C00101EB002042D007EBC0019DF81000E7
:10C2200000EB401001EB800090F8D80E0B289DF831
:10C23000080000EBC00101EB002036D007EBC00185
:10C240009DF8100000EB401001EB800090F8D80E34
:10C250000C289DF8080000EBC00101EB00203BD04A
:10C2600007EBC0019DF8100000EB401001EB8000CF
:10C2700090F8D80E0E2846D09DF8080000EBC001BB
:10C2800001EB002007EBC0019DF8100000EB40100F
:10C2900001EB800090F8D80E0F2873D099E507EBDA
:10C2A000C00080F8D35E08211BE007EBC00080F8D7
:10C2B000D35E9DF808000C2100EBC00202EB0020C9
:10C2C00007EBC0029DF8100000EB401002EB80006D
:10C2D00080F8D81E74E7FCE307EBC00080F8D35E5B
:10C2E0000D219DF8080000EBC00202EB002007EBD7
:10C2F000C0029DF8100000EB401002EB800080F8B7
:10C30000D81EA3218FE69DF808000F2100EBC00284
:10C3100002EB002007EBC0039DF8100000EB40107B
:10C3200003EB800080F8D81E9DF80800A12100EBE7
:10C33000C00202EB002007EBC0039DF8100000EBE9
:10C34000401003EB800080F8DC1E9DF8080000EB35
:10C35000C00202EB002007EBC0039DF8100000EBC9
:10C36000401003EB800080F8DA1E9DF8080000EB17
:10C37000400101EB00109DF8101007EB001000EBDE
:10C380000110FDE3FDE39DF80800A32100EBC002CE
:10C3900002EB002007EBC0029DF8100000EB4010FC
:10C3A00002EB800080F8DC1E9DF8080000EBC00165
:10C3B00001EB002007EBC0019DF8100000EB4010DE
:10C3C00001EB800090F8DA0EA2283DD101E59DF83E
:10C3D0000800A12100EBC00202EB002007EBC00225
:10C3E0009DF8100000EB401002EB800080F8DC1E8E
:10C3F0009DF8080000EBC00101EB002008EBC00035
:10C4000080F8D34EE5E49DF80800A12100EBC002BE
:10C4100002EB002007EBC0029DF8100000EB40107B
:10C4200002EB800080F8DA1E9DF8080000EBC002E5
:10C4300002EB002007EBC0029DF8100000EB40105B
:10C4400002EB800080F8DC1EFDE39DF8080000EBA5
:10C45000C00101EB002007EBC0019DF8100000EBCC
:10C46000401001EB800090F8D80E0628AED19DF860
:10C47000080000EBC00101EB002007EBC00080F8D2
:10C48000D35E9DF80800072100EBC00202EB0020FC
:10C4900007EBC0029DF8100000EB401002EB80009B
:10C4A00080F8D81EA721BEE59DF8080000EBC0016A
:10C4B00001EB002007EBC00080F8D35E9DF8080078
:10C4C000A72100EBC00202EB002007EBC0029DF8A1
:10C4D000100000EB401002EB800080F8DC1E9DF89D
:10C4E00008004B4600EB4001C1EBC01009EBC00057
:10C4F000407930289DF8080000EB400146D0C1EBA0
:10C50000C01003EBC000407931289DF808007CD0B2
:10C5100000EB4001C1EBC01003EBC00040793328B1
:10C520009DF8080000EB400170D0C1EBC01003EB98
:10C53000C000407934289DF8080000EB400101EB71
:10C5400000109DF8101007EB001000EB011090F8A0
:10C55000421A73D021F0010180F8421A9DF80800B8
:10C5600000EB400101EB001007EB00119DF81000FB
:10C5700001EB001191F8420A20F0020281F8422AF0
:10C580000020CDE900008DF82850CCE101EB00102F
:10C590009DF8101007EB001000EB011090F8421A04
:10C5A00021F0010180F8421A9DF8080000EB4001DB
:10C5B00001EB00109DF8101007EB001000EB0110CC
:10C5C00090F8421A21F0020180F8421A9DF8080002
:10C5D00000EBC00101EB002007EBC0019DF810004B
:10C5E00000EB401001EB800090F8DB0E3128C7D142
:10C5F0009DF8080000EB400101EB00109DF81010C1
:10C6000007EB001000EB011001E018E01FE190F8CB
:10C61000421A21F0200180F8421A9DF8080000EB30
:10C62000C00101EB002007EBC0019DF8100000EBFA
:10C63000401001EB800080F8155FA1E729E100EBD5
:10C64000C00101EB002007EBC0019DF8100000EBDA
:10C65000401001EB800090F8160F00289DF80800AC
:10C6600000EBC00101EB002007EBC0019DF81000BA
:10C6700000EB401001EB80007DD080F8155F9DF845
:10C68000080000EB400101EB001007EB00119DF8E2
:10C69000100001EB001191F8420A20F0010281F82C
:10C6A000422A9DF8080000EB400101EB00109DF8C4
:10C6B000101007EB001000EB011090F8421A21F067
:10C6C000020180F8421A97F821060028B5D1387D7A
:10C6D0000128B2D1786DF98A8842AED29DF808005F
:10C6E00000EBC00101EB00209DF8101007EBC0002B
:10C6F00001EB411100EB810090F8150F01289CD14E
:10C700009DF8080000EBC00101EB002007EBC00121
:10C710009DF8100000EB401001EB800090F8490FED
:10C7200000288AD19DF808004FF0104100EBC002AC
:10C7300002EB002007EBC0029DF8100000EB401058
:10C7400002EB8000C0F8E01E9DF8080000EB4001FD
:10C7500001EB001007EB00119DF8100001EB001039
:10C7600090F8401A9DF8080000EBC00202EB002090
:10C7700007EBC00001E056E09CE180F8D11E9DF877
:10C78000080000EBC00101EB002007EBC0019DF8A1
:10C79000100000EB401001EB800090F8D81E9DF8CF
:10C7A000080000EBC00202EB002007EBC00090F88D
:10C7B000D40E81428AD19DF8080000EBC00101EB44
:10C7C000002007EBC0019DF8100000EB401001EBCA
:10C7D000800080F8DD5E9DF80800A42100EBC00217
:10C7E00002EB002007EBC0029DF8100000EB4010A8
:10C7F00002EB800080F8DA1EA3219DF8080003E018
:10C80000CDE3F8E3F8E3F8E300EBC00202EB00202D
:10C8100007EBC0029DF8100000EB401002EB800017
:10C8200080F8DC1EACE680F8154F9DF8080000EBA0
:10C83000400101EB001007EB00119DF8100001EB27
:10C84000001191F8420A40F0010228E75DE301EB94
:10C8500000109DF8101007EB001000EB011090F88D
:10C86000421A41F0010180F8421A9DF8080000EBDD
:10C87000400101EB00109DF8101007EB001000EBD9
:10C88000011090F8421A41F0020180F8421AA221E8
:10C8900016E021F0200180F8421A9DF8080000EB14
:10C8A000400101EB00109DF8101007EB001000EBA9
:10C8B000011090F8421A21F0020180F8421AA921D1
:10C8C0009DF8080000EBC00202EB00209DF810204C
:10C8D00007EBC00002EB421200EB820080F8DA1E88
:10C8E0004EE6DDE90001090141EA10710001CDE9E0
:10C8F00000019DF8080000EB4001C1EBC0109DF85D
:10C90000281003EBC00008448079DDE9002C3038A2
:10C91000C117104341EA0C01CDE900019DF8280040
:10C92000401C8DF828009DF828000628D9D39DF8D2
:10C930000800009900EBC00202EB002007EBC002E8
:10C940009DF8100000EB401002EB8000C0F8F11ED3
:10C950000021CDE900118DF8285021E0DDE900101B
:10C96000000140EA11700901CDE900109DF80800AE
:10C9700000EB4001C1EBC0109DF8281003EBC00094
:10C980000844407BDDE9002C3038C117104341EAF0
:10C990000C01CDE900019DF82800401C8DF828000D
:10C9A0009DF828000428D9D39DF80800009900EBD1
:10C9B000C00202EB002007EBC0029DF8100000EB64
:10C9C000401002EB8000C0F80C1F0021CDE90011DF
:10C9D0008DF8285021E0DDE90001090141EA1071DC
:10C9E0000001CDE900019DF8080000EB4001C1EB1A
:10C9F000C0109DF8281003EBC0000844407CDDE91E
:10CA0000002C3038C117104341EA0C01CDE9000178
:10CA10009DF82800401C8DF828009DF82800062865
:10CA2000D9D39DF80800009900EBC00202EB00206A
:10CA300007EBC0029DF8100000EB401002EB8000F5
:10CA4000C0F8F51E9DF8080000EB4001C1EBC010D6
:10CA500003EBC00041799DF8080000EBC00202EB37
:10CA6000002007EBC0029DF8100000EB401002EB25
:10CA7000800080F8DB1E9DF8080000EB400101EB10
:10CA8000001007EB00119DF8100001EB001090F86A
:10CA9000421A9DF8080000EBC00202EB002007EBF1
:10CAA000C0029DF8100000EB401002EB800080F8FF
:10CAB000F01E8BE49DF8080000EBC00101EB0020A4
:10CAC00007EBC00080F8D35E9DF8080000EBC001C2
:10CAD00000E046E301EB002007EBC0019DF81000E9
:10CAE00000EB401001EB800090F8D80E0A286DD0C2
:10CAF0009DF8080000EBC00101EB00209DF810102C
:10CB000007EBC00001EB411100EB810090F8D81E4B
:10CB10009DF8080000EBC00202EB002007EBC0000C
:10CB200090F8D40E814214D197F8210650B39DF8A5
:10CB3000080000EB400101EB00109DF8101007EB1E
:10CB4000001000EB011090F8421A41F0080280F842
:10CB5000422A9DF80800A72100EBC00202EB00204A
:10CB600007EBC0029DF8100000EB401002EB8000C4
:10CB700080F8DC1E9DF80800A22100EBC00202E054
:10CB800034E34CE334E002EB002007EBC0029DF8F5
:10CB9000100000EB401002EB800080F8DA1E9DF8D8
:10CBA000080000EBC00101EB002007EBC0019DF87D
:10CBB000100000EB401001EB800080F8165F0021B0
:10CBC000CDE900118DF82850CC469BE09DF8080077
:10CBD0000B2100EBC00202EB002007EBC0029DF826
:10CBE000100000EB401002EB800080F8D81EB0E788
:10CBF000C7F835509DF8080000EBC00101EB00209C
:10CC000007EBC0019DF81000102200EB401001EB73
:10CC1000800101F6F9610798FBF713FB9DF8080006
:10CC200000EBC00101EB002007EBC0019DF81000F4
:10CC300000EB401001EB8000D0F8F11EC7F819108E
:10CC4000D0F8F50E00E0FFE2C7F81D009DF80800DF
:10CC500000EB400101EB001007EB00119DF8100004
:10CC600001EB001090F8400A38769DF8080000EBC0
:10CC7000C00101EB002007EBC0019DF8100000EBA4
:10CC8000401001EB8000D0F80C0FC7F82100FE48DF
:10CC9000D0F86812C7F83910B0F86C02A7F83D0058
:10CCA000786D81B20220FCF72BF900210620FCF7F9
:10CCB0003BFF786D401C786500210520FCF734FFB0
:10CCC00047E7DDE90001090141EA10710001CDE902
:10CCD00000019DF8080000EB4001C1EBC0109DF879
:10CCE00028100CEBC0000844C07ADDE9002330387E
:10CCF000C11710431943CDE900019DF82800401CDD
:10CD00008DF828009DF828000A28DAD3DDE9001202
:10CD10009DF8080000EBC00303EB002007EBC00305
:10CD20009DF8100000EB401003EB8000C0F8F91EE6
:10CD3000C0F8FD2E0021CDE900118DF8285020E02B
:10CD4000DDE90001090141EA10710001CDE90001AE
:10CD50009DF8080000EB4001C1EBC0109DF82810C1
:10CD60000CEBC0000844407DDDE900233038C117DA
:10CD700010431943CDE900019DF82800401C8DF8AF
:10CD800028009DF828000A28DAD3DDE900129DF872
:10CD9000080000EBC00303EB002007EBC0039DF885
:10CDA000100000EB401003EB8000C0F8011FC0F83A
:10CDB000052F7EE69DF8080000EB4001C1EBC01096
:10CDC00059461BF83000042809D09DF8080000EBF4
:10CDD0004002C2EBC01011F83000152801D1ADF8A7
:10CDE00018009DF80800D94600EB4002C2EBC010C5
:10CDF00001EBC00042789DF8080000EB4003C3EB54
:10CE0000C01011F8300042EA0020A0F580513039FE
:10CE100022D09DF8080000EB4001C1EBC01009EBE7
:10CE2000C000494642789DF8080000EB4003C3EB80
:10CE3000C01019F8300042EA0022A2F580503138C3
:10CE40000CD09DF8080000EB4002C2EBC01011F8B6
:10CE50003000022804D019E0A62015E0A72013E036
:10CE60009DF8080000EB4002C2EBC01001EBC000CF
:10CE700002799DF8080000EB4003C3EBC01009EBFA
:10CE8000C000C07842EA0020ADF818009DF8080004
:10CE9000474600EBC00101EB002008EBC00090F812
:10CEA000D21E8DF810109DF8080008EB00119DF8B7
:10CEB0001000084480F8D059BDF81800A7287DD08C
:10CEC00007DC04287BD015287AD0A62842F0A68457
:10CED00037E000F51D60B0F5804004D0112870D017
:10CEE0001228F3D1F6E39DF8080000EBC00101EB36
:10CEF000002007EBC0019DF8100000EB401001EB93
:10CF0000800090F8D80E0028E0D19DF8080000EBD2
:10CF1000C00101EB002007EBC00080F8D35E9DF854
:10CF2000080000EBC00101EB002007EBC0019DF8F9
:10CF3000100000EB401001EB800080F8D84EFFF7A6
:10CF4000B1BA9DF8080000EBC00101EB002007EB2F
:10CF5000C00080F8D35E9DF8080000EBC00101EB33
:10CF6000002007EBC0019DF8100000EB401001EB22
:10CF7000800090F8D80E022840D09DF8080000EB01
:10CF8000C00101EB002007EBC0019DF8100000EB91
:10CF9000401001EB800090F8D80E052841D09DF894
:10CFA000080000EBC00101EB002007EBC0019DF879
:10CFB000100000EB401001EB800003E044E087E04C
:10CFC0004CE16DE190F8DC0EA5287FF431A89DF8C6
:10CFD000080000EB400101EB00109DF8101007EB7A
:10CFE000001000EB011090F8421A41F0040180F8A3
:10CFF000421AFFF71DB8FBE301E013E003219DF89F
:10D00000080000EBC00202EB002007EBC0029DF815
:10D01000100000EB401002EB800080F8D81EA92120
:10D02000E6E306219DF8080000EBC00202EB0020B9
:10D0300007EBC0029DF8100000EB401002EB8000EF
:10D0400080F8D81EA221D3E39DF8080000EBC001B0
:10D0500001EB002007EBC0019DF8100000EB401031
:10D0600001EB800090F8DC0EA42825D19DF8080083
:10D0700000EB400101EB00109DF8101007EB0010D1
:10D0800000EB011002E00000D410002090F8421ADA
:10D0900041F0200180F8421A9DF8080000EBC00121
:10D0A00001EB002007EBC0019DF8100000EB4010E1
:10D0B00001EB800080F8155F9DF8080000EBC001CF
:10D0C00001EB002007EBC00080F8D35EFFF778B8D3
:10D0D0009DF8080000EBC00101EB002007EBC00148
:10D0E0009DF8100000EB401001EB800090F8D80E86
:10D0F000012836D09DF8080000EBC00101EB0020AC
:10D1000007EBC0019DF8100000EB401001EB800020
:10D1100090F8D80E04289DF8080000EBC00101EB40
:10D1200000202BD007EBC0019DF8100000EB401051
:10D1300001EB800090F8D80E06289DF8080000EB5F
:10D14000C00101EB00201FD007EBC0019DF81000CB
:10D1500000EB401001EB800090F8D80E07285ED05D
:10D16000A7E49DF8080000EBC00101EB002007EBED
:10D17000C00080F8D35E0221FFF7B3B807EBC00010
:10D1800080F8D35E0521F7E707EBC00080F8D35E97
:10D190009DF80800072100EBC00202EB002007EB1E
:10D1A000C0029DF8100000EB401002EB800080F8F8
:10D1B000D81E9DF80800A12100EBC00202EB002060
:10D1C00007EBC0029DF8100000EB401002EB80005E
:10D1D00080F8DC1E9DF8080000EB400101EB001018
:10D1E00007EB00119DF8100001EB001090F8421AB7
:10D1F00041F0800180F8421A9DF8080000EB4001E0
:10D2000001EB00109DF8101008EB001000EB01106E
:10D2100090F8421A41F0040180F8421A49E49DF85E
:10D22000080000EBC00101EB002007EBC0019DF8F6
:10D23000100000EB401001EB800090F8DA0EA128FE
:10D240003FF4C5A8FFF79FB89DF8080000EBC001A8
:10D2500001EB002008EBC000FEF738BB9DF808008A
:10D26000A12100EBC00202EB002007EBC0029DF8F9
:10D27000100000EB401002EB800080F8DC1E9DF8EF
:10D28000080000EBC00202EB002007EBC0029DF893
:10D29000100000EB401002EB800080F8DA1ED3E7AC
:10D2A0009DF8080000EBC00101EB002007EBC00077
:10D2B00080F8D35E9DF80800A72100EBC00202EBC6
:10D2C000002007EBC0029DF8100000EB401002EBBD
:10D2D000800080F8DC1E9DF808004B4600EB400102
:10D2E000C1EBC01009EBC000407930289DF8080060
:10D2F00000EB400151D0C1EBC01003EBC0004079FE
:10D3000031289DF808007DD000EB4001C1EBC01032
:10D3100003EBC000407933289DF8080000EB400182
:10D3200071D0C1EBC01003EBC000407934289DF8E8
:10D33000080000EB400167D0C1EBC01003EBC00058
:10D340004079352872D09DF8080000EB400101EBD0
:10D3500000109DF8101007EB001000EB011090F882
:10D36000421A21F0010180F8421A9DF8080000EBF2
:10D37000400101EB001007EB00119DF8100001EBDC
:10D38000001191F8420A20F0020281F8422A00209E
:10D39000CDE900008DF82850D1E101EB00109DF897
:10D3A000101007EB001000EB011090F8421A21F06A
:10D3B000010180F8421A9DF8080000EB400101EBE2
:10D3C00000109DF8101007EB001000EB011090F812
:10D3D000421A21F0020180F8421A9DF8080000EB81
:10D3E000C00101EB002007EBC0019DF8100000EB2D
:10D3F000401001EB800090F8DB0E3128C7D19DF87A
:10D40000080002E013E013E134E100EB400101EB1E
:10D4100000109DF8101007EB001000EB011090F8C1
:10D42000421A21F0200180F8421AB0E753E100EBE4
:10D43000C00101EB002007EBC0019DF8100000EBDC
:10D44000401001EB800090F8160F00289DF80800AE
:10D4500000EBC00101EB002007EBC0019DF81000BC
:10D4600000EB401001EB80007DD080F8155F9DF847
:10D47000080000EB400101EB001007EB00119DF8E4
:10D48000100001EB001191F8420A20F0010281F82E
:10D49000422A9DF8080000EB400101EB00109DF8C6
:10D4A000101007EB001000EB011090F8421A21F069
:10D4B000020180F8421A97F821060028B5D1387D7C
:10D4C0000128B2D1786DF98A8842AED29DF8080061
:10D4D00000EBC00101EB00209DF8101007EBC0002D
:10D4E00001EB411100EB810090F8150F01289CD150
:10D4F0009DF8080000EBC00101EB002007EBC00124
:10D500009DF8100000EB401001EB800090F8490FEF
:10D5100000288AD19DF808004FF0104100EBC002AE
:10D5200002EB002007EBC0029DF8100000EB40105A
:10D5300002EB8000C0F8E01E9DF8080000EB4001FF
:10D5400001EB001007EB00119DF8100001EB00103B
:10D5500090F8401A9DF8080000EBC00202EB002092
:10D5600007EBC00000E050E080F8D11E9DF80800F5
:10D5700000EBC00101EB002007EBC0019DF810009B
:10D5800000EB401001EB800090F8D81E9DF80800D9
:10D5900000EBC00202EB002007EBC00090F8D40EB5
:10D5A00081428BD19DF8080000EBC00101EB002007
:10D5B00007EBC0019DF8100000EB401001EB80006C
:10D5C00080F8DD5E9DF80800A42100EBC00202EBAC
:10D5D000002007EBC0029DF8100000EB401002EBAA
:10D5E000800080F8DA1E9DF80800A32100EBC0023D
:10D5F00002EB002007EBC0029DF8100000EB40108A
:10D6000002EB800080F8DC1EC1E680F8154F9DF823
:10D61000080000EB400101EB001007EB00119DF842
:10D62000100001EB001191F8420A40F001022EE7D0
:10D6300001EB00109DF8101007EB001000EB01103B
:10D6400090F8421A41F0010180F8421A9DF8080052
:10D6500000EB400101EB00109DF8101007EB0010EB
:10D6600000EB011090F8421A41F0020180F8421AD2
:10D67000A22120E001EB00109DF8101007EB001034
:10D6800000EB011090F8421A21F0200180F8421AB4
:10D690009DF8080000EB400101EB00109DF8101010
:10D6A00007EB001000EB011090F8421A21F0020184
:10D6B00080F8421AA9219DF8080000EBC00202EB95
:10D6C00000209DF8102007EBC00002EB421200EB97
:10D6D00082000FE0B4E09DF80800A12100EBC00239
:10D6E00002EB002007EBC0029DF8100000EB401099
:10D6F00002EB800080F8DA1E49E6DDE9000109014D
:10D7000041EA10710001CDE900019DF8080000EB2D
:10D710004001C1EBC0109DF8281003EBC000084485
:10D720008079DDE9002C3038C117104341EA0C0143
:10D73000CDE900019DF82800401C8DF828009DF8D7
:10D7400028000828D9D39DF80800009900EBC002F2
:10D7500002EB002007EBC0029DF8100000EB401028
:10D7600002EB8000C0F8F11E0021CDE900118DF818
:10D77000285021E0DDE90001090141EA10710001B2
:10D78000CDE900019DF8080000EB4001C1EBC0109D
:10D790009DF8281003EBC0000844C07BDDE9002C95
:10D7A0003038C117104341EA0C01CDE900019DF862
:10D7B0002800401C8DF828009DF828000628D9D3A1
:10D7C0009DF80800009900EBC00202EB002007EB77
:10D7D000C0029DF8100000EB401002EB8000C0F882
:10D7E0000C1F0022CDE9002211468DF8285021E0BF
:10D7F0000EE20098090141EA10710001CDE9000133
:10D800009DF8080000EB4001C1EBC0109DF8281006
:10D8100003EBC0000844407DDDE9002C3038C1171F
:10D82000104341EA0C01CDE900019DF82800401C9D
:10D830008DF828009DF828000828DAD3FFF7F1B802
:10D840009DF8080000EBC00101EB002007EBC000D1
:10D8500080F8D35E9DF8080000EBC00101EB0020CA
:10D8600007EBC0019DF8100000EB401001EB8000B9
:10D8700090F8D80E03286BD09DF8080000EBC0018B
:10D8800001EB00209DF8101007EBC00001EB4111E7
:10D8900000EB810090F8D81E9DF8080000EBC00254
:10D8A00002EB002007EBC00090F8D40E814214D1A7
:10D8B00097F82106F0B39DF8080000EB400101EB5A
:10D8C00000109DF8101007EB001000EB011090F80D
:10D8D000421A41F0080280F8422A9DF8080000EB45
:10D8E000C00101EB002007EBC0019DF8100000EB28
:10D8F000401001EB800080F8165F9DF80800A7211A
:10D9000000EBC00202EB002007EBC0029DF8100004
:10D9100000EB401002EB800080F8DC1E9DF8080050
:10D92000A22100EBC00202EB002007EBC0029DF831
:10D93000100000E01EE000EB401002EB800080F8D9
:10D94000DA1E0021CDE900118DF82850CC4699E06F
:10D950009DF80800042100EBC00202EB002007EB59
:10D96000C0029DF8100000EB401002EB800080F830
:10D97000D81EB2E7C7F835509DF8080000EBC0018B
:10D9800001EB002007EBC0019DF81000102200EB16
:10D99000401001EB800101F6F9610798FAF751FC9C
:10D9A0009DF8080000EBC00101EB002007EBC0016F
:10D9B0009DF8100000EB401001EB8000D0F8F11E44
:10D9C000C7F81910D0F8F50EC7F81D009DF808002B
:10D9D00000EB400101EB001007EB00119DF8100077
:10D9E00001EB001090F8400A38769DF8080000EB33
:10D9F000C00101EB002007EBC0019DF8100000EB17
:10DA0000401001EB8000D0F80C0FC7F82100FE4851
:10DA1000D0F86812C7F83910B0F86C02A7F83D00CA
:10DA2000786D81B20220FBF76BFA00210620FCF72B
:10DA30007BF8786D401C786500210520FCF774F8B0
:10DA40004BE7DDE90001090141EA10710001CDE970
:10DA500000019DF8080000EB4001C1EBC0109DF8EB
:10DA600028100CEBC0000844C07ADDE900233038F0
:10DA7000C11710431943CDE900019DF82800401C4F
:10DA80008DF828009DF828000C28DAD3DDE9001273
:10DA90009DF8080000EBC00303EB002007EBC00378
:10DAA0009DF8100000EB401003EB8000C0F8F91E59
:10DAB000C0F8FD2E0021CDE900118DF8285020E09E
:10DAC000DDE90001090141EA10710001CDE9000121
:10DAD0009DF8080000EB4001C1EBC0109DF8281034
:10DAE0000CEBC0000844C07DDDE900233038C117CD
:10DAF00010431943CDE900019DF82800401C8DF822
:10DB000028009DF828000C28DAD3FFF73EB99DF8CD
:10DB1000080043469DF8101008EB0010084480F8F8
:10DB2000D0599DF80800DC4600EB4001C1EBC01065
:10DB30000BEBC000407870280AD19DF8080000EB7C
:10DB40004001C1EBC0100CEBC0008078FA282ED049
:10DB50009DF8080000EB4001C1EBC0100CEBC000C9
:10DB600040789DF8080000EB4001C1EBC0101CF8A4
:10DB700030009DF8080000EBC00101EB002003EB32
:10DB8000C00090F8D21E8DF810109DF8080003EB2D
:10DB900000119DF81000084480F8D059BDF8180015
:10DBA00001283FD0652847D0B12844D103E0B120F7
:10DBB000ADF81800DDE79DF8080000EBC00101EBAF
:10DBC000002003EBC0019DF8100000EB401001EBBA
:10DBD000800090F8D80E0028E7D19DF8080000EBEF
:10DBE000C00101EB002003EBC00080F8D35E9DF87C
:10DBF000080000EBC00101EB002003EBC0019DF821
:10DC0000100000EB401001EB800080F8D84EB821E6
:10DC10009DF8080000EBC00202EB002008EBC002F8
:10DC2000FDF74BBE9DF8080000EB4001C1EBC010B2
:10DC30000BEBC0000079B7E39DF8080000EB400152
:10DC4000C1EBC0100CEBC0000079B922ADF8182070
:10DC50009DF8080000EB4001C1EBC0100CEBC000C8
:10DC6000007900F00F018DF814108DF828501DE098
:10DC70009DF8080000EB400101EB001003EB0011E0
:10DC80009DF8280001EB001090F8411A9DF808005B
:10DC900000EB4007C7EBC0101CF830005038814241
:10DCA00012D09DF82800401C8DF828009DF808002F
:10DCB00000EB400101EB001003EB001090F8170A95
:10DCC0009DF828108842D3D89DF828009DF814109C
:10DCD00008448DF810009DF8080000EBC00101EB2E
:10DCE000002003EBC0079DF8100000EB401007EB8D
:10DCF000800090F8D80E012811D09DF8080000EBA4
:10DD0000C00101EB002003EBC0019DF8100000EB07
:10DD1000401001EB800090F8D80E01288BD19DF8BF
:10DD2000080000EBC00101EB002003EBC00080F80D
:10DD3000D35E9DF80800022100EBC00707EB00202E
:10DD400003EBC0079DF8100000EB401007EB8000CC
:10DD500080F8D81E9DF8080000EBC00101EB002000
:10DD6000FAE39DF8080000EB400101EB001008EB1E
:10DD7000001090F81C0A20B101287CD00228CDD1D7
:10DD800067E29DF8080008EB400000F50050B0F88D
:10DD9000F00F801F81B29DF808005F4600EB400243
:10DDA000C2EBC0120BEBC200401CFBF733FCCDE909
:10DDB00012059DF8080008EB400000F50050B0F88F
:10DDC000F01F9DF80800394400EB4002C2EBC01080
:10DDD0006FF0040202EBC0000844042107F056FB78
:10DDE000DDE91223C117CDE9000150405940084335
:10DDF00094D19DF8080008EB001080F8D0599DF8E8
:10DE0000080000EB400101E0D4100020C1EBC0117C
:10DE100007EBC100B9460079ADF81800BDF818004D
:10DE20003128ACD19DF8080008EB400000F5005007
:10DE3000B0F8F00F4121183890FBF1F0C217CDE98E
:10DE4000000288F804048DF828502F46BBE09DF8A6
:10DE5000080000EB4001C1EBC0119DF8280009EB60
:10DE6000C10100EB80100844007D9DF8281041445A
:10DE700081F8050400E0B0E09DF8080000EB4001E7
:10DE8000C1EBC0119DF8280009EBC10100EB801027
:10DE9000084408211A3007F0C5FA8DED090A10EE82
:10DEA000100A9DF8281008EB0111C1F815049DF81F
:10DEB000080000EB4001C1EBC0119DF8280009EB00
:10DEC000C10100EB801008440821323007F0AAFAA3
:10DED0008DED090A10EE100A9DF8281008EB0111CB
:10DEE000C1F811049DF8080000EB4001C1EBC0111E
:10DEF0009DF8280009EBC10100EB801008440821BF
:10DF00003A3007F08FFA8DED090A10EE100A9DF8ED
:10DF1000281008EB0111C1F819049DF8080000EB66
:10DF20004001C1EBC01109EBC1009DF8281001EBC5
:10DF3000811108440821423007F074FA8DED090A76
:10DF400010EE100A9DF8281008EB0111C1F81D040D
:10DF50009DF8080000EB400101EB00109DF828102F
:10DF600008EB001000EB011090F8421A41F080011C
:10DF700080F8421A9DF8080008EB400000F50050B8
:10DF8000B0F8F01F9DF80800494400EB4002C2EBD6
:10DF9000C0104FF0FF3202EBC000095C9DF8080092
:10DFA00000EBC00202EB002008EBC0039DF810005C
:10DFB00000EB401003EB800080F8141F9DF8280050
:10DFC000401C8DF828009DF82800DDE90012401A59
:10DFD00077EB0200FFF43BAF2DE69DF808005F46AB
:10DFE00000EB4001C1EBC0100BEBC000437D9DF87E
:10DFF000080000EB4002C2EBC0100BEBC000807DBC
:10E0000043EA0020C317CDE900039DF8080015215D
:10E0100000EB4002C2EBC0100BEBC000FBF7E4FAD0
:10E02000CDE91205DDE90001129B69405840084323
:10E03000D2D19DF8080000EB4001C1EBC011384679
:10E0400017F83120521E8DF810209DF8081008EBAB
:10E0500001129DF81010114481F8D0599DF810104C
:10E06000414481F805549DF8101008EB0111C1F8E6
:10E0700015549DF8081001EB4102C2EBC11100EBF1
:10E08000C1018A799DF8081001EB4103C3EBC1116E
:10E0900000EBC101497942EA012100EE101AF8EEC5
:10E0A000400A9FEDFA0A9DF8081080EE801A01EBF5
:10E0B0004102C2EBC11100EBC1010A799DF80810C1
:10E0C00001EB4103C3EBC11100EBC101C97842EA86
:10E0D000012100EE901A9DF81010F8EE600A71EE22
:10E0E000200A10EE902A08EB0111C1F811249DF8C6
:10E0F000081001EB4102C2EBC11100EBC1018A7AA9
:10E100009DF8081001EB4103C3EBC11100EBC10105
:10E11000497A42EA012100EE901A9DF80810B8EE03
:10E12000601AC1EE000A01EB4102C2EBC11100EB23
:10E13000C1010A7A9DF8081001EB4103C3EBC1113C
:10E1400000EBC101C97942EA012100EE101A9DF8E5
:10E150001010B8EE400A30EE800A10EE102A08EBDC
:10E160000111C1F819249DF8081001EB4102C2EB1E
:10E17000C11100EBC100C07A00069DF8080000EB59
:10E180004001C1EBC01018D407EBC000027B9DF822
:10E19000080000EB4003C3EBC01007EBC000C07ADF
:10E1A00042EA002000EE100AB8EE400ADFEDB80A9D
:10E1B00020EE200A10EE100A19E007EBC000037BE6
:10E1C0009DF8080000EB4001C1EBC01007EBC00058
:10E1D000C07A43EA0020404280B2FAF7EEF99FEDA0
:10E1E000AD1B53EC112BFAF707F9FAF736FA9DF845
:10E1F000101008EB0111C1F81D049DF8080000EB98
:10E20000400101EB00109DF8101008EB001000EB2E
:10E21000011090F8421A41F0800180F8421A9DF8EE
:10E22000080000EB4001C1EBC01107EBC100C17D4C
:10E230009DF8080000EBC00202EB002008EBC002D2
:10E240009DF8100000EB401002EB800080F8141FD6
:10E25000B7E09DF808005F4600EB4001C1EBC0103D
:10E260000BEBC000C3799DF8080000EB4002C2EB45
:10E27000C0100BEBC000007A43EA0020C317CDE9C1
:10E2800000039DF80800072100EB4002C2EBC0101C
:10E290000BEBC000FBF7A8F9CDE91205DDE90001A1
:10E2A000129B6940584008437ED19DF8080000EB5E
:10E2B0004001C1EBC01117F83100401E8DF810006D
:10E2C0009DF8080008EB001080F8D0599DF8100068
:10E2D000404480F805549DF8080000EB4001C1EB74
:10E2E000C01107EBC1008079FAF767F941EC110B17
:10E2F0009FED6A0B09F028FA9DF80800B0EE408AFD
:10E30000F0EE608A00EB4001C1EBC01107EBC100E9
:10E3100002799DF8080000EB4001C1EBC01107EB4A
:10E32000C100C07842EA0020FAF747F953EC182BF5
:10E33000FAF7D4F8FAF791F99DF8101008EB0111EB
:10E34000C1F815049DF8100008EB0010C0F8115436
:10E350009DF8100008EB0010C0F819549DF810004B
:10E3600008EB0010C0F81D549DF8080000EB4001B8
:10E3700001EB00109DF8101008EB001000EB0110ED
:10E3800090F8421A41F0800280F8422A9DF8080075
:10E3900000EB4001C1EBC01107EBC100427A9DF8D0
:10E3A000080000EBC00100E004E201EB002008EBF4
:10E3B000C0039DF8100000EB401003EB800080F8D4
:10E3C000142F9DF8080000EB400101EB001008EB52
:10E3D000001090F8170A88F80404EBE19DF8080093
:10E3E00000EB4001C1EBC0100BEBC0005946C378F5
:10E3F0009DF8080000EB4002C2EBC0100BEBC00020
:10E40000807843EA00208DF80C009DF8080000EBAE
:10E410004002C2EBC0109DF80C200BEBC000104472
:10E4200043789DF8080000EB4002C2EBC0109DF855
:10E430000C2001EBC000805C43EA0020C317CDE94B
:10E4400000039DF808009DF80C1000EB4002C2EBA1
:10E45000C0100BEBC000FBF7C7F8CDE91205DDE9F2
:10E460000001129B694058400843B6D19DF808004E
:10E470005B4600EB4001C1EBC0100BEBC0004078E5
:10E480008DF810008DF82850414625E000FF7F47A9
:10E490000000803D000000000000B0BF0000000050
:10E4A000000024409DF8080000EB400202EB001041
:10E4B0009DF8282001EB001000EB021090F8410AB3
:10E4C0009DF8102090429DF8280002D18DF8100090
:10E4D00010E0401C8DF828009DF8080000EB400279
:10E4E00002EB001001EB001090F8170A9DF82820AD
:10E4F0009042D7D89DF8080000EB400202EB0010D4
:10E500009DF8102001EB001000EB021090F8422A59
:10E5100042F0800280F8422A9DF8080000EB400299
:10E52000C2EBC01003EBC0000079ADF818009DF8F5
:10E5300008009DF8102001EB0010104480F8D0591D
:10E54000BDF81800F32806D007DC052874D0F128A0
:10E5500008D0F22889D189E18FE1F4286DD0F6281E
:10E56000F8D18DE19DF8080000EBC00202EB00201D
:10E5700001EBC0029DF8100000EB401002EB8000A0
:10E5800090F8D80E00289DF8080021D000EB40023A
:10E5900002EB00109DF8102001EB001000EB0210C0
:10E5A00090F8490AC00712D09DF80800C44600EB55
:10E5B000C00202EB002008EBC0029DF8100000EB47
:10E5C000401002EB800090F8580FC00720D0A8E060
:10E5D00000EBC00202EB002001EBC0029DF810002E
:10E5E00000EB401002EB800080F8D84E9DF8080048
:10E5F000F42200EBC00707EB002001EBC0079DF8F9
:10E60000100000EB401007EB800080F8DC2E88E063
:10E610009DF8080000EBC00202EB00200CEBC002EA
:10E620009DF8100000EB401002EB800090F84A0FBC
:10E6300098B38DF8285028E092E133E19DF8080066
:10E6400000EBC00202EB00209DF810200CEBC00094
:10E6500002EB421200EB82009DF82820104490F853
:10E660004B2F9DF8080000EB400707EB00109DF8CA
:10E6700028700CEB0010384490F81E0A824208D132
:10E680009DF82800401C8DF828009DF828000428DB
:10E69000D4D39DF82800042825D042E09DF8080036
:10E6A00000EBC00202EB00200CEBC0029DF8100052
:10E6B00000EB401002EB80009DF82820104490F8F9
:10E6C0004B0F9DF8082002EB420707EB02129DF862
:10E6D00028700CEB02123A4492F81E2A904208D19C
:10E6E0009DF82800401C8DF828009DF828000A2875
:10E6F000D4D39DF828000A2813D09DF8080000EB19
:10E70000C00202EB002008EBC0029DF8100000EBF5
:10E71000401002EB800090F8582F42F0010280F880
:10E72000582F9DF80C0011289DF8080000EB4002BE
:10E7300002EB00109DF8102001EB001000EB02101E
:10E7400090F8422A37D022F0080280F8422A9DF839
:10E75000080000EBC00202EB002001EBC0029DF8B4
:10E76000100000EB401002EB800090F8580FC0073B
:10E7700020D09DF8080000EBC00202EB002001EB66
:10E78000C0029DF8100000EB401002EB8000A0F8E2
:10E79000565F9DF80800052200EBC00303EB002044
:10E7A00001EBC0019DF8100000EB401001EB800070
:10E7B00080F8DC2E36E242F0080280F8422A8DF81A
:10E7C000285023E09DF8080000EB4002C2EBC01087
:10E7D00003EBC0029DF82800104442799DF8080020
:10E7E00000EBC00707EB002001EBC0079DF810000D
:10E7F00000EB401007EB80079DF82800384480F8B4
:10E80000172F9DF82820521C8DF828209DF82800ED
:10E810000A28D7D38DF8285023E09DF8080000EB94
:10E820004002C2EBC0109DF8282003EBC00010444A
:10E83000C27B9DF8080000EBC00707EB002001EB4E
:10E84000C0079DF8100000EB401007EB80009DF81A
:10E850002870384480F8302F9DF82800401C8DF82F
:10E8600028009DF828000228D7D3DBE19DF8080096
:10E87000F12200EBC00303EB002008EBC00191E79D
:10E880009DF80800032200EBC00303EB002001EB1E
:10E89000C0039DF8100000EB401003EB800080F8EF
:10E8A000D82EE3E79DF80820022002EBC20707EB11
:10E8B000022201EBC2079DF8102002EB421207EB87
:10E8C000820282F8D80E9DF80800F62700EBC002FD
:10E8D00002EB00209DF8102001EBC00002EB421279
:10E8E00000EB820080F8DC7E9DF8080000EBC0029F
:10E8F00002EB00209DF8102001EBC00002EB421259
:10E9000000EB820080F84A4F8DF8285023E09DF8F4
:10E91000080000EB4002C2EBC0109DF8282003EB7A
:10E92000C000104442799DF8080000EBC00707EBD7
:10E93000002001EBC0079DF8100000EB401007EB32
:10E9400080009DF82870384480F84B2F9DF82800EF
:10E95000401C8DF828009DF828000A28D7D361E1D3
:10E960009DF8080000EB4002C2EBC01003EBC000B2
:10E9700082799DF8080000EB4007C7EBC0100BEB55
:10E98000C000407942EA00229DF8080000EBC00375
:10E9900003EB002001EBC0039DF8100000EB4010DA
:10E9A00003EB8000A0F8562F9DF8080000EBC00292
:10E9B00002EB002001EBC0029DF8100000EB4010BC
:10E9C00002EB8000B0F8562F9DF8080000EB4003E2
:10E9D00003EB001001EB0010B0F82A0A8242BED30C
:10E9E0009DF80800F12200EBC00303EB002001EBCF
:10E9F000C0079DF8100000EB401007EB800080F886
:10EA0000DC2E9DF8080000EBC00202EB002008EBB2
:10EA1000C0019DF8100000EB401001EB800090F861
:10EA2000581F21F0010180F8581FFBE09DF80800F5
:10EA30005A4600EB4001C1EBC0100BEBC00000795F
:10EA40008DF810008DF85450C14619E09DF808006B
:10EA500000EB400101EB00109DF8541009EB001091
:10EA600000EB011090F8410A9DF8101088429DF8C3
:10EA7000540002D18DF8100010E0401C8DF85400B5
:10EA80009DF8080000EB400101EB001009EB0010BD
:10EA900090F8170A9DF854108842D7D89DF80800BE
:10EAA00000EB4001C1EBC01002EBC000C078ADF834
:10EAB0001800BDF81800182812D2DFE800F0110C79
:10EAC0000E118E8E868E881111118A8E8E8E8E8CEE
:10EAD00011118E118E8E1A2000E00D208DF80C0081
:10EAE0009DF80C00001FC1B29DF808005F4600EBC6
:10EAF0004003C3EBC0130BEBC300C01CFAF7A2FB2F
:10EB00008DF85C009DF8080000EB4001C1EBC011DE
:10EB100007EBC1009DF80C10084410F8010C9DF89B
:10EB20005C1088427ED19DF8080000EB4001C1EBEB
:10EB3000C01107EBC10138464978002972D09DF811
:10EB4000081001EB4102C2EBC11100EBC1029DF8BC
:10EB50000C101144CA789DF8081001EBC10303EBB7
:10EB6000012109EBC1039DF8101001EB411103EBEA
:10EB7000810181F8142F9DF8081009EB01129DF80E
:10EB80001010114481F8D059BDF81810CE293CF46A
:10EB9000C4AD24DCB9293CF4F6AD7CF792A9C329B5
:10EBA0007DD0C5297CF4B5A99DF8081001EB410280
:10EBB00002EB011109EB011191F81C1A00299DF8D3
:10EBC0000C106DD00E29ADD1FEE3072086E708209A
:10EBD00084E70C2082E70A2080E706207EE7E1290F
:10EBE000D5D006DCD5293AD0D729A7D0D92999D1B3
:10EBF0007CE2E5297CF49BA989F860459DF8080032
:10EC000000EBC00101EB002009EBC0019DF81000F2
:10EC100000EB401001EB800090F8D80E00289DF822
:10EC2000080000E0F0E200EBC00101EB00207DF401
:10EC3000D1A809EBC00080F8D35E9DF8080000EB76
:10EC4000C00101EB002009EBC0019DF8100000EBB2
:10EC5000401001EB800080F8D84EFCF75EBD9DF8B7
:10EC6000081001EB4102C2EBC11107EBC100C078F3
:10EC700089F862009DF8080000EB400101EB0010EC
:10EC80009DF8101009EB001000EB011099F86210CC
:10EC9000A4EBD11290F8421A62F3000101E0F9E20C
:10ECA0005DE380F8421A9DF8080000EB400101EB9B
:10ECB00000109DF8101009EB001000EB011099F8FE
:10ECC00062104A0990F8421A62F3410180F8421A30
:10ECD0009DF8080000EB400101EB00109DF81010BA
:10ECE00009EB001000EB011090F8420AC0F340015C
:10ECF0009DF8080000EBC00202EB00209DF81020F8
:10ED000009EBC00002EB421200EB820090F8F00E1B
:10ED1000C0F34000814249D09DF808004A4600EB0C
:10ED2000C00101EB002009EBC0019DF8100000EBD1
:10ED3000401001EB80019DF8080000EB400303EB5D
:10ED400000109DF8103009EB001000EB031090F854
:10ED5000420A430891F8F00E63F3410081F8F00E87
:10ED60009DF8080000EB400101EB00109DF8101029
:10ED700002EB001000EB011090F8420A800716D554
:10ED80009DF80800D92100EBC00303EB002009EB3C
:10ED9000C0029DF8100000EB401002EB800080F8EC
:10EDA000DC1E9DF808100220FAF7BEFE42E09DF836
:10EDB000080000EBC00101EB002002EBC0019DF850
:10EDC000100000EB401001EB800080F8E54E9DF84C
:10EDD0000800D92100EBC00303EB002002EBC003C5
:10EDE0009DF8100000EB401003EB800080F8DC1E63
:10EDF0009DF8080000EB400101EB001002EB001150
:10EE00009DF8100001EB001191F8420A20F0200358
:10EE100081F8423A9DF8080000EBC00101EB0020A8
:10EE200009EBC0019DF8100000EB401001EB8000E1
:10EE300080F8164F9DF8080000EB400101EB001030
:10EE400009EB00119DF8100001EB001090F8420A48
:10EE500000F001019DF8080000EBC00202EB002069
:10EE600009EBC0029DF8100000EB401002EB80009F
:10EE700090F8F00E00F0010081426AD09DF8080081
:10EE800000EBC00101EB00209DF8101009EBC00061
:10EE900001EB411100EB81009DF8081001EB4102EC
:10EEA00002EB01119DF8102009EB011101EB021199
:10EEB00091F8421A90F8F02E61F3000280F8F02EDB
:10EEC0009DF8080000EB400101EB00109DF81010C8
:10EED00009EB001000EB011090F8420AC0073CF467
:10EEE000A7A99DF808004F4600EBC00101EB0020E8
:10EEF00009EBC0019DF8100000EB401001EB800011
:10EF000090F8160F00289DF8080000EBC00101EBF7
:10EF1000002009EBC0019DF8100000EB401001EB50
:10EF2000800017D080F8155F9DF8080000EB4001C5
:10EF300001EB001007EB00119DF8100001EB001130
:10EF400091F8420A20F0010281F8422A97F821063E
:10EF500018B1A7E080F8154FF8E7387D012865D192
:10EF6000786DF98A884261D29DF8080000EBC001F3
:10EF700001EB002007EBC0019DF8100000EB4010F2
:10EF800001EB800090F8150F01284FD19DF8080083
:10EF900000EBC00101EB002007EBC0019DF8100061
:10EFA00000EB401001EB800090F8490FF0BB9DF89A
:10EFB000080000EB400101EB001007EB00119DF889
:10EFC000100001EB001090F8401A9DF8080000EBCB
:10EFD000C00202EB002007EBC00080F8D11E9DF8B4
:10EFE0000800C32100EBC00202EB002007EBC002C7
:10EFF0009DF8100000EB401002EB800080F8DC1E52
:10F000009DF8080000EB400101EB001007EB001138
:10F010009DF8100001EB0010C0F8445A9DF808104C
:10F020000220FAF781FD8DF8285018E03AE09DF8AB
:10F03000080000EBC00101EB002007EBC0019DF8C8
:10F04000100000EB401001EB80019DF828000844FF
:10F0500080F8175F9DF82810491C8DF828109DF83E
:10F0600028001428E3D38DF8285017E09DF80800F5
:10F0700000EBC00101EB002007EBC0019DF8100080
:10F0800000EB401001EB80009DF82810084480F848
:10F09000335F9DF82800401C8DF828009DF828005B
:10F0A0000A28E3D39DF8080000EB400101EB0010B3
:10F0B0009DF8101009EB001000EB011090F8420AC7
:10F0C00080077CF581A99DF80800D92100EBC002DA
:10F0D00002EB002009EBC0029DF8100000EB40108D
:10F0E00002EB800080F8DC1EFCF76EB99DF808107A
:10F0F00001EB410202EB011109EB011191F81C1A1D
:10F1000000299DF80C1002D00A297DD193E008292E
:10F110007AD18DF8285024E09DF8081001EB4102C7
:10F12000C2EBC1119DF8282000EBC1011144C97840
:10F1300001F00F01092918D89DF8081001EB4102D0
:10F14000C2EBC1119DF8282000EBC1011144C97820
:10F1500001F0F001902908D89DF82810491C8DF87D
:10F1600028109DF828100629D6D39DF828100629C6
:10F170004AD39DF8081001EB4102C2EBC11100EB2C
:10F18000C101C9780A049DF8081001EB4103C3EBE3
:10F19000C11100EBC101097942EA01229DF8081072
:10F1A00001EB4103C3EBC11100EBC10149790A43F3
:10F1B0009DF8081001EBC10303EB012109EBC1032A
:10F1C0009DF8101001EB411103EB8101C1F8F12E04
:10F1D0009DF8081001EB4102C2EBC11100EBC10127
:10F1E00089790A049DF8081001EB4103C3EBC111B2
:10F1F00000EBC101C97942EA01229DF8081001EB38
:10F200004103C3EBC11100E022E100EBC100007A31
:10F2100002439DF8080000EBC00101EB002009EB60
:10F22000C0039DF8100000EB401003EB8000C0F815
:10F23000F52EFCF732BA8DF8285025E09DF808101D
:10F2400001EB4102C2EBC1119DF8282000EBC10186
:10F250001144C97801F00F0109293CF6B4A99DF8C1
:10F26000081001EB4102C2EBC1119DF8282000EB10
:10F27000C1011144C97801F0F0019029EDD89DF841
:10F280002810491C8DF828109DF828100829D5D37E
:10F29000FCF799B99DF8080000EBC00101EB0020D4
:10F2A00009EBC0029DF8100000EB401002EB80005B
:10F2B00080F8DC6E9DF8080000EBC00101EB002037
:10F2C00009EBC00080F8D34E9DF8080000EB400128
:10F2D00001EB00109DF8101009EB001000EB01107D
:10F2E00090F8421A41F02002FCF7F3BA0A799DF82F
:10F2F000081001EB4103C3EBC11107EBC100C0785B
:10F3000042EA0022FCF777BA9DF8080000EBC00142
:10F3100001EB002009EBC00080F8D34E9DF80800F7
:10F3200000EBC00101EB002009EBC0029DF81000CA
:10F3300000EB401002EB800080F8DC6E9DF80800C6
:10F3400000EB400101EB00109DF8101009EB0010DC
:10F3500000EB011090F8421A41F00402C4E70C29B6
:10F3600076D18DF8285024E09DF808109DF82830BB
:10F3700001EB4102C2EBC11100EBC102D118C97807
:10F3800001F00F01092918D89DF8082002EB42036B
:10F39000C3EBC21100EBC1029DF828101144C978DB
:10F3A00001F0F001902908D89DF82810491C8DF82B
:10F3B00028109DF828100A29D6D39DF828100A296C
:10F3C00046D30022134600E068E0CDE9002229463A
:10F3D0008DF828501EE0009A1B0243EA12631202C5
:10F3E000CDE900239DF8082002EB4203C3EBC212D3
:10F3F0009DF8283000EBC2021A44D278DDE90037CC
:10F400001A4341EA0703CDE900239DF82820521C46
:10F410008DF828209DF82820052ADCD3DDE9003767
:10F420009DF8082002EBC20C0CEB022209EBC20C87
:10F430009DF8102002EB42120CEB8202C2F8F93E5A
:10F44000C2F8FD7E0023CDE900338DF8281020E0BE
:10F45000D1E0DDE900231B0243EA12631202CDE989
:10F4600000239DF8082002EB4203C3EBC2129DF873
:10F47000283000EBC2021A44127ADDE900371A4341
:10F4800041EA0703CDE900239DF82820521C8DF89E
:10F4900028209DF82820052ADBD399E08DF82850F4
:10F4A00024E09DF808109DF8283001EB4102C2EBE2
:10F4B000C11100EBC102D118C97801F00F0109296F
:10F4C00018D89DF8082002EB4203C3EBC21100EBF1
:10F4D000C1029DF828101144C97801F0F00190296B
:10F4E00008D89DF82810491C8DF828109DF8281080
:10F4F0000C29D6D39DF828100C297CD30022CDE905
:10F50000002229468DF82850BC461FE0DDE90002A4
:10F51000120242EA10620002CDE900029DF80800E2
:10F5200000EB4002C2EBC0109DF828200CEBC0009D
:10F530001044C078DDE90023104341EA0302CDE91D
:10F5400000029DF82800401C8DF828009DF8280036
:10F550000628DBD3DDE900239DF8080000EBC00797
:10F5600007EB002009EBC0079DF8100000EB4010EE
:10F5700007EB8000C0F8F92EC0F8FD3E0022CDE96F
:10F5800000228DF828101FE0DDE90002120242EA95
:10F5900010620002CDE900029DF8080000EB400275
:10F5A000C2EBC0109DF828200CEBC0001044407A3C
:10F5B000DDE90023104341EA0302CDE900029DF892
:10F5C0002800401C8DF828009DF828000628DBD371
:10F5D000DDE900129DF8080000EBC00303EB0020FA
:10F5E00009EBC0039DF8100000EB401003EB800016
:10F5F000C0F8011F00E011E1C0F8052F9DF80800D8
:10F6000000EBC00101EB002009EBC0019DF81000E8
:10F6100000EB401001EB800090F8D81E9DF8080028
:10F6200000EBC00202EB002009EBC00090F8D40E02
:10F6300081427DD199F821064F46B8B19DF8080066
:10F6400000EB400101EB00109DF8101009EB0010D9
:10F6500000EB011090F8421A41F0080280F8422AAB
:10F660009DF808100220FAF75FFA78E0C7F83550E5
:10F670009DF8080000EBC00101EB002007EBC00182
:10F680009DF81000102200EB401001EB800101F604
:10F69000F9610798F8F7D5FD9DF8080000EBC00167
:10F6A00001EB002007EBC0019DF8100000EB4010BB
:10F6B00001EB8000D0F8F11EC7F81910D0F8F50E54
:10F6C000C7F81D009DF8080000EB400101EB001099
:10F6D00007EB00119DF8100001EB001090F8400AB4
:10F6E00038769DF8080000EBC00101EB002007EB25
:10F6F000C0019DF8100000EB401001EB8000D0F835
:10F700000C0FC7F821006748D0F86812C7F8391005
:10F71000B0F86C02A7F83D00786D81B20220F9F7CD
:10F72000EFFB00210620FAF7FFF9786D401C00E09E
:10F7300003E078650021052095E79DF8080000EBBF
:10F74000400101EB00109DF8101009EB001000EBD8
:10F75000011090F8421A41F0040180F8421A9DF815
:10F76000080000EBC00101EB002009EBC0019DF88F
:10F77000100000EB401001EB800080F8165F9DF850
:10F78000080000EBC00101EB002009EBC0019DF86F
:10F79000100000EB401001EB800080F8DC6E9DF85B
:10F7A000080000EBC00101EB002009EBC0019DF84F
:10F7B000100000EB401001EB800090F8D80E0428F8
:10F7C0002CD19DF8080000EB400101EB00109DF8E2
:10F7D000101009EB001000EB011090F8421A41F0F4
:10F7E000800180F8421A9DF8080000EBC00101EB8F
:10F7F000002009EBC00080F8D34E9DF808000521D9
:10F8000000EBC00202EB002009EBC0029DF81000E3
:10F8100000EB401002EB800080F8D81E98F86702D9
:10F82000A0B19DF8080008EB400000F50050B0F8CA
:10F83000F01F9DF80800012300EB4002C2EBC0124C
:10F840000BEBC2009DF80820FBF758F88DF8285004
:10F85000594613E089F86055FBF75FBF9DF8080033
:10F8600000EB4002C2EBC0109DF8282001EBC00065
:10F8700085549DF82800401C8DF828009DF828002C
:10F880001428EBD308480178427811448278114457
:10F89000C278D1427BF4EBA919B0BDEC028BBDE874
:10F8A000F08F0000D41000200F0800202DE9F74F42
:10F8B00092B04FF00008ADF82080ADF80480ADF8AC
:10F8C0000880ADF80C808DF810808DF814808DF8CC
:10F8D0001880CDE90A88CDE90A88ADF83C80FEA001
:10F8E000D0E90010CDE90C10FDA0D0E90010CDE961
:10F8F0001010FD4880F80480129800EB400101EBE5
:10F900000011FA4800EB011797F8161A8DF810103D
:10F91000129900EB0110139900900844834690F867
:10F92000D0291298042A00EBC00101EB0020EF4916
:10F9300001EBC00A1399139801EB41110AEB810501
:10F9400007EB001921D105208BF8D00985F8D88E56
:10F9500099F8420A20F0800189F8421A97F8160AAD
:10F96000A121072811D2DFE800F010040606090BD8
:10F970000D00E52007E085F8DC1E06E0B12002E07E
:10F98000312000E0F12085F8DC0E9DF810C0129BBC
:10F99000149802224121D64EC3EB0313A1384FF035
:10F9A000320E03EB8304BCF1070F7BD2DFE81CF0BF
:10F9B0007A000700B102F903750517078C0799F85B
:10F9C000410AC146002101F02DFE8DF8140095F882
:10F9D000D81E9AF8D40E814202D101218AF8D31E92
:10F9E0009BF8D009401C8BF8D009149BA221A620BB
:10F9F000CE2B7DD012DC4FF0A502B92B79D006DCDE
:10FA0000B22B77D0B52B35D0B62B4BD123E1C32BFE
:10FA100071D0C52B70D0CA2BF7D111E1E12B6CD07E
:10FA200006DCD52B09D0D72B68D0D92BEDD10FE030
:10FA3000E52B6ED0E72BE8D155E2F52006F834002F
:10FA40009DF8140006EBC4056870A970D52009E084
:10FA5000F52006F834009DF8140006EBC405687024
:10FA6000A970D920E8702846032101F00CFD287107
:10FA700005202CE2F52106F834109DF8143006EB31
:10FA8000C40188464B7097F81C1AB52759B1D5F8B0
:10FA9000E01EB1F1104F3DD34FF010410022CDE9EF
:10FAA0000A123BE0AAE2D5F8E00EB0F5100F05D33C
:10FAB0004FF410000021CDE90A0103E0D5F8E00E73
:10FAC000CDE90A0988F80220484610E0BDF8200078
:10FAD000C0F10200C200DDE90A01F8F7A2FBBDF89F
:10FAE000202008EB0201C870BDF82000401C06E091
:10FAF00054E12FE0BAE098E045E11BE1FEE1ADF80A
:10FB00002000BDF820000328E0D3404688F80670A6
:10FB100009E1DDE1D5F8E01ECDE90A1988F8020017
:10FB2000484610E0BDF82000C0F10300C200DDE946
:10FB30000A01F8F776FBBDF8202008EB0201C87037
:10FB4000BDF82000401CADF82000BDF820000428BE
:10FB5000E8D361E0F52106F834109DF8143006EB87
:10FB6000C40188464B7097F81C1AB92761B1D5F8C3
:10FB7000E01EB1F1104F32D0D5F8E02ECDE90A29C0
:10FB800088F80200484641E0D5F8E00EB0F5100FC5
:10FB900007D0D5F8E00ECDE90A0988F802204846DA
:10FBA00016E04FF410000021CDE90A01F5E7BDF899
:10FBB0002000C0F10200C200DDE90A01F8F731FBC4
:10FBC000BDF8202008EB0201C870BDF82000401CE1
:10FBD000ADF82000BDF820000328E8D395E74FF0EA
:10FBE00010410022CDE90A12CAE7BDF82000C0F199
:10FBF0000300C200DDE90A01F8F713FBBDF820207D
:10FC000008EB0201C870BDF82000401CADF82000D0
:10FC1000BDF820000428E8D3404688F80770072183
:10FC200001F031FC88F80800ABE0F52006F834005C
:10FC30009DF8140006EBC4056870A970C32011E795
:10FC4000F52006F834009DF8140006EBC405687032
:10FC5000A970CA2006E7F52006F834009DF81400C4
:10FC600006EBC4056870A970B620FBE6F52006F81F
:10FC700034009DF8141006EBC4008046417097F8DC
:10FC80001C0AB22318B188F80220484642E0A42199
:10FC900088F8021048460FE0D5F80C0FBDF8201088
:10FCA000BDF82020C1F10101C900C84008EB0201E4
:10FCB000C870BDF82000401CADF82000BDF8200041
:10FCC0000228E9D3404688F80530052101F0DBFB26
:10FCD00088F8060073E100000169323031303000ED
:10FCE00001693230453030000F080020D410002068
:10FCF0000C450020D5F80C0FBDF82010BDF82020D1
:10FD0000C1F10201C900C84008EB0201C870BDF88A
:10FD10002000401CADF82000BDF820000328E9D3E6
:10FD2000404688F80630062101F0ADFB88F8070050
:10FD30000820CCE0F52106F834109DF8141006EBED
:10FD4000C4077970B87048460EE0D5F8100FBDF8BA
:10FD50002010C1F10301C900C840BDF8201039448A
:10FD6000C870BDF82000401CADF82000BDF8200090
:10FD70000428EAD3E120F8713846072101F083FB1B
:10FD800038720920A3E0F52006F834009DF814002D
:10FD900006EBC4056870A970C52063E6F52006F877
:10FDA00034009DF8141006EBC4008046417097F8AB
:10FDB0001C0A4FF0CE0A30B1AE2188F802104F462F
:10FDC000ADF820905AE0AC2188F802104F46ADF80B
:10FDD000209014E0D5F8F90ED5F8FD1EBDF82020CE
:10FDE000C2F10402D200F8F71CFABDF8202008EB9B
:10FDF0000201C870BDF82000401CADF82000BDF81D
:10FE000020000528E6D3ADF8207014E0D5F8010FE6
:10FE1000D5F8051FBDF82020C2F10402D200F8F782
:10FE200000FABDF8202008EB02010872BDF820009E
:10FE3000401CADF82000BDF820000528E6D388F866
:10FE40000DA040460D2101F01EFB88F80E000F208A
:10FE50003DE0D5F8F90ED5F8FD1EBDF82020C2F121
:10FE60000502D200F8F7DDF9BDF8202008EB020109
:10FE7000C870BDF82000401CADF82000BDF820007F
:10FE80000628E6D3ADF8207014E0D5F8010FD5F8B8
:10FE9000051FBDF82020C2F10502D200F8F7C1F914
:10FEA000BDF8202008EB02014872BDF82000401C7C
:10FEB000ADF82000BDF820000628E6D388F80FA092
:10FEC00040460F2101F0DFFA88F81000112091E27E
:10FED000F52006F834009DF8140006EBC4056870A0
:10FEE000A970E520BEE5F52006F834009DF8140061
:10FEF00006EBC4056870A970E720B3E5F52006F8A5
:10FF000034009DF8140006EBC4056870A970D72072
:10FF1000A8E599F8413A8DF8143095F8D87E9AF80A
:10FF2000D43E9F4202D101278AF8D37E9BF8D03974
:10FF30005B1C8BF8D0399DF8143023B19DF8143038
:10FF40005B1E8DF814300A2858D2DFE800F02AFE34
:10FF50004276D7FDFC05FB5806F834209DF81400C6
:10FF600006EBC40740307870B9703021F9703971F0
:10FF7000352078713320B8713120F8713972797277
:10FF8000B9720320F872781C0B21F9F75BF938730A
:10FF90000D20ADF83C0095F8D80E04282ED1052090
:10FFA0002AE0042206F834209DF8141006EBC40061
:10FFB00040314170512181700521C170EEE0072070
:10FFC00018E2287103206871681C0521F9F73AF9D5
:10FFD000FEE3042306F834309DF8142006EBC40039
:10FFE0004032427081700521C170ADF83C3095F807
:10FFF000D80E0228D2D1032085F8D80E1DE106F8CC
:020000040801F1
:1000000034209DF8140006EBC40540306870A970D8
:100010003120E87085F804E003206871681C052130
:10002000F9F710F9A8710720ADF83C0099F8420AD9
:1000300020F0200189F8421AFFE006F834209DF8EC
:10004000140006EBC40740307870B9703121F970A4
:1000500030203871D5F8E02EB2F5100F00D270467E
:10006000787195F8DD0E012803D095F8DD0E10B1FA
:1000700003E0B97101E087F806E0ADF8208013E0F5
:10008000D5F8E00EBDF82010C1F105018900C84087
:10009000BDF8201000F00F0039443030C871BDF8B1
:1000A0002000401CADF82000BDF820000628E7D352
:1000B00087F80DE0ADF8208013E0D5F80C0FBDF8FF
:1000C0002010C1F103018900C840BDF8201000F0E4
:1000D0000F00394430308873BDF82000401CADF863
:1000E0002000BDF820000428E7D30320B874781C52
:1000F0001221F9F7A7F8F87414207BE106F83420F0
:100100009DF8140006EBC40740307870B97087F88A
:1001100003E03121397187F805E087F806E0ADF892
:10012000208018E0D5F80C0FBDF82010C1F10301B4
:100130008900C840BDF8201000F00F00394430306D
:10014000C87103E05EE03AE13AE14EE0BDF820001C
:10015000401CADF82000BDF820000428E2D3ADF823
:100160002080302108E0BDF820003844C172BDF87D
:100170002000401CADF82000BDF820001928F2D363
:10018000032087F82400781C2421F9F75BF887F80E
:1001900025002620F1E306EBC4014870ADF83C20B1
:1001A000EDE399F8413A8DF8143095F8D87E9AF835
:1001B000D43E9F4202D101278AF8D37E9BF8D039E2
:1001C0005B1C8BF8D0399DF8143023B19DF81430A6
:1001D0005B1E8DF814300A28E2D2DFE800F0050635
:1001E000204AF2F1F02E132FDBE606F834209DF8BA
:1001F000140006EBC40540306870A9703120E87027
:100200003520DEE606F834209DF8140006EBC40520
:1002100040306870A97085F803E03020D1E60423EF
:1002200006F834309DF8142006EBC40040324270CA
:1002300081700521C170ADF83C30A0E306F8342090
:100240009DF8140006EBC40540306870A970312099
:10025000E87085F804E003206871681C0521F8F750
:10026000F1FFA87199F8420A20F0200189F8421A9A
:10027000A5E606F834209DF8140006EBC4074030CC
:100280007870B9703120F8703971D5F8E01EB1F18D
:10029000104F09D07146797195F8DD1E012905D0FE
:1002A00095F8DD0E30B102E03021F4E7B871ADF819
:1002B000208015E07046F9E7D5F8E00EBDF8201073
:1002C000C1F107018900C840BDF8201000F00F00FF
:1002D00039443030C871BDF82000401CADF8200012
:1002E000BDF820000828E7D387F80FE0ADF820809C
:1002F00013E0D5F80C0FBDF82010C1F105018900FD
:10030000C840BDF8201000F00F00394430300874A8
:10031000BDF82000401CADF82000BDF820000628E4
:10032000E7D33020B875ADF8208008E0BDF8201084
:100330003944C875BDF82010491CADF82010BDF82F
:1003400020100629F2D37877ADF8208008E0BDF8B8
:10035000201039448877BDF82010491CADF82010D2
:10036000BDF820100629F2D387F82400ADF82080CC
:1003700009E0BDF82010394481F82500BDF82010AF
:10038000491CADF82010BDF820100629F1D387F8DC
:100390002B00ADF8208009E0BDF82010394481F829
:1003A0002C00BDF82010491CADF82010BDF820101D
:1003B0000629F1D387F83200ADF820800CE067E021
:1003C00061E018E0BDF82010394481F83300BDF831
:1003D0002010491CADF82010BDF820100629F1D3DB
:1003E000032087F83900781C3921F8F72BFF87F8AC
:1003F0003A003B20C1E206F834209DF8140006EBD9
:10040000C40740307870B97087F803E03121397142
:100410003321797187F806E0ADF8208013E0D5F834
:100420000C0FBDF82010C1F105018900C840BDF8CE
:10043000201000F00F0039443030C871BDF82000A2
:10044000401CADF82000BDF820000628E7D3ADF829
:100450002080302108E0BDF8200038444173BDF809
:100460002000401CADF82000BDF820001928F2D370
:10047000032087F82600781C2621F8F7E3FE87F88A
:100480002700282079E2102006F83400302082E688
:10049000102006F8340031207DE699F8410A8DF8E5
:1004A0001400BDF8200000EB40100AEB800090F82B
:1004B000D81E9AF8D40E814202D101218AF8D31EA7
:1004C0009BF8D009401C8BF8D00940460CE0BDF8E1
:1004D000200007EB001090F8410A9DF814108842A4
:1004E0000AD0BDF82000401CADF8200097F8170A8C
:1004F000BDF820108842EAD8BDF8200007EB0010B4
:1005000090F8401A1398401A401C8DF818009DF876
:10051000140020B19DF81400401E8DF8140095F8C9
:10052000D90E0F2803D295F8D90E401C00E04046A2
:1005300085F8D90E14984FF0FA09B12813D008DCC9
:10054000A4287DD0A5287CD0A6289CD0AA2879D123
:1005500066E0B22814D0B32851D06521B82828D03D
:10056000B928F4D137E09DF81400503006F8340073
:1005700006EBC4002021417080F802900320FCE1CA
:100580009DF81400503006F8340095F8D90E06EBAB
:10059000C40540F0300068700120A870E87047463C
:1005A00085F8048028460521F9F714FACDE90A07F1
:1005B00062E09DF81400503006F8340095F8D90E2A
:1005C00006EBC40540F030006870A9700120E870A7
:1005D0009DF8180049E09DF81400503006F83400EA
:1005E00095F8D90E06EBC40540F030006870A9708C
:1005F0000120E8709DF8180040F0100035E09DF8EB
:100600001400503006F8340095F8D90E06EBC405F6
:1006100040F0300068700120A870E870052024E0E8
:100620009DF81400503006F8340095F8D90E06EB0A
:10063000C40540F0300068700120A870E87002E046
:1006400003E023E055E108200FE09DF8140050304E
:1006500006F8340095F8D90E06EBC40540F03000DA
:1006600068700120A870E8700620287128460521CE
:10067000F9F7B0F9CDE90A0868710A98000AA8717B
:100680000320E87185F80890FFF77BBBADF8208068
:100690000EE0BDF8200007EB001090F8410A9DF82D
:1006A000141088420AD0BDF82000401CADF820008C
:1006B00097F8170ABDF820108842EAD8ADF80480F0
:1006C00011E0BDF80400BDF82010084407EB00104D
:1006D00090F8410A9DF81410884208D1BDF8040032
:1006E000401CADF80400BDF804000628E9D39DF8CD
:1006F0001400503006F8340095F8D90E06EBC40506
:1007000040F0300068700520A870BDF8040000EBD0
:100710004000C01CE870ADF80C802AE0ADF80880FD
:100720001EE0BDF82000BDF80C20104400EB401086
:100730000AEB8000D0F80C1FBDF80800C0F10200E1
:10074000C000C140BDF80C00BDF8082000EB40001F
:10075000104428440171BDF80800401CADF80800A1
:10076000BDF808000328DCD3BDF80C00401CADF830
:100770000C00BDF80C00BDF804108842CED3BDF8C3
:100780000C0000EB4000C01D81B22846F9F722F9A9
:10079000CDE90A080146BDF80C0000EB40002844F2
:1007A000C1710A98010ABDF80C0000EB4000284412
:1007B0000172BDF80C00032100EB40002844417297
:1007C000BDF80C0000EB4000284480F80A9000E0DF
:1007D000AFE1BDF80C0000EB40000B30CDE0BDF800
:1007E00020100098084490F8D019491C80F8D019BE
:1007F00097F81C0A38B11399491CC9B2012834D0A2
:10080000022876D143E01498312802D0452870D1CF
:1008100015E0ADF820800CA90CE0BDF82000BDF873
:10082000203006EBC402085CD054BDF82000401C08
:10083000ADF82000BDF820000728EED318E5ADF88C
:10084000208010A90CE0BDF82000BDF8203006EB98
:10085000C402085CD054BDF82000401CADF8200054
:10086000BDF820000728EED302E58DF814109DF89E
:10087000140006F8340006EBC4050320687085F800
:100880000280EA7085F804800920687110E08DF814
:1008900014109DF8140006F8340006EBC40503207C
:1008A000687085F8028085F8038085F804806A7195
:1008B00028460621F8F798FECDE90A08000AE871F3
:1008C0000A98A871FFF734BAF9499BF8D009401C7F
:1008D0008BF8D00999F8410A8DF814001498F32880
:1008E00074D007DC052872D0F12808D0F22846D150
:1008F00013E044E0F4286BD0F62840D1DDE0F52089
:1009000006F834009DF8140006EBC405687085F8FD
:1009100002800520E870F12001E1F52006F834009E
:100920009DF8140006EBC407787087F80280F22067
:10093000387195F8480F787195F8480F012829D03B
:1009400095F8480F202872D00620ADF83C00BDF87D
:100950003C00F8703846BDF83C10F8F745FECDE98C
:100960000A08BDF83C10000A7854BDF83C100A98FB
:1009700039444870BDF83C00801CADF83C00CD48BF
:10098000CD4D1299E9B301297DD002297CD00329EC
:100990007BD16EE12520ADF83C004146ADF82080CA
:1009A0000DE0BDF82000284490F8210FBDF820206C
:1009B0003A449071BDF82000401CADF82000BDF80D
:1009C00020000F28EDD3ADF8201010E047E0B2E092
:1009D00098E0BDF82000284490F8330FBDF820209F
:1009E0003A445075BDF82000401CADF82000BDF819
:1009F00020000A28EDD395F8420FF877ADF82010C3
:100A00000FE00BE1BDF82000284490F8430FBDF83B
:100A10002010394481F82000BDF82000401CADF8BA
:100A20002000BDF820000528ECD390E7FFE70A205E
:100A3000ADF83C0040460BE0BDF82000284490F89B
:100A4000430FBDF8201039448871BDF82000401CC8
:100A5000ADF82000BDF820000428EDD377E7F5209D
:100A600006F834009DF8140006EBC4077870404681
:100A700087F80280F321397195F8481F79710C21AC
:100A8000ADF83C1002E0D7E0E3E001E195F8421F49
:100A9000B9710BE0BDF82000284490F8430FBDF871
:100AA00020103944C871BDF82000401CADF820006A
:100AB000BDF820000528EDD349E70620ADF83C003D
:100AC000F52006F834009DF8140006EBC4056870A4
:100AD00085F80280BDF83C00E870F620287199F88E
:100AE000480A68712846BDF83C10F8F77DFDCDE94D
:100AF0000A08BDF83C10000A6854BDF83C100A987A
:100B0000294436E7F52006F834009DF8140006EB7A
:100B1000C405687085F802800520E870F42028710B
:100B200028460521F8F760FDCDE90A08000A68713A
:100B30000A98A87182E640F21320ADF83C00F52037
:100B400006F834009DF8142006EBC400814642707C
:100B5000BDF83C20120A8270BDF83C20C27005220C
:100B6000027140460CE0BDF82000384490F81E2A7F
:100B7000BDF8203009EB03004271BDF82000401C95
:100B8000ADF82000BDF820000A28ECD3B7F82A0AF7
:100B90008A46010A89F80F10B7F82A0A89F8100066
:100BA000B5F8560F010A89F81110B5F8560F89F8F3
:100BB0001200B5F8561F129801EB802081B2032075
:100BC000F8F732F94546ADF8208050464FF40073EF
:100BD0000EE0BDF82010014491F86620BDF82070A9
:100BE00009EB0701CA74BDF82010491CADF82010AC
:100BF000BDF820109942ECD34846BDF83C10F8F7F8
:100C0000F3FCCDE90A05BDF83C20000A09F8020012
:100C1000BDF83C200A9809EB0201AAE6BDF83C1099
:100C2000B1B38021F9F7B3FBBDF83C00C5F8A400CF
:100C300021480121A03029E0BDF83C1041B3082132
:100C4000F9F7A5FBBDF83C0068671B48012170302F
:100C50001CE0BDF83C00D8B14FF480711748F9F79B
:100C600096FBBDF83C00C5F8BC0013480121B83024
:100C70000CE0BDF83C1059B14FF48061F9F787FBE7
:100C8000BDF83C00E8650C4801215830F8F702FD3A
:100C9000074890F86702002807D006EBC40000233D
:100CA000BDF83C10129AF9F729FE15B0BDE8F08F97
:100CB000D4100020000C02400060024000000240FE
:100CC0002DE9F04700242DED048B804689469FEDE9
:100CD0001E9B25462646E20040464946F7F7A1FA04
:100CE000C7B22046F7F769FC41EC110BB0EE490A98
:100CF000F0EE690A06F028FD380907F00F0100EB55
:100D00008000B0EE408AF0EE608A01EB4000F7F719
:100D100054FC53EC182BF7F76FFB41EC180B2846EB
:100D20003146F7F757FC53EC182BF7F7BEFAF7F7F5
:100D30007CFC641CE4B205460E46082CCBD3BDEC0B
:100D4000048BBDE8F087000000000000000059405F
:100D500070B50F4D40F224442146284606F091F923
:100D6000012813D1298828462A1D1188214606F01A
:100D700025F90849012081F871090748D0F88C004D
:100D800001F50051C0F57A70A1F8F80F70BD0000B0
:100D900000440040D41000200060024010B50C4C0C
:100DA00040F22441204606F06CF901280ED120883B
:100DB000201D00880749012081F87D090648406C04
:100DC00001F50051C0F57A70A1F8FA0F10BD0000CE
:100DD000004C0040D41000200060024010B50B4CC5
:100DE00040F22441204606F04CF901280DD120881C
:100DF000A0880749012081F889090648406901F562
:100E00000051C0F57A70A1F8FC0F10BD00500040F1
:100E1000D41000200060024010B50C4C40F2244178
:100E2000204606F02EF901280ED12088201D0088CA
:100E30000749012081F895090648C06A01F500516B
:100E4000C0F57A70A1F8FE0F10BD00000048004008
:100E5000D41000200060024010B5124C104920460A
:100E6000F8F702FC00212046F8F714FC0E4C402154
:100E7000204606F0FFF80028F9D080210B48F9F74A
:100E800088FA084C0A49183C2046F8F7EDFB012186
:100E90002046F8F7FFFB07490120087110BD00004C
:100EA00000802020A060024000440040000C02406E
:100EB000008800200F08002010B5124C1049204671
:100EC000F8F7D2FB00212046F8F7E4FB0E4C402156
:100ED000204606F0CFF80028F9D008210B48F9F792
:100EE00058FA084C0A49303C2046F8F7BDFB01216E
:100EF0002046F8F7CFFB07490120087110BD00001C
:100F00002080002070600240004C0040000C024035
:100F1000008020100F08002010B5124C1049204608
:100F2000F8F7A2FB00212046F8F7B4FB0E4C402155
:100F3000204606F09FF80028F9D04FF480710B4846
:100F4000F9F727FA074C0A49A83C2046F8F78CFB2A
:100F500001212046F8F79EFB06490120087110BDCB
:100F600000800028B86002400050004000000240AD
:100F7000208000100F08002010B5124C10492046A8
:100F8000F8F772FB00212046F8F784FB0E4C402155
:100F9000204606F06FF80028F9D04FF480610B4826
:100FA000F9F7F7F9074C0A49303C2046F8F75CFBA3
:100FB00001212046F8F76EFB06490120087110BD9B
:100FC000008000185860024000480040000C0240B9
:100FD000008800100F0800202DE9F047012190B093
:100FE000480503F073FF8648F8F75EFB4027380199
:100FF0000024CDE90540C50107940894CDE90945D1
:1010000046040C940D94DFF8FC917F480B94CDE9D5
:101010000207CDE9006969460E947948F8F7ECFBC0
:10102000012210217648F8F7D1FBDFF8D4A1AAF10C
:10103000180A5046F8F738FB4FF47A78CDE90348A0
:10104000E811CDE9054007940894CDE909456F48BA
:101050000B940C940D9400960E94CDE90190694682
:101060005046F8F7C9FB01215046F8F713FBDFF8AB
:1010700090A1AAF1300A5046F8F716FBE811CDE925
:10108000054007940894CDE909450C940D94DFF8C8
:10109000809160480B94CDE90207CDE9006969466B
:1010A0000E945046F8F7A8FB012210215046F8F79D
:1010B0008DFBDFF84CA1AAF1600A5046F8F7F4FA6C
:1010C000CDE90348E811CDE9054007940894CDE93E
:1010D000094551480B940C940D9400960E94CDE95B
:1010E000019069465046F8F787FB01215046F8F712
:1010F000D1FADFF80CA10AF1180A5046F8F7D4FA31
:10110000E811CDE9054007940894CDE909450C9410
:101110000D94DFF8089142480B94CDE90207CDE920
:10112000006969460E945046F8F766FB01221021CB
:101130005046F8F74BFBDFF8C8A0AAF1900A5046DA
:10114000F8F7B2FACDE90348E811CDE90540079474
:101150000894CDE9094533480B940C940D940096FE
:101160000E94CDE9019069465046F8F745FB012100
:101170005046F8F78FFADFF88890A9F148094846F9
:10118000F8F792FA0397E811CDE90540079408941F
:10119000CDE9094525480B940C940D94224F0096F7
:1011A0000E94CDE9017069464846F8F725FB012207
:1011B00010214846F8F70AFBDFF84490A9F17809B6
:1011C0004846F8F771FACDE90348E811CDE9054042
:1011D00007940894CDE9094515480B940C940D9497
:1011E00000960E94CDE9017069464846F8F704FB75
:1011F00001214846F8F74EFA10B0BDE8F08700002C
:10120000A0600240044400400C4500206C4E0020C9
:10121000044C004064470020545200200450004019
:10122000BC4900203C56002004480040144C0020DB
:10123000245A00202DE9FC410121084603F046FE16
:101240000121042003F042FE0121082003F03EFEAC
:101250000121402003F03AFEDFF8FC80072205213F
:101260004046F9F77DF8072206214046F9F778F85D
:10127000072208214046F9F773F807220921404662
:10128000F9F76EF8354F08220A213846F9F768F861
:1012900008220B213846F9F763F80822022140465C
:1012A000F9F75EF808220C213846F9F759F80226BA
:1012B0008DF8056000244FF459708DF80640012523
:1012C00000908DF807508DF8046069464046F9F7A4
:1012D0000BF88DF805604FF4E0508DF80640009053
:1012E0008DF807508DF8046069463846F8F7FCFF22
:1012F0004FF4916000908DF806408DF804506946D7
:101300004046F8F7F1FF280200908DF806408DF86E
:10131000045069461248F8F7E7FF8DF806404FF48D
:10132000F040104C00908DF8045069462046F8F7C4
:10133000DBFFA9032046F9F72AF869032046F9F7ED
:1013400026F8A1142046F9F722F8E1142046F9F70F
:101350001EF8BDE8FC810000000C024000080240BD
:10136000000002400018024070B50024FFF762FF41
:10137000FFF732FE00F022F80E4D002185F86C19BF
:10138000012285F86C290C48017081704170C2708F
:101390004FF47A718160042085F86C0904E02046DE
:1013A00000F062F9641CE4B295F86C09A042F6D82A
:1013B00070BD0000D410002010410020F8B51120AD
:1013C0008DF8000002258DF8015001248DF80240AF
:1013D0008DF80340684600F0E7FA26208DF80000FB
:1013E0008DF8014000268DF802608DF803406846B4
:1013F00000F0DAFA0E208DF800008DF801508DF81B
:1014000002408DF80340684600F0CEFA27208DF8A0
:1014100000008DF801408DF802608DF803406846A9
:1014200000F0C2FA0F208DF800008DF801508DF801
:1014300002408DF80340684600F0B6FA34208DF87B
:1014400000008DF801408DF802608DF80340684679
:1014500000F0AAFA2F208DF800008DF801508DF8C9
:1014600002408DF80340684600F09EFA35208DF862
:1014700000008DF801408DF802608DF80340684649
:1014800000F092FAF8BD01B9102110F8012B10F804
:10149000013B491E5A400904090CF8D102F07F00B3
:1014A000704700002DE9FF5F14460F464FF4805649
:1014B0004FF480684FF4C0694FF00C0A40F2244B9F
:1014C000002580B1012830D0022851D0032871D1E5
:1014D0000121880403F01EFD0097012C6DD0022C21
:1014E00070D094B377E00121480403F013FD009716
:1014F000012C03D0022C06D054B10DE0ADF80460ED
:10150000ADF8088008E0ADF80460ADF8089003E09D
:10151000ADF80450ADF80850ADF80650ADF80C50D9
:10152000ADF80AA069463B4C5DE00121C80403F018
:10153000F1FC0097012C03D0022C07D05CB10EE027
:10154000ADF80460ADF8088009E040E0ADF8046053
:10155000ADF8089003E0ADF80450ADF80850ADF8D0
:101560000650ADF80C50ADF80AA069462A4C3AE096
:101570000121080503F0CEFC0097012C03D0022CBA
:1015800006D054B10DE0ADF80460ADF8088008E075
:10159000ADF80460ADF8089003E0ADF80450ADF884
:1015A0000850ADF80650ADF80C50ADF80AA06946E9
:1015B0001A4C18E02CE000E004E0ADF80460ADF84F
:1015C000088008E0ADF80460ADF8089003E0ADF8DD
:1015D0000450ADF80850124CADF80650ADF80C5060
:1015E000ADF80AA06946204605F082FD012120469B
:1015F00005F0E7FC01225946204605F061FD102167
:10160000204605F0DBFC0122C021204605F0E3FC6A
:10161000BDE8FF9F00440040004C004000500040E7
:10162000004800402DE9FC410024CDE900446F460C
:1016300064220023F6F7C4FD0E46054610461946FF
:101640000A220023F6F7BCFD010102F00F00081882
:10165000385504F10104E4B228463146082CE7D39A
:10166000DDE90001BDE8FC812DE9F05F624F06462F
:101670000025042087F86C0906EB460000EB0610F5
:1016800007EB001494F81D0A012803D1002130460D
:1016900000F0B4F806EB4602B84607EB82074FF0BD
:1016A000000B87F870B987F872B987F871B987F8B5
:1016B00073B94FF00509C7F8789987F8A0B987F88A
:1016C000A2B9012087F8A10987F8A309D4F8180A5C
:1016D00000EB80004000C7F8A80994F8152AD4F858
:1016E000101A3046FFF7DEFE94F8161A06EBC60213
:1016F000414B072002EB062203EBC206072911D259
:10170000DFE801F010040607070A1400484600E06D
:101710000F2086F8D40E05E0D4F8180A6421484357
:10172000C7F8A8094FF0A10AC1465EE00320F0E720
:1017300005EB451006EB800080F8E4BE012380F83D
:10174000E63E80F8E5BE80F8E7BE4FF47A73C0F855
:10175000EC3E04EB051383F842BA80F8D8BE94F847
:10176000161A07293FD2DFE801F03E0408080A0CE8
:101770000E00E52180F8DC1E35E05146FAE7B12184
:10178000F8E73121F6E7F12180F8DC1E002125E0A1
:1017900001EBC10707EB012701EB410C02EBC70787
:1017A0000CEB011C002009EB0C1211E002EB001CF9
:1017B0009CF840CA93F8488AC44507D193F840CAB8
:1017C00000EB401807EB880888F849CF401CC0B2EE
:1017D00092F817CA8445E9D8491CC9B299F86C092E
:1017E0004A468842D4D86D1CEDB294F8170AA84234
:1017F0009ED8BDE8F09F0000D41000202DE9F041F4
:10180000054661484FF48042531006685F488414CF
:10181000C71439B1C5B1012D18D0022D18D0032D30
:101820001BD117E035B1012D06D0022D06D0032DB6
:1018300013D105E0114604E0194602E0214600E01C
:101840003946F8F7A6FD08E0114604E0194602E023
:10185000214600E03946F8F79AFD642007F0C2F807
:1018600000224FF416512846FFF71CFEDFF82081B6
:1018700005EB450008EB8000002280F8A229C0F8A3
:10188000A42905EB450000EB051008EB0011D1F889
:10189000183A08F540504364012380F83D3091F830
:1018A000161A3C4C962305EB8500204406290AD2E3
:1018B000DFE801F0090305050733762102E08370B4
:1018C00001E06E218170C5EB0511334B01EB810105
:1018D000C02403F8314003EBC10462700821A170F9
:1018E000E27006F00F0105EB0512114421718078BA
:1018F00060712020A071E171802020724C20607204
:101900005420A0722548264F0B2645B1012D0FD03B
:10191000022D24D0032D14D12CE06621D2E78021A2
:10192000F8F735FDC7F8A4601D480121A03006E096
:101930000821F8F72CFD7E67194801217030F7F770
:10194000A9FE98F8670228B1204600232A460B21F9
:10195000F8F7D4FFBDE8F041642007F043B84FF436
:1019600080711048F8F713FDC7F8BC600C480121DE
:10197000B830E4E74FF48061F8F709FDFE650848E8
:1019800001215830DBE70000187AFF1F00180240E1
:10199000D41000200C5E00200C450020000C0240FA
:1019A000006002400000024030B50F23C278017889
:1019B0000125FAB1144A126801F1E02102F4E06253
:1019C000C2F5E062C2F30722C2F10404D3404278B8
:1019D000A24084781C401443220181F8002400783E
:1019E00000F01F018D404009800000F1E020C0F8A8
:1019F000005130BD01F01F0085404809800000F112
:101A0000E020C0F8805130BD0CED00E0024A1140EA
:101A1000014302480160704780FFFF1F08ED00E0AE
:101A2000BFF34F8F04480168044A01F4E061114399
:101A30000160BFF34F8FFEE70CED00E00400FA05F4
:101A400010B50021074B0A46002003EBC004401CE0
:101A5000C0B262548028F8D3491CC9B20829F3D314
:101A600010BD00000F6800202DE9FE4F0026171A58
:101A70008146701E3546A3EB010A8846002F02DD21
:101A80004FF0010102E003D14FF00001019102E0AB
:101A9000C7F100070190BAF1000F02DD4FF001001D
:101AA00002E003D14FF00000009002E0C7F1000A0D
:101AB00000905046574501DD3C4600E00446601C5E
:101AC0004FF0000B029016E008F0FF0109F0FF0054
:101AD0000C9A00F015F83E445544A64202DD0199E7
:101AE000361B8944A54202DD00992D1B88440BF169
:101AF00001001FFA80FB02998B45E5DBBDE8FE8FF4
:101B000030B5CC0801F0070301259D40EBB2064D2E
:101B100005EBC005C808285C0AB1184302E063EA77
:101B20000000C043285530BD0F6800202DE9FC415E
:101B300001210A2003F0CAF901248DF8044000268F
:101B40004FF4C0508DF80660032700908DF80570A3
:101B50008DF8074069464548F8F7C6FB8DF8044004
:101B60008DF806608DF80570A5028DF80740404C91
:101B7000009569462046F8F7B7FB29462046F8F756
:101B800006FCC82006F02EFF29462046F8F701FC87
:101B9000642006F027FF0021FD2000F025FA002137
:101BA000122000F021FA0021AE2000F01DFA0021E1
:101BB000D52000F019FA0021A02000F015FA00212C
:101BC000A82000F011FA00213F2000F00DFA0021BA
:101BD000D32000F009FA0021084600F005FA0021A0
:101BE000402000F001FA0021A02000F0FDF90021C2
:101BF000C02000F0F9F90021DA2000F0F5F9002109
:101C0000122000F0F1F90021812000F0EDF900210F
:101C10007F2000F0E9F90021D92000F0E5F900214A
:101C2000822000F0E1F90021DB2000F0DDF9002145
:101C3000342000F0D9F90021A42000F0D5F90021CA
:101C4000A62000F0D1F90021202000F0CDF90021DC
:101C5000084600F0C9F9FFF7F3FE0021AF2000F0BD
:101C6000C3F900F055F8BDE8FC810000000C02400B
:101C7000000402400346012000E05843491EC9B257
:101C8000FBD270472DE9F84F82460A980D46504323
:101C90006421B0FBF1F0984600F0FF0B4FF0010912
:101CA0000AEB02072B4600245046FAB21946CDF83B
:101CB0000090FFF7D9FE05EB0806F3B2FAB2F1B2D5
:101CC0005046CDF80090FFF7CFFE5246F3B22946BA
:101CD0001046CDF80090FFF7C7FEF3B2FAB2F8B2A3
:101CE0002946CDF80090FFF7BFFE4F460AEB0B06E2
:101CF00009E02819C3B2C1B2F2B250460097FFF70B
:101D0000B3FE641CE4B24445F3D3BDE8F88F000091
:101D100070B50025B020294600F066F9002108467C
:101D200000F062F90021102000F05EF9084E002456
:101D300006EBC4000121405D00F056F9641CE4B2DA
:101D4000802CF5D36D1CEDB2082DF0D370BD0000D2
:101D50000F68002070B50B4C05460221204603F0A9
:101D60007FFA0028F9D02946204603F082FA0121A3
:101D7000204603F075FA0028F9D0204603F077FAE0
:101D8000C0B270BD003800402DE9FC4F1D468846AA
:101D900081468B460090082B0ED0680700D00120AA
:101DA00000EBD500690810FB01F0C0B2203A02F048
:101DB000FF0A0026019046E00620F7E7082D10D024
:101DC0000C2D14D0102D16D0182D3FD121490AEB1F
:101DD000CA0001EB80000027845DE0070FD00B9A5A
:101DE00010E01D490AEB4A0001EB4000F3E70AEB63
:101DF0004A001A49EDE71A4901EB0A10EBE70B9884
:101E000030B3002241464846FFF77AFE7F1C640843
:101E100008F10100FFB200F0FF08082FDDD309F13F
:101E2000010000F0FF09082D0AD00099A9EB01007C
:101E3000B0EB550F04D10BF10800894600F0FF0B01
:101E4000761CD846F6B201988642B7D3BDE8FC8F1F
:101E50000122D7E764A20108D8950108009801087B
:101E6000749C01082DE9F84F1D00DDE90A799246BE
:101E70008B4680464FF0000611D11046F6F79DFBC9
:101E800041EC100B05F0C8FB9FED1C1B51EC100B37
:101E900053EC112BF6F709FAF6F7A8FBC5B2082F99
:101EA00000D1022600241CE0281B401EC1B20A20DB
:101EB000FFF7E0FEBAFBF0F00A21B0FBF1F201FB04
:101EC0001200CDF8009088B13030C2B206EB570155
:101ED00001FB0480C0B23B465946FFF755FF641C26
:101EE000E4B2AC42E0D32846BDE8F88F06EB5701D8
:101EF00001FB0480C0B23B463022EDE70000000049
:101F00000000F03F2DE9FF4F81B0064600900F46DC
:101F10004FF0000A8946580700D0012000EBD3009B
:101F20000490002032E0002029E00E98002410F8F0
:101F30000A500AF101001FFA80FAE80701D00F9A4F
:101F400002E00F9848B3002239463046FFF7D8FD2B
:101F50007F1C641C6D08E4B2FFB2082CEDD3761C24
:101F60000098F6B2311A0398814204D109F10800B1
:101F7000009E00F0FF0908F101004F46C0B203992E
:101F800080468842D1D30BF10100C0B20499834648
:101F90008842C8D305B0BDE8F08F0122D4E72DE90F
:101FA000F8431D46DDE908781646894604460EE0EA
:101FB0003B4649462046CDF80080FFF7E5FE082F56
:101FC0000ED004EB5700C4B26D1EEDB2761C002D8E
:101FD00004D03278202A01D37E2AE9D9BDE8F883DB
:101FE000A41DE4B2F0E700002DE9F041114C0646D3
:101FF0004FF4006500292946204602D0F8F7C9F9B8
:1020000001E0F8F7C4F94FF4805739462046F8F755
:10201000BEF939460848F8F7BCF93046FFF79AFE92
:1020200039462046F8F7B5F929462046BDE8F04183
:10203000F8F7AFB9000C0240000402402DE9F04F60
:1020400087B00027ADF80C70ADF80470ADF80870DB
:10205000ADF81470ADF81070ADF800704FF0F20BE1
:102060004FF0A30AFD4EDFF8F883FDE391F8230655
:10207000022802D10720ADF80000BDF8000030446E
:102080008079BDF800203244D27840EA0260BDF881
:10209000002032441279BDF80030120433445B79D9
:1020A00042EA03221043EF4A5368984279D05060C5
:1020B000BDF8000030448078BDF8002032445278EA
:1020C00040EA0225B1F8EA24BDF800002844801C4B
:1020D000824266D30846B1F8EA14BDF80020491BD5
:1020E000891A891EA0F8EA14BDF800002946304478
:1020F000F7F77AFABDF80010294431444978BDF861
:1021000000202A44B25C41EA022181427AD1BDF822
:1021100000003044007900F001000490BDF8000098
:10212000304480790024C0F34209EB1F0FE0BDF872
:10213000000020443044C0794A460499F7F760FC17
:10214000BDF8001021443144C871641CA4B29C4203
:10215000EDDB98F8670240B1A81C81B2BDF8000021
:10216000012330440422F8F7C9FBBDF800003044D5
:10217000C079012188F821164FF00009C8F8289588
:1021800088F82695B84A82F83290C2F83490ADF8B3
:10219000149011287ED00DDCA0F10B00062815D27A
:1021A00000E0FCE3DFE810F007086D08A5089F08D1
:1021B0009F0A1D00A2286FD004DC12286DD0A12830
:1021C00004D1F5E2A32869D0A42868D000204946AC
:1021D000BDF800200244B154401C80B20528F7D35A
:1021E000F2E3ADF80C904446D2E1BDF80C0000EBF0
:1021F000400101EB001004EB001090F8160A0728CC
:102200007DD200E0F3E3DFE800F07A040404047A0E
:102210009B00484682E0BDF80000BDF81410084459
:102220003044007AB8B3012802D002286ED112E0FF
:10223000BDF80C0000EB400101EB0010BDF80410EC
:1022400004EB001000EB011090F8421A21F0040199
:1022500080F8421A5AE0BDF80C0000EB400101EB97
:102260000010BDF8041004EB001000EB011090F812
:10227000421A21F0080180F8421ABDF80C0000EB68
:10228000400202EB0010BDF8042004EB001000EB4C
:10229000021005E0FDE339E0FCE3FCE3FCE3FCE3D2
:1022A000C0F8449ABDF80C100220F7F73DFC00205E
:1022B0004A46BDF80C1001EBC10303EB012104EB0E
:1022C000C103BDF8041001EB411103EB810101448E
:1022D00081F8172F401C80B21428EAD30020BDF8E3
:1022E0000C1001EBC10303EB012104EBC103BDF8AA
:1022F000041001EB411103EB8101014400E042E1D4
:1023000081F8332F401C80B20A28E8D3BDF81400AE
:10231000401CADF81400BDF80400401CADF80400EA
:10232000BDF80C0000EB400101EB001004EB0010C5
:1023300090F8170ABDF8041088423FF66CAF22E10E
:10234000CC46ADF804900FE1BDF80000BDF81410C4
:1023500008443044007A042805D005DC58B101282F
:1023600040D0022878D11BE1082876D010287DD0F3
:10237000202871D1C1E1BDF80C0000EBC00101EBD8
:10238000002004EBC001BDF8040000EB401001EB9D
:10239000800090F8480F102820D1BDF80C0000EB09
:1023A000C00101EB002004EBC001BDF8040000EB0C
:1023B000401001EB800080F848CFBDF80C00F321FD
:1023C00000EBC00202EB002004EBC002BDF80400E9
:1023D00000EB401002EB800080F8DC1EBDF814001A
:1023E000401CBAE0BDF80C0000EBC00202EB00207C
:1023F00004EBC002BDF8040000EB401002EB8000CB
:1024000080F8DCBEBDF80C0000EB400101EB0010D1
:10241000BDF8041004EB001000EB011090F8421A14
:1024200021F0080180F8421ABDF80000BDF8141030
:1024300008443044017ABDF80C0000EBC00202EB06
:10244000002004EBC002BDF8040000EB401002EBDA
:10245000800080F8481F0AE081E0A1E0205E0020B3
:10246000D410002014080020D4400020D2E0002026
:10247000BDF80010BDF814201144014431444A7ADB
:10248000BDF80C1001EBC10303EB012104EBC10308
:10249000BDF8041001EB411103EB8101014481F807
:1024A000212F401C80B20F28E2D30020BDF800107D
:1024B000BDF814201144014431440A7EBDF80C10CB
:1024C00001EBC10303EB012104EBC103BDF80410D0
:1024D00001EB411103EB8101014481F8332F401CD2
:1024E00080B20A28E2D3BDF80000BDF814100844F9
:1024F000304490F82200BDF80C1001EBC10202EB51
:10250000012104EBC102BDF8041001EB411102EB03
:10251000810181F8420F0020BDF80010BDF81420A1
:1025200011440144314491F82320BDF80C1001EB13
:10253000C10303EB012104EBC103BDF8041001EB5F
:10254000411103EB8101014481F8432F401C80B20B
:102550000528E1D3BDF814002030ADF81400BDF813
:102560000400401CADF80400BDF80C0000EB400175
:1025700001EB001004EB001090F8170ABDF80410EE
:1025800088423FF6E1AEBDF80C00401CADF80C00EF
:1025900094F86C09BDF80C1088423FF626AE1FE691
:1025A000BDF80C0000EBC00202EB002004EBC002FF
:1025B000BDF8040000EB401002EB800080F8DCBEA8
:1025C000BDF80C0000EB400101EB0010BDF8041059
:1025D00004EB001000EB011090F8421A21F0080102
:1025E00080F8421ABDF80000BDF8141008443044C9
:1025F000017ABDF80C0000EBC00202EB002004EBF6
:10260000C002BDF8040000EB401002EB800080F82F
:10261000481FE3E6BDF80C00F32100EBC00202EB1B
:10262000002004EBC002BDF8040000EB401002EBF8
:10263000800080F8DC1EBDF80C0000EB400101EBCF
:102640000010BDF8041004EB001000EB011090F82E
:10265000421A21F0080180F8421ABDF80000BDF8C6
:10266000141008443044017ABDF80C0000EBC0029D
:1026700002EB002004EBC002BDF8040000EB4010A8
:1026800002EB800080F8481FBDF80000BDF8141070
:1026900008443044417ABDF80C0000EBC00202EB64
:1026A000002004EBC002BDF8040000EB401002EB78
:1026B000800080F8421F0020BDF80010BDF81420F3
:1026C0001144014431448A7ABDF80C1001EBC10376
:1026D00003EB012104EBC103BDF8041001EB411130
:1026E00003EB8101014481F8432F401C80B205288F
:1026F000E2D3BDF81400C01D2FE7BDF80C0000EBBD
:10270000C00202EB002004EBC002BDF8040000EBA5
:10271000401002EB800080F8DCBEBDF80C0000EB3E
:10272000400101EB0010BDF8041004EB001000EBB9
:10273000011090F8421A21F0080180F8421ABDF801
:102740000000BDF8141008443044017ABDF80C00B4
:1027500000EBC00202EB002004EBC002BDF8040055
:1027600000EB401002EB800080F8481F0020BDF80D
:102770000010BDF814201144014431444A7ABDF8D8
:102780000C1001EBC10303EB012104EBC103BDF805
:10279000041001EB411103EB8101014481F8432F47
:1027A000401C80B20428E2D3BDF81400401DD4E6DA
:1027B000A81E0D2190FBF1F0C0B20490ADF80C9072
:1027C0004446ACE1484686E1BDF80C0000EB400110
:1027D00001EB0010BDF8041004EB001000EB011039
:1027E00090F8420A80077DD407EB8700BDF80010FF
:1027F00000EBC70008443044007A0021FEF760FA7D
:10280000BDF80C2002EB420303EB0212BDF80430CA
:1028100004EB021202EB031292F8402A89EA010348
:1028200042401A435ED1BDF80C0000EBC00101EB41
:10283000002004EBC001BDF8040000EB401001EBE8
:10284000800090F8150F01287DD1BDF800003044BC
:10285000407BBDF800103144897A40EA0161BDF83F
:1028600000003044C07A00E0FEE3BDF80020000420
:102870003244127B40EA02200143BDF80C0000EB19
:10288000C00202EB002004EBC002BDF8040000EB24
:10289000401002EB8000C0F8E01EBDF8000030449C
:1028A000007DBDF800103144497C40EA0160BDF86C
:1028B00000103144897CBDF8002009043244D27CE8
:1028C00041EA02210843BDF80C1001EB410202EB82
:1028D0000111BDF8042004EB011101EB0211C1F854
:1028E000440A00E0F4E0BDF80C0000EB400101EB0D
:1028F0000010BDF8041004EB001000EB011090F87C
:10290000421A41F0200180F8421ABDF80C10022052
:10291000F7F70AF9BDF80C0000EB400101EB0010DD
:10292000BDF8041004EB001000EB011090F8401A01
:10293000BDF80C0000EBC00202EB002004EBC0006D
:1029400080F8D11E00E051E0BDF80C0000EB400122
:1029500001EB001004EB001090F8160A012804D0D7
:10296000022847D0032841D144E0BDF8000030449C
:10297000407A10B1012839D13AE0BDF80C0000EBE3
:10298000400101EB001004EB001090F81C0A002835
:10299000BDF80C0000EBC00101EB002000E0FDE3FE
:1029A00004EBC001BDF8040000EB401001EB800017
:1029B000D0F8E00E03D0B0F1104F03D105E0B0F530
:1029C000100F02D0B52101E0B0E0C321BDF80C002A
:1029D00000EBC00202EB002004EBC002BDF80400D3
:1029E00000EB401002EB800080F8DC1E6BE0FCE3A3
:1029F000B921EBE7BDF80C0000EBC00101EB0020B2
:102A000004EBC001BDF8040000EB401001EB8000B6
:102A100090F8D81EBDF80C0000EBC00202EB0020BD
:102A200004EBC00090F8D40E81424CD1BDF80000F8
:102A30003044807BBDF8001000043144C97B40EA7B
:102A40000121BDF800003044007C0143BDF80C00BA
:102A500000EBC00202EB002004EBC002BDF8040052
:102A600000EB401002EB8000C0F80C1FBDF8000026
:102A70003044417ABDF80C0000EBC00202EB0020AC
:102A800004EBC002BDF8040000EB401002EB800034
:102A900004E0F0E302E1EFE328E248E080F8DD1E25
:102AA000BDF80C00A42100EBC00202EB002004EBF7
:102AB000C002BDF8040000EB401002EB800080F87B
:102AC000DA1E514682E77F1C0498FFB2874213D278
:102AD000BDF80400401CADF80400BDF80C0000EB8C
:102AE000400101EB001004EB001090F8170ABDF84C
:102AF000041088423FF668AEBDF80C0000EB4001C0
:102B000001EB001004EB001090F8170ABDF8041058
:102B100088420BD8BDF80C00401CADF80C0094F8AE
:102B20006C09BDF80C1088423FF64CAE01E1ADF8DF
:102B30000C90444642E0ADF804901EE0BDF8000061
:102B40003044007A0021FEF7BBF8BDF80C2002EB00
:102B5000420303EB0212BDF8043004EB021202EB55
:102B6000031292F8402A89EA010342401A432CD00A
:102B7000BDF80400401CADF80400BDF80C0000EBEB
:102B8000400101EB001004EB001090F8170ABDF8AB
:102B900004108842D2D8BDF80C0000EB400101EBD4
:102BA000001004EB001090F8170ABDF804108842DA
:102BB000BCD8BDF80C00401CADF80C0094F86C09B2
:102BC000BDF80C108842B6D8B3E0BDF80C0000EB9D
:102BD000400101EB0010BDF8041004EB001000EB05
:102BE000011090F8401ABDF80C0000EBC00202EB97
:102BF000002004EBC00080F8D11EBDF80C0000EBF3
:102C0000400101EB001004EB001090F8160A0128B7
:102C100032D0022801D00328BDD1BDF80C0000EB52
:102C2000C00101EB002004EBC001BDF8040000EB83
:102C3000401001EB800090F8D81EBDF80C0000EBAE
:102C4000C00202EB002004EBC00090F8D40E8142D9
:102C5000A1D1BDF80C00AA2100EBC00202EB0020BC
:102C600004EBC002BDF8040000EB401002EB800052
:102C700080F8DA1E514600E0CA21BDF80C0000EBD6
:102C8000C00202EB002004EBC002BDF8040000EB20
:102C9000401002EB800080F8DC1E7CE7484640E0F4
:102CA000ADF804901EE0BDF800003044007A002129
:102CB000FEF706F8BDF80C2002EB420303EB02130B
:102CC00008EB0312BDF8043002EB031292F8402A1D
:102CD00089EA010342401A432CD0BDF80400401C8D
:102CE000ADF80400BDF80C0000EB400101EB001151
:102CF00008EB011090F8170ABDF804108842D2D8EA
:102D0000BDF80C0000EB400101EB001108EB0110D5
:102D100090F8170ABDF8041088420AD8BDF80C00D4
:102D2000401CADF80C0098F86C09BDF80C209042DE
:102D3000B6D85FE1BDF80C00BDF8042000EB4001FF
:102D400001EB0010414608EB001000EB021090F878
:102D5000402ABDF80C0000EBC00303EB002008EB99
:102D6000C00080F8D12EBDF800003044407ABDF894
:102D7000002000043244927A40EA0222BDF80000AA
:102D80003044C07A0243BDF80C0000EBC00303EBF3
:102D9000002001EBC003BDF8040000EB401003EB82
:102DA0008000C0F80C2FBDF80C0000EB400202EBD5
:102DB000001001EB001090F8160A012841D00228FB
:102DC00001D003289CD1BDF80C0000EBC00202EB3F
:102DD000002001EBC002BDF8040000EB401002EB44
:102DE000800090F8D82EBDF80C0000EBC00303EB78
:102DF000002001EBC00090F8D40E824280D1BDF8D3
:102E00000C00A52200EBC00303EB002001EBC00384
:102E1000BDF8040000EB401003EB800080F8DA2ED0
:102E2000BDF80C0000EBC00303EB002008EBC00171
:102E3000BDF8040000EB401001EB800080F8DCAE30
:102E40005EE7BDF80C0000EBC00202EB002001EBD6
:102E5000C002BDF8040000EB401002EB800090F8C7
:102E6000D82EBDF80C0000EBC00303EB002001EBF3
:102E7000C00090F8D40E8242E2D1BDF80C00B2221C
:102E800000EBC00303EB002001EBC003BDF804001E
:102E900000EB401003EB800080F8DA2EBDF80C0048
:102EA000E52200EBC00303EB002001EBC003BDF8FB
:102EB000040000EB401003EB800080F8DC2E002CB7
:102EC000BED1BDF804000128BAD1BDF80C0000EB5A
:102ED000C00202EB002008EBC001BDF8040000EBCB
:102EE000401001EB8000D0F80C0F09E7BDF800009E
:102EF0003044007A05287DD2BDF800003044007AC5
:102F0000401EADF80C00BDF800003044407ABDF81A
:102F1000001000043144897A40EA0120BDF8001015
:102F20003144C97A0843C117FDF7CAFEBDF80C1039
:102F3000444601EB410202EB011208EB0211C1F819
:102F4000100ABDF800003044007B0021FDF7B8FEF8
:102F5000BDF80C1001EB410202EB011204EB02116F
:102F600081F8140ABDF800003044407B0021FDF7D1
:102F7000A7FEBDF80C1001EB410202EB011204EBBD
:102F8000021181F8150ABDF800003044807B002151
:102F9000FDF796FEBDF80C1001EB410202EB0112A9
:102FA00004EB021181F8160ABDF800003044C07B22
:102FB0000021FDF785FEBDF80C1001EB410202EB8C
:102FC000011204EB021181F8170ABDF80000304429
:102FD000007C0021FDF774FEBDF80C1001EB4102EE
:102FE00002EB011204EB0211C1F8180ABDF800004F
:102FF000304400E035E2407C0021FDF761FEBDF881
:103000000C1001EB410202EB011204EB021181F8FA
:103010001C0ABDF80C0000EB400101EB001104EBB1
:10302000011090F8160A0628484655D09CE0BDF8D5
:103030000000BDF8041008443044807C0021FDF7F6
:103040003FFEBDF804204FF00309B2FBF9F2BDF8D2
:103050000C1001EB410303EB011304EB031101EB33
:10306000021181F8400A00E086E3BDF80000BDF8D7
:10307000041008443044C07C0021FDF721FEBDF857
:103080000420BDF80C10B2FBF9F201EB410303EB95
:10309000011304EB031101EB021181F8410ABDF8A1
:1030A0000000BDF8041008443044007D0021FDF705
:1030B00007FEBDF80420BDF80C10B2FBF9F201EBDD
:1030C000410303EB011304EB031101EB021181F83F
:1030D000480ABDF80400C01CADF80400BDF80C009F
:1030E00000EB400101EB001104EB011090F8170A0E
:1030F000BDF8041000EB4000884298D845E0BDF8C8
:103100000000BDF8041008443044807C0021FDF725
:10311000D7FDBDF80C1001EB410202EB0111BDF827
:10312000042004EB0111520801EB021181F8400A5E
:10313000BDF80000BDF8041008443044C07C0021F4
:10314000FDF7BEFDBDF80C1001EB410202EB0111D1
:10315000BDF8042004EB0111520801EB021181F8C3
:10316000410ABDF80400801CADF80400BDF80C0055
:1031700000EB400101EB001004EB001090F8170A7F
:10318000BDF80410B1EB400FB9D3BDF80C1002200C
:10319000F6F7CAFCBDF80C00C0B200E0D8E2FEF7BA
:1031A00063FABDF80C00012100EB400204EB820041
:1031B00080F83115B7E2BDF800003044007A44468B
:1031C00088F86D02BDF800003044407A88F86C023F
:1031D000BDF800003044807A88F86B02BDF800002A
:1031E0003044C07A88F86A0200E0A2E2BDF800002C
:1031F0003044007B84F86902BDF800003044407B15
:1032000084F8680204F51A74F6F7AAFBF6F766FB71
:103210002078A4F51A74FF2829D1F6F717FBBDF81A
:1032200000003044007A84F86D02BDF8000030449C
:10323000407A84F86C02BDF800003044807A84F84B
:103240006B02BDF800003044C07A84F86A02BDF811
:1032500000003044007B84F86902BDF8000030446F
:10326000407B84F86802F6F77BFBF6F737FB606D6E
:1032700018B10F2002E0F5E0FEE0102084F82506EA
:1032800051E21020444688F82506BDF8000030447D
:10329000007A88F86D02BDF800003044407A88F862
:1032A0006C02BDF800003044807A88F86B02BDF8EB
:1032B00000003044C07A84F86A02BDF8000030444F
:1032C000007B84F86902BDF800003044407B84F83C
:1032D000680204F51A74F6F743FB01F0A1FEA06042
:1032E000A068A0681FE20E2188F8251688F8619072
:1032F00019E24946ADF80C90444638E0ADF80410A8
:1033000014E0BDF80C0000EB400202EB0010BDF829
:10331000042004EB001000EB021090F8420AC007F2
:1033200012D1BDF80400401CADF80400BDF80C003B
:1033300000EB400202EB001004EB001090F8170ABB
:10334000BDF804209042DCD8BDF80C0000EB400230
:1033500002EB001004EB001090F8170ABDF80420EF
:10336000904208D8BDF80C00401CADF80C00BDF828
:103370000C000428C2D3BDF80C00042869D3FF4A0E
:1033800089465170FE490120C1F88802C1F88802BF
:1033900094F86500E8B30D2084F82506BDF8000018
:1033A0003044407ABDF800103144097A40EA0120E7
:1033B000ADF80800BDF800003044C07ABDF8001038
:1033C0003144897A40EA0120508000204FF4007394
:1033D000BDF8001001443144097B04EB000C8CF86B
:1033E0006610401C80B29842F2D3E448408800F254
:1033F000FF3081B20120F5F783FD50B184F8619070
:10340000DE48418864225143BDF80820B1FBF2F147
:1034100000E01CE084F860100121A1714188491C82
:1034200041804088BDF80810884210D914F85C0F1C
:1034300040F001002070207820F00600801C2070F1
:10344000BDF80800608000210120F6F76DFB4846BA
:1034500043E1102084F8250614F85C0F40F080004A
:10346000207060E1BDF800003044017A88F86110F6
:10347000112188F8251656E14946ADF80C904446CE
:1034800038E0ADF8041014E0BDF80C0000EB400289
:1034900002EB0010BDF8042004EB001000EB02105A
:1034A00090F8420AC00712D1BDF80400401CADF8E4
:1034B0000400BDF80C0000EB400202EB001004EB2E
:1034C000001090F8170ABDF804209042DCD8BDF82F
:1034D0000C0000EB400202EB001004EB001090F82F
:1034E000170ABDF80420904208D8BDF80C00401C13
:1034F000ADF80C00BDF80C000428C2D3BDF80C00D8
:1035000004287DD39D4B002058709D490120C1F8AF
:103510008802C1F8880294F86500E8B3122084F8A4
:103520002506BDF800003044007A84F8610094F864
:103530006100401EADF80C000020BDF800100144F1
:1035400031444A7ABDF80C1001EB410C0CEB01112F
:1035500004EB0111014481F81E2A401C80B20A28A4
:10356000EBD3BDF800003044007DBDF800103144BD
:10357000C97C40EA0120ADF80800BDF800003044E5
:10358000807DBDF800103144497D40EA012058801B
:1035900000204FF4007100E056E0BDF80020024426
:1035A0003244D27D04EB000C8CF86620401C80B2C3
:1035B0008842F0D358889946BDF80C1000EB812062
:1035C000401E81B20320F5F79BFCE8B3B9F8021066
:1035D000484664225143BDF80820B1FBF2F184F85B
:1035E00060100121A171B9F80210491CA9F802105C
:1035F000B9F80210BDF80820914242D9002000E03D
:1036000091E0BDF80C1001EB410202EB011104EB5B
:10361000011101EB001191F8492A42F0010281F8F1
:10362000492A401C80B21028E9D3BDF80C0000EBF9
:10363000400101EB001004EB001090F8281A41F053
:10364000010180F8281A00E046E0BDF80C0000EB0C
:10365000400101EB001004EB001090F8281A21F053
:103660000601891C80F8281ABDF80810BDF80C0066
:1036700000EB400202EB001004EB0010A0F82A1A45
:1036800025E04088012827D10020BDF80C1001EB6F
:10369000410202EB011104EB011101EB001191F861
:1036A000492A22F0010281F8492A401C80B21028E0
:1036B000EBD3BDF80C0000EB400101EB001004EB74
:1036C000001090F8281A21F0010180F8281ABDF89E
:1036D0000C100220F6F728FA00202949C1F88802C8
:1036E000C1F888021FE0D8F8540044460A21B0FB14
:1036F000F1F0BDF800103144097A884213D1BDF8C9
:1037000000003044007A18B1606D0A38606504E04A
:10371000C4F85490102084F8250600210520F6F7FF
:1037200003FA0120A071B8F8EA04424620B3002051
:103730001EE000200146BDF800200244B154401CA8
:1037400080B20528F7D3A8F8EA1407B0BDE8F08FD7
:103750000020A1F8EA04F8E7BDF80010294401446C
:1037600031448978BDF800300344F154401C80B2E4
:10377000B2F8EA148142EFD8414603E01408002071
:1037800000004242B8F8EA0400287EF46FACDCE79F
:103790002DE9F74F002084B0FE4E0190054680468B
:1037A000009096F826054FF0000B012876D196F888
:1037B0002106012872D108EB480101EB081000270F
:1037C00006EB001A56E00AEB071494F8420A0006CA
:1037D0004ED594F8420A40F0040084F8420A94F866
:1037E000420A000744D594F8420A20F0080084F801
:1037F000420AC6F835B008EBC80101EB082006EB19
:10380000C00007EB471100EB8109E24809F6F961B6
:103810001022253004F52464F4F713FDD9F8F10ED5
:10382000C6F81900D9F8F50EC6F81D0020783076D4
:10383000D9F80C0FC6F82100D648D0F86812C6F89F
:103840003910B0F86C02A6F83D006068C6F83F0079
:10385000706D81B20220F5F753FB00210620F6F7C8
:1038600063F9706D401C706500210520F6F75CF966
:103870007F1CBFB29AF8170AB842A4D8414602206A
:10388000F6F752F908F101001FFA80F8B8F1040FB9
:1038900091D386F821B60B2086F82506BE4F00206E
:1038A000387000980DE001F0BBFBC6F87002D6F846
:1038B0007002C0F300400190D6F87002C0F34200DD
:1038C00000900028EFD096F82306B3493A31022839
:1038D00016D1B24890F832202AB1002180F8321077
:1038E00001F074F969E0072555200870FD20487043
:1038F000AA2088700020C870087161224A718871FE
:10390000F520485500208B46D6F87012C0F103020E
:10391000D200D1402B1803EB0B02D170401C80B2B7
:103920000428F1D396F8220630B39D48D0F8081247
:103930003078B8B3002001433CD0002059463218FB
:1039400092F8A8252B180B44DA71401C80B2142879
:10395000F5D30020321892F834262B180B44DA766F
:10396000401C80B20A28F5D30BEB0501069881F8BC
:10397000250005F1260405E00BEB05010698C8714A
:1039800005F10804CCB18349069881F8E70406984C
:103990001021FF2311287DD013DCA0F10B00062895
:1039A00022D200E004E0DFE800F01F1FFF11F42046
:1039B0000120C0E7012086F82605002007B0BDE8F9
:1039C000F08FA22810DA12280ED10FE2714880F889
:1039D0002516744900205A4626180B5C9355401C46
:1039E00080B20A28F8D30A34F8E26A4890F85C10EA
:1039F000C90704D0012080F31388FEF711F84FF0B7
:103A0000000977E100EB400101EB091002EB001621
:103A100096F8160A032814D096F8160A012810D032
:103A200096F8160A02280CD096F8160A042808D030
:103A300096F8160A05287DD096F8160A06287AD038
:103A400054E101200BF80400E41CA0B20223029010
:103A50000BF80030401C80B21D230BF80030401CD6
:103A600084B20020A7E006EB081292F8400A5946FB
:103A70000BF80400641CA0B292F8424A0BF8004014
:103A8000401C84B292F8420A400709D492F8420AD4
:103A9000000700E059E103D492F8420A800777D585
:103AA00000201F46D2F8443AC0F1030C4FEACC0C78
:103AB00023FA0CF300EB040C01F80C30401C80B22C
:103AC0000428EFD3241DA3B209EBC90404EB092297
:103AD00007EBC20408EB4812002004EB8207D7F87A
:103AE000F12EC0F10304E400E240C4180A55401C62
:103AF00080B20428F3D31B1D9AB20020D7F8F53EFC
:103B0000C0F10304E400E34084180B55401C80B26C
:103B10000428F3D3121D92B20020D7F80C3FC0F155
:103B20000204E400E34084180B55401C80B20328D3
:103B3000F3D301E050E080E0D21C1FFA82FA0024A7
:103B4000D7F8F90ED7F8FD1EC4F10502D200F4F73C
:103B500068FB04EB0A020BF80200641CA4B2062CFA
:103B6000EED30AF106001FFA80FA0024D7F8010FFD
:103B7000D7F8051FC4F10502D200F4F752FB04EB9D
:103B80000A020BF80200641CA4B2062CEED30CE06F
:103B90000EE062E1D410002014080020D440002080
:103BA00000004042108E0108ACE00AF1060084B229
:103BB00008F1010080B2FF4B96F8171A8046414584
:103BC0003FF651AF0298029A201A0BEB0201030A4A
:103BD00001F8023D487089E002205E460BF80400BF
:103BE000E41CA4B22346002090461AE0421C325541
:103BF000641CA1B23C1894F805447454491C8CB25E
:103C0000002108EB0010471897F8117401EB040C21
:103C100006F80C70491C89B21029F4D31034A4B2F0
:103C200090B298F8041447468142DFD80BEB0300AA
:103C3000002100F8021DE11A57E003200BF80400F0
:103C4000E41CA7B202200BF80700781C80B20E21FA
:103C50000BF80010401C84B200219646DA463AE088
:103C600006EB011292F8400A0AF80400641CA0B2A4
:103C700092F8424A0AF80040401C84B292F8420A84
:103C8000000726D509EBC90C0CEB09220EEBC2028A
:103C900001EB4113002002EB8302131893F8173F46
:103CA00000EB0408D4460AF80830401C80B20A2809
:103CB000F3D30A34A3B20020141894F8304F00EB69
:103CC00003080CF80840401C80B20228F4D39B1C67
:103CD0009CB2491C89B296F8170A8842C0D80AEBF0
:103CE0000700002100F8021DE11B417009F10100ED
:103CF0001FFA80F9AF4A92F86C19484649453FF6D9
:103D000081AE6BE17878401C78707878052804D211
:103D1000A84890F85C20D20707D0A64880F825165E
:103D200090F85C10C90704D005E00D2180F8251635
:103D300001E080F860307888010A0BF80410798877
:103D40000BEB04004170A41C48E19A4F87F825163C
:103D500097F86100DC460BF804000022641C38E090
:103D600097F8610002EB421600EBC00101EB002066
:103D700007EBC00000EB860090F80207012826D16F
:103D800097F8610000EB400101EB001007EB001019
:103D900000EB021090F810090CF80400641CA3B2A8
:103DA000002097F8611001EBC10404EB012107EB3F
:103DB000C10101EB8601014491F803171C180CF8AE
:103DC0000410401C80B20A28EBD30A339CB2521C68
:103DD00092B297F8610000EB400101EB001007EB95
:103DE000001090F8E7089042BAD8F7E07878401CC5
:103DF0007870787805280CD26E4A92F8610000EB52
:103E0000400606EB001002EB001090F8F808C0071F
:103E10000FD0684A82F8251692F8610000EB400145
:103E200001EB001002EB001090F8F808C00704D076
:103E300005E0122082F8250601E082F860305D4836
:103E400090F861100BF8041079880BEB0400090A54
:103E5000417079888170E41CC0E05648012181716D
:103E6000416D0A22B1FBF2F259460BF80420426D73
:103E7000641C0A2A01D90A2300E0436D0022029241
:103E800099460B552222641C0A5500268046DA46C4
:103E9000641C9CE0D8F8540038B1D8F85400801B5A
:103EA000401E81B20220F4F7BFFF98F81800514677
:103EB0000AF80400641CA2B20020D8F81930C0F13E
:103EC0000304E400E34084180B55401C80B204282E
:103ED000F3D3121D92B20020D8F81D30C0F10304B4
:103EE000E400E34084180B55401C80B20428F3D34F
:103EF000121D92B20020D8F82130C0F10204E40073
:103F0000E34084180B55401C80B20328F3D3D21C25
:103F100097B20024414651F8250F4968C4F10502C3
:103F2000D200F4F77EF9E2190AF80200641CA4B288
:103F3000062CEFD3BF1DBFB20024414651F82D0F10
:103F40004968C4F10502D200F4F76BF9E2190AF8E6
:103F50000200641CA4B2062CEFD3BF1D98F83E30BB
:103F6000B8B2414652460AF80030401C98F83D303D
:103F700080B20AF80030401C98F83C3080B20AF851
:103F80000030401C98F83B3080B20AF80030401CEA
:103F900091F83A3080B21354401C91F8393080B215
:103FA0001354401C83B20020D1F83F40C0F10307F6
:103FB000FF0001E0D4100020FC40C718D455401C7D
:103FC00080B20428F0D31B1D761C9CB2B6B2029AB4
:103FD0000021B6EB09009141FFF45CAF661B0BEBCF
:103FE0000500310A5F46804641708670DFF878A090
:103FF0009AF8670228B1B1B2404600230422F6F7CE
:104000007DFC0023B9460AE0E91801EB0907F879BD
:10401000DDE90021F5F704FDF8715B1C9BB29E42BF
:10402000F2DCB1B24D464046F5F7DEFA010A2955F9
:10403000641CA1B26854491C9AF823068CB2022869
:104040000AD1601F010AE970287181B2681D01F070
:104050002EF92855641CA4B2044804600121001FF5
:10406000F5F718FB2046A9E4D4100020BC640240F8
:1040700070B5164C40F224452946204603F001F85D
:10408000002821D02946204602F098FF104D00213B
:104090002846F5F7FFFA61102846F5F7E5FA0D49CD
:1040A000012081F824062088A088281D0268C2F516
:1040B000FA62A1F8EA244FF4FA6101602846BDE8EB
:1040C00070400121F5F7E6BA70BD00000010014014
:1040D00088640240D410002010B5074C05492046E2
:1040E000F5F7C2FA00212046F5F7D4FA034901207A
:1040F000087010BD00800028B86402401408002039
:104100002DE9F04301218FB0880500F0DFFEDFF8D4
:1041100094904846F5F7C8FA402005010390002422
:10412000CDE90545C60207940894CDE909464FF04C
:1041300000681E480B940C940D941B4FCDF8008022
:104140000E94CDE9017069464846F5F755FB01220A
:1041500010214846F5F73AFBDFF84890A9F13009FD
:104160004846F5F7A1FA4FF4FA60CDE90340CDE9EE
:10417000054507940894CDE909460D480B940C9425
:104180000D94CDF800800E94CDE901706946484643
:10419000F5F732FB01214846F5F77CFA0FB0BDE890
:1041A000F0830000B8640240041001404E08002073
:1041B000205E00207CB50121032000F087FE134D16
:1041C000072206212846F6F7CBF807221146284693
:1041D000F6F7C6F8C020022100908DF805100024E3
:1041E0008DF8064001208DF807008DF8041069460F
:1041F0002846F6F779F8072000908DF804408DF8EE
:10420000074069460248F6F76FF87CBD000402409B
:104210000000024070B50024FFF7CCFFFFF770FFED
:104220004FF4E13000F086F800F066F801214020FC
:1042300000F064FE012000F0E5FE2D490B2081F81E
:104240002506002581F8145581F8165581F8155575
:1042500081F817554FF47A70C1F81C0581F8245580
:10426000012381F8263581F8253581F82735C200EC
:10427000C1F82C2581F8FC5481F8FE3481F8FD3416
:1042800081F8FF34C1F8040581F8085581F80A3532
:1042900081F8093581F80B354210C1F81025154A0F
:1042A000157095705370D37042F21076966042F696
:1042B000F82604EB440201EB820282F8305582F8C2
:1042C000325582F8313582F83355C2F83865641CAE
:1042D000042CEED391F8202622B191F82026521E0C
:1042E00081F8222604F07EFBBDE8704000F022B980
:1042F000D41000200441002038B546208DF800007D
:1043000002208DF8010001248DF802408DF8034051
:104310006846FDF749FB25208DF800008DF8014027
:1043200000208DF802008DF803406846FDF73CFB45
:1043300038BD00001FB504460121102000F002FE28
:104340000020ADF804000094ADF80600ADF80800B8
:10435000ADF80C000C200D4CADF80A006946204663
:1043600002F0C6FE0121204602F02BFE012240F29F
:104370002441204602F0A4FE1021204602F01EFE39
:104380000122C021204602F026FE1FBD0010014080
:104390002DE9F04F8DB034225F496846F3F751FFA5
:1043A0005E4D002695F8220600287CD0DFF870B11B
:1043B0000121CBF888124FF0000985F82496594F57
:1043C000594C02E0B85DA055761C5648F3F757FFEC
:1043D000B042F7D8DFF85481C8F800600121A8F195
:1043E0000400F5F757F94FF4FA7004F0FBFA85F87A
:1043F0002496DFF830A100260AF1750A03E01AF8C6
:104400000600A055761C47487530F3F738FFB042D8
:10441000F5D8C8F8006045480121001FF5F73AF9C2
:104420004FF47A7004F0DEFA4E46A94685F8246609
:10443000DFF8F0A000250AF1020A03E01AF80500EF
:1044400060556D1C3748801CF3F719FFA842F5D85A
:10445000C246C8F8005035480121001FF5F71AF987
:104460004FF47A7004F0BEFAB04689F8246600264C
:1044700002E0B85DA055761C2A48F3F700FFB04271
:10448000F7D85546CAF80060DFF8A0A00121AAF1CC
:10449000040A5046F5F7FEF84FF47A7004F0A2FAD9
:1044A0002349684600E034E0F3F7DDFE1D49684625
:1044B000891DF3F7D8FE4F4689F824860026E94681
:1044C00003E019F80600A055761C6846F3F7D7FEFE
:1044D000B042F6D82E6001215046F5F7DBF84FF4D4
:1044E0007A7004F07FFA464687F824860D4900204A
:1044F0000A310A5C2254401C0728FAD3401E286067
:1045000001215046F5F7C6F8642004F06BFACBF8A9
:1045100088620DB0BDE8F08F88930108D4100020A8
:1045200000004242AC9001084E080020BC640240EA
:10453000901600202DE9F04FDFF8EC8387B00024BF
:1045400098F8220600287CD0F8480125C0F8885247
:1045500098F8231608F27650DFF8D4B3F54E0090A1
:10456000022904D0A24688F824A6F34FEEE00020EA
:104570003055641C642CFBD3814688F82406EE4930
:10458000002096310A5C3254401C0828FAD30027D8
:1045900008F2E45406E008EB070090F8E405F1198E
:1045A00008727F1C2046F3F76AFEB842F3D82C202D
:1045B000F1190872002408F20C60B2460937019024
:1045C00007E008EB040090F80C163A190AF80210FC
:1045D000641C0198F3F753FEA042F2D8D7A1D54846
:1045E000F3F741FED348F3F74AFECBF80000D0487A
:1045F0000121001FF5F74EF84FF47A7705E001200E
:1046000004F0F0F9641CBC427ED898F82406002817
:10461000F5D0CB48D0F81802C749B331D0B100204B
:104620004A4654462254401C6428FBD3C24688F8AC
:1046300024260026885DA055761C0E2EFAD30098FD
:1046400000E077E0F3F71BFE0004000C33D00026F7
:1046500051462AE0B44A82F824960026544604E0E3
:10466000B548B330805DA055761CB348B330F3F73E
:1046700006FEB042F4D8CBF80060AD480121001F1F
:10468000F5F708F8A84C05E0012004F0ABF9761C1A
:10469000BE42B9D894F824060028F5D015E08A194E
:1046A00092F87625A3199A73761C8642F7D3A3A1B4
:1046B000A048F3F7D8FD9F48F3F7E1FDCBF80000E1
:1046C0009B480121001FF4F7E5FF3C4698F82406BB
:1046D00088B39C489C494C46006808609948001D76
:1046E000006848609748083000688860002008EB40
:1046F000000282F8A845401C1428F8D3CD7A8B7AA2
:104700004A7A087A02AE00E00CE186E82D00CA7908
:104710008879CDE900024B790A798CA1944802F09E
:104720004FFD00210320F5F7FFF9002802D07F4854
:10473000C0F8884231E2FFE7012004F053F9761C0B
:10474000A642C3D921E2385D3055641C7A48F3F79C
:1047500096FDA042F7D8D946CBF800407448012115
:10476000001FF4F797FF4FF4FA7004F03BF9C346CB
:1047700088F824A6DFF8C081002408F1750803E05A
:1047800018F804003055641C6B487530F3F777FD5A
:10479000A042F5D8C9F8004065480121001FF4F790
:1047A00079FF4FF47A7004F01DF9D0468BF824A6F7
:1047B000DFF884A100240AF1020A03E01AF80400D9
:1047C0003055641C5C48801CF3F759FDA042F5D8B5
:1047D000C9F8004056480121001FF4F75BFF4FF471
:1047E0007A7004F0FFF88BF82486002402E0385D2C
:1047F0003055641C5048F3F742FDA042F7D8C9F881
:1048000000404B480121001FF4F744FF4FF47A7039
:1048100004F0E8F8C2465F468BF82486DFF818817A
:10482000002408F16A0803E018F804003055641CFD
:1048300041486A30F3F723FDA042F5D8C9F800409B
:104840003B480121001FF4F725FF4FF4FA7805E0FB
:10485000012004F0C7F8641C444563D897F8240687
:104860000028F5D087F824A6DFF8CCB000240BF19F
:10487000390B03E01BF804003055641C2E48393016
:10488000F3F7FDFCA042F5D8C9F800402848012103
:10489000001FF4F7FFFE05E0012004F0A3F8641CFC
:1048A0004445DAD897F824060028F5D087F824A6DE
:1048B0002348D0F818024FF00004A0B9DFF878B010
:1048C0000BF1110B03E01BF804003055641C1A486F
:1048D0001130F3F7D4FCA042F5D809E0381990F86C
:1048E00076053055641C0098F3F7C9FCA042F5D852
:1048F000C9F800400E480121001FF4F7CBFE05E087
:10490000012004F06FF8641C4445A6D897F82406EB
:104910000028F5D087F824A6DFF81CB000240BF19E
:10492000480B2BE0AAE00000D41000200000424217
:10493000BC6402404E080020AC9001080D0A000043
:1049400000004342107AFF1FF065002025303278C6
:10495000253032782530327825303278253032785B
:104960002530327825303278253032782500000025
:10497000801600201BF804003055641C8A48F3F7A9
:104980007EFCA042F6D8C9F8004001218748F4F720
:1049900081FE05E0012004F025F8641C4445B4D8EC
:1049A00097F824060028F5D0D34687F824A6DFF828
:1049B000F8A100240AF1110A03E01AF804003055A6
:1049C000641C79481130F3F75AFCA042F5D8C9F8B5
:1049D000004001217548F4F75DFEC24605E0012064
:1049E00004F000F8641C544548D897F824060028C1
:1049F000F5D0D84687F824B66B4800243730015DDF
:104A00003155641C0C2CFAD3611ECB46C9F800103A
:104A100001216648F4F73EFE05E0012003F0E2FFC5
:104A2000641C54452AD897F824060028F5D060A1C4
:104A3000614804F065F9D8B15F4A00214318134476
:104A400091465B797C1884F86135491C1429F5D3AB
:104A500097F8BD0568B359495948F3F704FC524922
:104A600057484239F3F7FFFB87F8248600240AE011
:104A7000012003F0B7FF641C5445D8D985E05048A5
:104A8000005D3055641C4E48F3F7F9FBA042F6D8A0
:104A9000CBF8004001214548F4F7FCFD05E001207A
:104AA00003F0A0FF641C54456FD897F82406002833
:104AB000F5D0642003F096FF002087F82406044612
:104AC00039484330B046025D3255641C0B2CF9D393
:104AD000601ECBF8000001213448F4F7DBFD05E04F
:104AE000012003F07FFF641C54454ED897F824063C
:104AF0000028F5D033A1304804F002F9061E37D063
:104B0000642003F06FFF00200446391881F8A8459F
:104B1000401C1428F9D30020494632180A44527820
:104B20003B1883F8AD25401C0F28F6D30021032045
:104B3000F4F7FAFF10B12448C0F88842642003F06B
:104B400051FF87F824461849002440463E390A5D43
:104B50000255641C072CFAD3601ECBF8000001211B
:104B60001248F4F797FD642003F03CFF564610E02E
:104B7000012003F037FF641C5445BBD905E0012038
:104B800003F030FF641CB44203D985F31388FCF7AB
:104B900047FF97F824060028F1D00B490020C1F800
:104BA000880207B0BDE8F08FF4900108B8640240B5
:104BB00049434349443A0000205E002090160020FB
:104BC0001C080020493A0000000042422DE9F0474D
:104BD0000020574E01463154401C6428FBD3554DEC
:104BE000884685F82416544900200A5C3254401C3B
:104BF0000828FAD3002705F2E45405E0E81990F8F4
:104C0000E405F11908727F1C2046F3F738FBB8421F
:104C1000F4D82C20F1190872002405F20C69093728
:104C200005E0281990F80C0639197054641C4846A0
:104C3000F3F725FBA042F4D840A13D48F3F713FB5E
:104C40003B48F3F71CFB3E4F3860A7F1040A0121F3
:104C50005046F4F71FFD05E0012003F0C3FE641C7D
:104C6000642C03D895F824060028F5D03548D0F8F0
:104C7000180231491D31B8B1002042463254401C5F
:104C80006428FBD3A84685F824260024085D305507
:104C9000641C0E2CFAD32C48F3F7F1FA0004000C34
:104CA00031D00024414628E04046A84685F8240635
:104CB0000024894603E019F804003055641C1E489E
:104CC0001D30F3F7DCFAA042F5D83C6001215046D4
:104CD000F4F7E0FC464605E0012003F083FE641C87
:104CE000642C1FD896F824060028F5D01AE00A197B
:104CF00092F8762533199A73641C8442F7D30FA176
:104D00000B48F3F7B0FA0A48F3F7B9FA3860012113
:104D10005046F4F7BFFC05E0012003F063FE641C7D
:104D2000642C03D895F824060028F5D0BDE8F08758
:104D30004E080020D4100020429101080D0A000006
:104D4000BC640240000043424A1600202DE9FC5F8B
:104D50000121592000F0BAF800248DF80440022007
:104D6000DFF894B04FF47C578DF807000097694640
:104D70005846F5F7B9FAFC20DFF8809000908DF8DE
:104D8000044001258DF8075069464846F5F7ACFA0E
:104D9000DFF86CA04FF440468DF8044000968DF883
:104DA000075069465046F5F79FFA0720DFF8548010
:104DB00000908DF804408DF8075069464046F5F79D
:104DC00093FA07214046F5F7E4FA31465046F5F7E5
:104DD000E0FA39465846F5F7DCFAFC214846F5F783
:104DE000D8FA0948D0F828120848012902D00470DE
:104DF000BDE8FC9F0570FBE7001002400018024070
:104E0000000C02400000024000004242D41000208A
:104E100010B5FFF79BFF642003F0E4FD1048D0F8C5
:104E20003C12104819B1002180F8221610BD0E491D
:104E3000D1F8182292B1012280F82226D1F8082256
:104E4000D1F80C1242EA4101C94380F8231690F8C8
:104E5000231601F0030180F8231610BD0222EBE7B0
:104E600000804142D4100020000043427CB5012163
:104E7000102000F02BF84CF20400012400908DF873
:104E8000044000208DF8060003208DF80500084D31
:104E90008DF8074069462846F5F726FA042128468A
:104EA000F5F775FA0348C0F8B842C0F8BC427CBDBB
:104EB0000010024000004242FFF7D8BF4FF40061EB
:104EC0000148F5F75DBA000000040240044A0029D9
:104ED000116801D0014300E0814311607047000078
:104EE00030380240044A0029116801D0014300E033
:104EF000814311607047000010380240044A0029C5
:104F0000116801D0014300E0814311607047000047
:104F100034380240044A0029116801D0014300E0FE
:104F2000814311607047000040380240044A002964
:104F3000116801D0014300E0814311607047000017
:104F400020380240044A0029116801D0014300E0E2
:104F5000814311607047000044380240044A002930
:104F6000116801D0014300E08143116070470000E7
:104F70002438024070B5204B1968204C11F00C0108
:104F800004D06610042903D0082903D004601BE074
:104F9000066019E0184A121F1168C1F380551168A4
:104FA00001F03F0115B1B6FBF1F101E0B4FBF1F105
:104FB00014681268C4F388146143C2F30142521C9E
:104FC0005200B1FBF2F1016019680F2202EA1111DF
:104FD0000B4A545C0168E14041601C68072505EA02
:104FE0009424145D21FA04F484601B6805EA5333A9
:104FF000D25CD140C16070BD083802400024F4008A
:105000000000002005490028086802D040F0040094
:1050100001E020F00400086070470000000806501E
:1050200001480068704700000808065070B501206C
:1050300080F310880C4D10212846F5F7A8F90821B7
:105040002846F5F7A6F9D720F4F712F8FF20F4F771
:105050000FF8044610212846F5F79BF9002181F34B
:105060001088204670BD00000000024070B501208D
:1050700080F31088194C0020A080FFF7D7FF0006AE
:1050800009D4012003F0AEFCA088401C80B2A080AF
:10509000C828F2D31EE0A088C8281BD2104D1021CA
:1050A0002846F5F774F908212846F5F772F99F208C
:1050B000F3F7DEFFFF20F3F7DBFFFF20F3F7D8FF66
:1050C000607010212846F5F764F9002080F31088FD
:1050D000607870BD002080F3108870BD1E10002025
:1050E0000000024070B5012188B08803FFF712FF6D
:1050F00001210220FFF7EAFE00244FF400602F4E4A
:105100008DF8044000908DF8074069463046F5F769
:10511000EBF801218DF8041002258DF805500803E5
:105120008DF806408DF80710009069463046F5F777
:10513000DBF805220D213046F5F712F905220E2184
:105140003046F5F70DF905220F213046F5F708F93D
:105150004FF4604000908DF8045003208DF8050056
:105160008DF806408DF8074069463046F5F7BCF8E3
:10517000134D284600F04AF8ADF810406815ADF818
:1051800012001820ADF814000720ADF81800ADF893
:1051900008404FF48270ADF80C40ADF80A00ADF84D
:1051A0000E40ADF8164002A9284600F064F801212F
:1051B000284600F021F808B070BD0000000402404D
:1051C0000038004070B50B4C05460221204600F027
:1051D00047F80028F9D02946204600F04AF8012176
:1051E000204600F03DF80028F9D0204600F03FF8B6
:1051F000C0B270BD003800400029018802D041F0E3
:10520000400101E021F0400101807047114910B5D3
:1052100088420AD1841401212046FFF79FFE2046D0
:10522000BDE810400021FFF799BE0B49884202D12A
:105230000121041404E0094988420AD10121C41360
:105240002046FFF773FE2046BDE810400021FFF71F
:105250006DBE10BD0030014000380040003C0040F1
:105260000246002012890A4200D00120704780893E
:1052700070478181704730B502884C8802F44153F1
:105280000A88CD8822438C882C4322430C892243F0
:105290004C8922438C892243CC8922431A430280C1
:1052A000828B22F400628283098A018230BD024629
:1052B000002003E012F8013B1844C0B2491E89B235
:1052C000F8D2704770B501218D070024284601F0FF
:1052D00051FBE8B3F5F702FB0020264B3BE003EB64
:1052E0008401D1F840261278012AD1F8402603D053
:1052F0005278012A08D02AE01070D1F84026507068
:10530000D1F84026907030E0D1F840269278F2B97A
:10531000D1F840265668761C5660D1F8402652686F
:10532000D1F84066B668B24211D3D1F84066012286
:10533000B270D1F84026D278012A16D0D1F8402692
:105340005070D1F840265060D1F84016C87000E087
:1053500005E0641CE4B293F83E16A142BFD828468B
:10536000BDE87040012101F04FBAD1F84016486005
:10537000EDE70000D41000200CB500222549009272
:105380000192086840F4803008604FF4A063086818
:1053900000F4003001900098401C0090019810B972
:1053A00000989842F3D10868800330D5012001901D
:1053B00018484030026842F0805202601648026885
:1053C00042F48042026013480830026802600268BA
:1053D000026002680260031F104A1A600A6842F005
:1053E00080720A600A689201FCD50D4A40F205619C
:1053F0001160016821F003010160016841F00201C0
:1054000001600168C1F381010229FAD10CBD01924A
:105410000CBD0000003802400070004008544007F6
:10542000003C02407CB500229FED170A00928DEDF2
:10543000010A6D4601AC16E0835CA3F13006102E24
:1054400005D2009B1B010093865C303E07E0413B88
:10545000062B0CD2009B1B010093865C373E1E433B
:10546000521CD2B200968A42E6D3002006E0BFEE7C
:10547000000A7CBD2A5C2254401CC0B2B0EB510F24
:10548000F8D39DED010A7CBD0000000030B5054653
:105490000022104611E0AB5CA3F13004102C02D2C4
:1054A00044EA001007E0A3F14104062C08D20401ED
:1054B000A3F137002043521CD2B28A42EBD330BD55
:1054C0004FF0FF3030BD00002DE9FC414E4D4FF054
:1054D000380895F86A02002105F51A75FBF7F0FB0C
:1054E00001240826CDE90064024618200023414625
:1054F000FCF7B8FC071D07EB47004006000E082329
:105500002D2241460094FCF73FFC687800217F1C67
:10551000FBF7D6FB024607EB4700CDE900644006E7
:10552000000E00234146FCF79DFC074407EB4700B3
:105530004006000E08232D2241460094FCF724FC6F
:10554000287800217F1CFBF7BBFB024607EB4700D6
:10555000CDE900644006000E00234146FCF782FCC2
:10556000074407EB47004006000E0823202241466F
:105570000094FCF709FC687900217F1CFBF7A0FB75
:10558000024607EB4700CDE900644006000E002309
:105590004146FCF767FC074407EB47004006000E56
:1055A00008232D2241460094FCF7EEFB28790021C8
:1055B0007F1CFBF785FB024607EB4700CDE9006443
:1055C0004006000E00234146FCF74CFC074407EB65
:1055D00047004006000E08232D2241460094FCF7A8
:1055E000D3FBE87800217F1CFBF76AFB024607EB40
:1055F0004700CDE900644006000E00234146FCF759
:1056000031FCBDE8FC810000D41000200249C870C4
:105610000120887170470000D41000202DE9FC5F44
:1056200000252C46F4F79CFCF84FB87900287CD074
:10563000A94687F80690FCF703FAF878DFF8D0B3AC
:1056400001264FF008084FF0100A0E286ED2DFE84E
:1056500010F00E008200EB007901BD01E402370476
:105660005C05A505F205850646078F07E307F5F7F4
:1056700025F901280AD0022808D0042806D00828D5
:1056800004D10220FFF7C2FF87F86090CDE900A6A1
:1056900000211523DFA20846FCF781FC97F8610082
:1056A00010B3CDE9008644460523DFA21421002073
:1056B000FCF775FCCDE9004697F861200023142122
:1056C0001E20FCF7CFFBCDE9004697F861000A23C6
:1056D00000EB400101EB001007EB00121421282021
:1056E00002F6EE02FCF75BFC97F86000FF2825D07D
:1056F00017F8600FCDE900060A2364221E21184620
:10570000FCF7C0FACDE900863A7800232D2132203B
:10571000FCF7A8FB00EB4000322101EB400008231E
:105720002522C0B22D21009601E0D2E30EE3FCF762
:105730002BFB17F86009642807D007E3CDE9008642
:1057400015232D21BAA2142044E287F8609002208C
:10575000FFF75CFFF1E7F5F7B1F801280BD002285D
:1057600009D0042802D0082805D101E0082000E073
:105770000320FFF74BFF97F8210638B197F8220670
:1057800038B1012808D0022811D108E01523ACA2B5
:1057900007E01523ADA204E01523B0A201E0152314
:1057A000B1A2CDE9008600210846FCF7F8FBB878E5
:1057B000012802D002280CD101E0AF4801E0AE4838
:1057C0001230CDE9000609231A460A210020FCF711
:1057D00099FBA94818234838CDE900061A4600214C
:1057E0006820FCF78FFBCDE9008644461523A3A271
:1057F0001A210020FCF7D3FBCDE900461523A5A212
:1058000024210020FCF7CBFBCDE900467A6D002374
:1058100024215420FCF726FB786D10B90220FFF7F5
:10582000F5FEFFF751FE88E7F5F748F8012806D0A6
:10583000022804D0042809D0082818D10EE097F8CF
:105840005C0020F0800087F85C0010E097F85C00B6
:1058500020F0800087F85C00082006E097F85C00E4
:1058600020F0800087F85C000320FFF7CFFE97F858
:10587000210638B197F8220668B101280ED0022817
:1058800014D118E0CDE900860021152385A2084631
:10589000FCF785FB15E015236CA201E015236FA230
:1058A000CDE9008600210846FCF779FB97F8E7046C
:1058B0000F2803D005E015236BA2F1E70120FFF7C5
:1058C000A5FEB878012802D002280CD101E06A4870
:1058D00001E069481230CDE9000609231A460A2181
:1058E0000020FCF70FFB97F8600010B10020FFF7D5
:1058F0008DFE614818234838CDE900061A4600217C
:105900006820FCF7FFFACDE900A65446102367A2F1
:1059100014212820FCF743FBCDE90086152365A25E
:1059200024211220FCF73BFB97F85C0000067FF572
:1059300078AFCDE90046102363A22E210020FCF7AA
:105940002EFB6EE7F4F7BAFF012806D0022809D033
:1059500004280ED008281ED121E03879D8B1387932
:10596000401E04E03879032815D23879401C38717C
:1059700011E0387930B1012806D0022806D003287A
:1059800009D105E0042004E0052002E0062000E043
:105990000720FFF73BFEF878032805D0CDE602206C
:1059A000FFF734FE4846E2E7334804220021243062
:1059B00000F0C8FECDE900A938792F49243101EB68
:1059C000001238790007010E1023F2E3F4F776FF96
:1059D000082802D10320FFF719FEF8780428DDD14A
:1059E000254804220021643000F0ACFE97F822061E
:1059F00020B1012875D0022872D198E01023CDE99A
:105A0000008612A21946002083E06AE0D41000202C
:105A1000000042424669726D77617265446F776E2D
:105A20006C6F616400000000506F72743A000000F7
:105A3000446F776E6C6F6164204661696C21000071
:105A40004E6F205369676E616C0000005479706579
:105A50003A53746174696F6E000000005479706588
:105A60003A436C6F75640000547970653A436C6F0B
:105A700075642D546573740010B001084F66666C30
:105A8000696E65205265636F72642055706C6F613A
:105A9000640000005265636F7264206E756D62650C
:105AA000723A00004F66666C696E6500424C55455F
:105AB000534B5900454E4552475920544543484E93
:105AC0004F4C4F4759000000557067726164652064
:105AD00045525220436865636B2047756E00000095
:105AE00019E044461023AFF28C02CDE90086194636
:105AF0000020FCF754FACDE900461023F5A2382126
:105B00000020FCF74CFACDE900461123F34A382176
:105B10001E20FCF744FA97F8230600B397F82306F3
:105B200001281CD097F82306022854D005E6CDE9B9
:105B3000008610234446EAA219460020FCF72FFAFB
:105B4000CDE900461023E3A238210020FCF727FA14
:105B5000CDE9004611233821E54A1E20D9E77819FE
:105B600090F8610518B96D1CADB2152DF7D3CDE9CC
:105B7000008644461023DFA21A210020FCF70FFA0A
:105B8000CDE900467A1910231A21202002F2615231
:105B9000FCF705FACDE900461023D8A22421002005
:105BA000FCF7FDF9CD4ACDE9004624211023393216
:105BB0000846FCF7F4F9CDE900461023D1A22E21C6
:105BC0000020FCF7ECF9C54ACDE900460F232A3244
:105BD0002E2124202EE3CDE9008644461023CBA2BB
:105BE00024210020FCF7DBF9BC4ACDE90046102354
:105BF000613224211E20FCF7D2F9CDE900461023A2
:105C0000C0A22E210020FCF7CAF9B44ACDE9004613
:105C1000102329322E211E200CE3F4F74FFE012819
:105C200004D0022807D008280FD10BE0387960B1E2
:105C30003879401E04E03879032806D23879401CB0
:105C4000387102E00320FFF7E1FCF87805287DD1E8
:105C500004220021AF4800F075FDCDE900A63A7995
:105C6000BA46012300213E20521CFCF7FBF8CDE987
:105C7000008647461023A8A200214820FCF78FF990
:105C8000DFF890820823A8F1F408CDE900861A46CF
:105C900000217820FCF736F9CDE900761023A1A287
:105CA00008214820FCF77BF908231A46194678207A
:105CB000CDE90089FCF726F9CDE9007610239CA2F6
:105CC00019460020FCF76BF99AF8040000EB40013C
:105CD00001EB00110AEB011090F81D0A4FF01003C0
:105CE000012840D094A2CDE9007610211E20FCF7B7
:105CF00056F9CDE90076B046102391A21821002074
:105D0000FCF74DF99AF8040000EB400101EB00109C
:105D10000AEB001090F8160ACDE9007805289AF8E9
:105D2000040000EB400101EB00100AEB00101CD056
:105D300090F8160A7749403101EB00120C23182124
:105D40003620FCF72CF9C346B84600E025E2CDE941
:105D5000007B10237DA220210020FCF720F90927D9
:105D60004FF0200A9EE07CA2BDE790F81C0A69492A
:105D7000B031E1E707EB47014FF07A09B9EB410F8A
:105D800002D2641CA4B20027307900EB400101EB81
:105D9000001006EB001000EB051090F8420AC00955
:105DA000CDE90080307900EB400101EB001006EBFB
:105DB000001000EB051090F8402A0AEBC400C1B2B5
:105DC00007EB47004006000E0023FCF74BF8384471
:105DD00087B207EB4701B9EB410F02D2641CA4B2B2
:105DE0000027307900EB400101EB001006EB0010BA
:105DF00000EB051090F8420A0823C00900900AEB56
:105E0000C400C1B207EB47004006000E2D22FBF78D
:105E1000BBFF7F1CBFB207EB4701B9EB410F02D2BA
:105E2000641CA4B20027307900EB400101EB0010A4
:105E300006EB001000EB051090F8420AC009CDE90E
:105E40000080307900EB400101EB001006EB001000
:105E500000EB051090F8412A0AEBC400C1B207EB31
:105E6000470040065646000E0023FBF7FBFF384470
:105E700087B207EB4701B9EB410F02D2641CA4B211
:105E8000002706EBC400C1B207EB47004006000E36
:105E900008233B22CDF800B0FBF776FF7F1C6D1C7A
:105EA000BFB2ADB22E4E307900EB400101EB0010D5
:105EB00006EB001090F8170AA8423FF65BAFD1E35B
:105EC000F4F7FCFC01284DD0022850D0082858D106
:105ED00054E0CBE355524C3A000000005716002026
:105EE000547970653A436C6F75642D546173740016
:105EF000CA900108494343494400000041504E20E4
:105F00003A000000494D45493A00000053534944C6
:105F10003A000000B4B001084F6E4C696E65203A3B
:105F2000200000004F66664C696E653A2000000054
:105F3000547970653A00000052533438350000003F
:105F400050726F746F636F6C3A00000047756E2D6E
:105F5000416464723A0000004C4F5241000000005E
:105F6000D4100020387940B13879401E04E03879E7
:105F7000032806D23879401C387102E00320FFF76D
:105F800045FBF87806289AD10126BE71042200212B
:105F9000F84800F0D7FBCDE900A63A7901230021AB
:105FA0004020521CFBF75EFFCDE90086C34610235C
:105FB000F1A214210020FBF7F2FF092697E006EB7F
:105FC00046014FF07A0ABAEB410F02D2641CA4B228
:105FD00000264FF00108CDE900B8387900EB400108
:105FE00001EB001007EB001000EB051090F8402AC1
:105FF0004FF0140909EBC400C1B206EB460040069D
:10600000000E0023FBF72EFF304486B206EB46015C
:10601000BAEB410F02D2641CA4B20026142000EB9C
:10602000C400C1B206EB46004006000E08232D2234
:10603000CDF80080FBF7A8FE761CB6B206EB460151
:10604000D146BAEB410F02D2641CA4B20026CDE9BE
:1060500000B8387900EBC00101EB002007EBC0006D
:1060600005EB451100EB810090F8140F642110FB43
:1060700001F0020A142707EBC400C1B206EB460088
:106080004006000E0023FBF7EDFE304486B206EB1F
:106090004601B9EB410F02D2641CA4B2002607EB03
:1060A000C400C1B206EB46004006000E08232522BC
:1060B000CDF80080FBF768FE761CB6B206EB460111
:1060C000B9EB410F02D2641CA4B2002607EBC40056
:1060D000C1B206EB46004006000E08233B22CDF875
:1060E0000080FBF751FE761C6D1CB6B2ADB2A54F19
:1060F000387900EB400101EB001007EB001090F83D
:10610000170AA8423FF65BAFACE2F4F7D7FB0828CA
:1061100002D10320FFF77AFAF8783C460728F3D13A
:10612000944804220021403000F00CFBCDE90086A9
:1061300047461023944A14210020FBF730FFA14664
:1061400005EB450000EB051109EB0110804690F8C6
:10615000280AC0071DD005EB8501142000EB41047F
:10616000CDE90076E1B2052388A20020FBF717FFF6
:10617000CDE90076E1B201236A1C1E20FBF772FE16
:10618000CDE9007608F61E22E1B20A232A20FBF7A9
:1061900006FF6D1CADB2042DD2D363E2F4F78EFB83
:1061A000012807D002280CD0042812D0082828D1B2
:1061B0002BE03EE0387910B13879401E1CE0052014
:1061C0001AE03879042802D23879401C14E0484695
:1061D00012E03879052814D2DFE800F0030507093A
:1061E000100009200BE00A2009E00B2007E00C203A
:1061F000FFF70CFA97F82006387102E00D20FFF740
:1062000005FAF878082804D02CE20220FFF7FEF9FE
:10621000DDE73879574C0422803404EB001000216C
:1062200000F090FACDE900A93879102304EB0012B0
:1062300000210020EDE1F4F741FB012806D00228FF
:1062400009D004280ED0082849D145E0387978B320
:106250003879401E04E03879032840D23879401C50
:1062600038713CE0387900EB400101EB001007EB9E
:10627000001090F81D0A01280AD0387900EB40017F
:1062800001EB001007EB001090F81D0A88B126E022
:1062900038794C4600EB400101EB001007EB001091
:1062A00080F81D9A39790220F3F73EFCCBF888423A
:1062B00015E0387900EB400101EB001007EB00100E
:1062C00080F81D6A3879FBF7CFF9CBF88862397905
:1062D0000220F3F729FC02E00820FFF797F9F8788D
:1062E000092891D1042200212A4800F02BFACDE997
:1062F00000864446152328A214212820FBF74FFED0
:10630000CDE900463A79012314214620521CFBF7BF
:10631000A9FD387900EB400101EB001007EB0010FC
:1063200090F81D0A01280AD0387900EB400101EBF2
:10633000001007EB001090F81D0A18B10AE01523B1
:1063400017A201E0152319A2CDE900461E21002065
:10635000FBF725FE152318A2322105E1F4F7AEFA6A
:106360001A4C012834D002283DD0042848D00828EF
:106370005AD14AE094B1010847756E2D52535349E2
:106380003A000000D4100020108E0108506F727483
:106390002D000000A4B20108504F52543A000000F2
:1063A000545950453A4C4F52410000005459504501
:1063B0003A525334383500005061737320456E747F
:1063C0006572204368616E6765000000D44000205C
:1063D000387948B394F8490010B13879FBF744F99B
:1063E0003879401E0AE0387903281DD294F8490014
:1063F00010B13879FBF738F93879401C387113E05F
:1064000084F8496084F83D600EE00820FFF7FEF84C
:1064100084F83C6094F8490030B1CBF8889284F855
:1064200049903879FBF720F9F8780A282FD104220F
:1064300000218F4800F086F945461523AFF2A802E7
:10644000CDE9008612212820FBF7A9FDCDE90056F1
:106450003A79012312214620521CFBF703FDCDE9B6
:106460000056152383A21C210020FBF798FDCDE9DF
:106470000056152385A226210020FBF790FDCDE9CB
:106480000056152387A230210020FBF788FD94F8E1
:106490004900012854D1BE7194F83E0078B1CBF880
:1064A000889284F83E9038790121FBF7A7F9CDE96D
:1064B0000086152380A238210020FBF770FD94F898
:1064C0004800E8B384F84890CDE9008615237EA201
:1064D00038210020FBF763FDCBF88862C2E0F4F7B7
:1064E000EDF9012813D0022811D0042802D0082881
:1064F0000DD109E0F2F738FF142802D087F867922F
:1065000005E087F8676202E00820FFF77FF8F87877
:106510000B2815D1564804220021403000F012F912
:10652000CDE90086444615236BA21A210020FBF713
:1065300036FDCDE90046152324216CA2002000E0A1
:1065400069E0FBF72CFDCDE9004615236BA22E2157
:106550000020FBF724FD97F867024FF0150308B100
:106560006CA200E071A23821CDE90046002050E085
:10657000F4F7A4F9012806D002280BD0042812D081
:10658000082821D11DE0387910B13879401E08E083
:10659000022006E03879032802D23879401C00E056
:1065A0004846387110E0387987F82006002103202A
:1065B000F3F7BAFA40B10220FFF728F8FDF72AFEF8
:1065C00002E00820FFF722F8F8780C284AD1284882
:1065D00004220021803000F0B5F8CDE900A697F83C
:1065E00020065446224D1023C03505EB00121946F3
:1065F0000020FBF7D4FC97F820063979884231D087
:10660000CDE9004638790C2305EB0012202100204B
:10661000121DFBF7C4FC25E0F4F750F9012819D04E
:10662000022817D0042802D0082813D10FE0F3F76E
:10663000D1FA86F31388BFF34F8F3F4801683F4A72
:1066400001F4E06111430160BFF34F8FFEE70820C2
:10665000FEF7DCFFF8780D2804D104220021384829
:1066600000F070F8BDE8FC5FFBF752BBBDE8FC9F93
:10667000E4B20108313A4469702073776974636841
:106680002031616E6432204F4E000000323A496E74
:106690007365727420736C617665206D6F64756CC0
:1066A00065000000333A5061737320456E74657263
:1066B000205374617274000053746174653A5365B9
:1066C0006E64696E6700000053746174653A436FCD
:1066D0006D706C6574650000496E73657274205549
:1066E0002D4469736B204669727374005468616E3F
:1066F000205061737320456E74657200466F726D31
:1067000061743A46415433323B4D41583A33324733
:106710000000000046696E6420552D4469736B2C9F
:106720004F7574707574696E6700000053746174FE
:10673000653A49646C6500000CED00E00400FA0560
:10674000E4B301082DE9F84F0025924688468146BA
:10675000012715E000242E0109EB040101EB0810CC
:1067600000EB051000970278E006F1B2000E10234E
:10677000FBF70AFB641CE4B2102CEDD36D1CEDB2E8
:106780005545E7D3BDE8F88F0648002101728172B4
:1067900001214172C1726422026181710220FEF7FF
:1067A00035BF0000D4100020124810B5016841F434
:1067B000700101601048016841F0010101600E4A5A
:1067C00000210832116002680C4B1A400260031D60
:1067D0000B4A1A60026822F48022026006480C30DC
:1067E0000160FEF7C9FD03494FF000608039086081
:1067F00010BD000088ED00E000380240FFFFF6FE0B
:1068000010300024FEF75EBDC943018270470029A5
:10681000018802D041F0010101E021F00101018075
:1068200070470000464910B5884206D1012108464C
:10683000FEF794FB002101205BE0B0F1804F09D00E
:10684000404988420DD101210220FEF76FFB002153
:10685000022070E001210846FEF768FB00210120BC
:1068600069E03949884206D101210420FEF75EFB28
:10687000002104205FE03549884206D1012108202B
:10688000FEF754FB0021082055E03149884206D12B
:1068900001211020FEF74AFB002110204BE02D497A
:1068A000884206D101212020FEF740FB0021202054
:1068B00041E02949884206D101210220FEF74EFB22
:1068C0000021022015E02549884202D101210C0453
:1068D0000AE02349884202D101214C0404E0214905
:1068E00088420AD101218C042046FEF737FB0021A3
:1068F0002046BDE81040FEF731BB1B49884206D157
:1069000001214020FEF712FB0021402013E017492F
:10691000884206D101218020FEF708FB002180205B
:1069200009E0134988420AD1841501212046FEF767
:10693000FDFA00212046BDE81040FEF7F7BA10BD71
:10694000000001400004004000080040000C00402E
:1069500000100040001400400004014000400140CD
:10696000004401400048014000180040001C004065
:106970000020004002460020138A92890B4202EA5E
:10698000010202D0002A00D001207047002A82892B
:1069900001D00A4300E08A438281704730B5028803
:1069A000164C174DA0420DD0A8420BD0B0F1804F2D
:1069B00008D0144B984205D0134B984202D0134B89
:1069C000984203D122F070034A881A43104B984230
:1069D00006D0104B984203D022F440730A891A4320
:1069E00002804A68C2620A880285A04201D0A84299
:1069F00001D1897A01860121818230BD00000140E8
:106A0000000401400004004000080040000C004069
:106A1000001000400014004010B5FEF7F9F9FEF731
:106A20004BFA00F0A9F9F3F775F9154C14F85C0F5F
:106A300020F001002070207840F006002070002037
:106A4000608001460120F3F76FF8F3F787FEF2F755
:106A500097FAF2F7FBFEF3F749FFFAF785FCFDF72B
:106A6000D9FBFBF763F8FFF78FFEF3F7BDFA4FF49E
:106A7000FA6024F8460C012004F8480C10BD000010
:106A8000D41000202DE9F0410024F3F785FCB94E25
:106A900096F8F2040025012805D186F8F254F2F7A1
:106AA0001DFF0120B0713AE104EB440006EB8000C9
:106AB00090F83215012901D180F8325590F831153E
:106AC000002979D190F8A2190129FAD104EB4401E7
:106AD00001EB041106EB011292F8161A00296BD093
:106AE00080F8A25992F8160A072864D2DFE800F06D
:106AF000EC04376591E1E10004EBC40000EB0420F5
:106B000006EBC00090F8D31E012909D090F8D21EE0
:106B100001EB411100EB810191F8D81E00294AD107
:106B200090F8D21E491C80F8D21E90F8D01E29B1D0
:106B300090F8D01E80F8D21E80F8D05E90F8D21E59
:106B400001EB411100EB810191F8D81E052932D0EB
:106B500090F8D21E01EB411100EB8100A6E004EB9E
:106B6000C40000EB042006EBC00090F8D31E0129FE
:106B700009D090F8D21E01EB411100EB810191F890
:106B8000D81E002917D190F8D21E491C80F8D21EB9
:106B900090F8D01E29B190F8D01E80F8D21E80F84F
:106BA000D05E90F8D21E01EB411100EB810191F80B
:106BB000D81E0F29CCD187E0AFE004EBC40000EB76
:106BC000042006EBC00090F8D31E012908D090F8ED
:106BD000D21E01EB411100EB810191F8D81E71BB6F
:106BE00090F8D21E491C80F8D21E90F8D01E29B110
:106BF00090F8D01E80F8D21E80F8D05E90F8D21E99
:106C000001EB411100EB810191F8D81E07299FD1BA
:106C10005AE004EBC40000EB042006EBC00191F83D
:106C2000D30E012808D091F8D20E00EB401001EBF2
:106C3000800090F8D80E10B991F8D20E19E037E024
:106C400091F8D23E02EB031393F8413A02EB00179E
:106C500097F8517ABB4205D091F8D20E401C81F8CA
:106C6000D20E0AE091F8D23E5B1C81F8D23E401C65
:106C7000C0B292F8173A8342E2D891F8D00E28B108
:106C800091F8D00E81F8D20E81F8D05E91F8D20E34
:106C900000EB401001EB800090F8D80E052813D0CF
:106CA00091F8D20E00EB401001EB800080F8D85E26
:106CB0000AE004EBC40000EB042006EBC00090F8EF
:106CC000D21E491C80F8D21E04EBC40000EB042045
:106CD00006EBC00090F8D21E92F8172A914201D319
:106CE00080F8D25E90F8D11E51B190F8D21E80F893
:106CF000D01E90F8D11E491E80F8D21E80F8D15EB9
:106D000090F8D21E01EB411100EB810191F8DC2ECD
:106D100090F8D21E2046F8F7C9FD641CE4B296F83C
:106D20006C09A0423FF6C0AE96F8220620B196F854
:106D3000FE04012807D010E096F80A0501280CD1BE
:106D400086F80A5501E086F8FE5496F8252696F84E
:106D5000211696F82206FCF71BFDF3F7AFFE96F816
:106D6000240618B186F82456FBF768F9BDE8F0410F
:106D7000FEF754BCD4100020FEB5012100240846C3
:106D8000FEF7C8F8A720ADF80000002640F2E73073
:106D900001904FF08045ADF80260ADF8086069469B
:106DA0002846FFF7FBFD724981F83E6604EB44007C
:106DB00001EB800091F83E3600F5A66201EB8303FB
:106DC000C3F8402691F83E26521C81F83E2691F8E1
:106DD0003E3600F51A6201EB8303C3F8402691F8B2
:106DE0003E26521C81F83E2691F83E3600F5176289
:106DF00001EB8303C3F8402691F83E26521C81F82C
:106E00003E2691F83E2600F5405001EB8202C2F882
:106E1000400691F83E06401C81F83E0604EBC40291
:106E200002EB0422002001EBC20300EB401291F8B8
:106E30003E6603EB820201EB860602F6E462C6F8C8
:106E4000402691F83E26521C81F83E26401CC0B2D6
:106E50001028EAD3641CE4B2042CA7D3454891F867
:106E60003E2601EB8202C2F8400691F83E06401C25
:106E700081F83E063F4891F83E26283801EB820211
:106E8000C2F8400691F83E06401C81F83E0639489B
:106E900091F83E261C3801EB8202C2F8400691F8B8
:106EA0003E06401C81F83E06324891F83E261038D6
:106EB00001EB8202C2F8400691F83E06401C81F8C0
:106EC0003E062D4891F83E2601EB8202C2F84006AC
:106ED00091F83E06401C81F83E06284891F83E266F
:106EE00001EB8202C2F8400691F83E06401C81F890
:106EF0003E06204891F83E26343801EB8202C2F863
:106F0000400691F83E06401C81F83E061C4891F868
:106F10003E2601EB8202C2F8400691F83E06401C74
:106F200081F83E06124891F83E26083001EB8202B5
:106F3000C2F8400691F83E06401C81F83E06104813
:106F400091F83E260C3801EB8202C2F8400691F817
:106F50003E06401C81F83E0601212846FFF757FCFB
:106F6000012211462846FFF711FD00F00BF8FEBD87
:106F7000D4100020F8150020FC160020341A002040
:106F80001041002008B51C208DF8000001208DF86C
:106F9000010002218DF802108DF803006846FAF70F
:106FA00003FD08BDF9F7FABEF9F718BFFDF760B8A1
:106FB000F9F7CEBEF9F730BFF3F7ECBAC943018059
:106FC00070470029818902D041F4005101E021F489
:106FD000005181817047002A828A01D00A4300E073
:106FE0008A438282704700001C4910B5884206D14E
:106FF00001211020FDF7B2FF0021102028E01849E0
:10700000884202D101214C0410E01649884202D185
:1070100001218C040AE01449884202D10121CC04E8
:1070200004E0124988420AD101210C052046FDF7EF
:107030007DFF2046BDE810400021FDF777BF0C49D9
:10704000884209D101212020FDF788FF002120205E
:10705000BDE81040FDF782BF10BD000000100140E8
:107060000044004000480040004C004000500040F8
:10707000001401400246002012880A4200D001207C
:10708000704770B501F01F0501260024C1F34213BB
:1070900006FA05F2012B0FD0022B0FD0838A4FEA9C
:1070A00011210088134206FA01F600EA060001D019
:1070B00000B10124204670BD8389F0E7038AEEE722
:1070C00010B5C1F3421301F01F040121A140012BAF
:1070D00007D0022B07D01430002A026805D00A43DB
:1070E00004E00C30F8E71030F6E78A43026010BD88
:1070F0007FB50446008A0D46C98820F440500143FC
:107100002182A08941F20C618843A9882A89114310
:107110006A8902431143A181A08A20F44071A889A1
:107120000843A0826846FDF725FF1A48844202D032
:107130001948844201D1039800E00298A18909040A
:1071400000EBC00101EB0010296801D5490000E007
:107150008900B0FBF1F06422B0FBF2F109010B09E8
:107160006FF018056B4300EB8300A3891D044FF0FB
:10717000320306D503EBC000B0FBF2F000F00700CD
:1071800005E003EB0010B0FBF2F000F00F00084345
:1071900020817FBD001001400014014070B5002423
:1071A000064DFDF78BFE20B1641CAC42F9D3FA20EA
:1071B00070BDBDE87040F2F705B90000404B4C00CF
:1071C0000FB4084B10B504A902AA039801F0D4F932
:1071D000044602A9002001F000FC204610BC5DF826
:1071E00014FB0000DB89010803B4019841000098FA
:1071F00050EAC12018BF04204A0D18BF40F001001A
:1072000040F2FF72B2EB515F08BF40F0020001286C
:1072100008BF052002B0704730B583B0044601F0C6
:1072200087F99FED090B05468DED000B00222146E5
:107230006846F1F76AFA284601F090F99DED000BD7
:1072400003B030BD0000000000000000000000009E
:1072500070B5D94B00242DED020B2DED108BDDE91F
:107260001010984205DA20F000429A4201D809D164
:1072700041B19DED100BBDEC108B02B0BDE870402C
:1072800001F012B9B0F5801F26DA11430BD00028A7
:1072900013DA012001F062F9BDEC108B02B0BDE8F9
:1072A000704001F015B9022001F058F901F0E4F83E
:1072B00051EC100B81F000419EE06FF035049FED22
:1072C000C00B53EC102B9DED100B51EC100BF1F794
:1072D00093F8CDE91001084604EB2051C0F31304E4
:1072E000B948A1F2FF31204400F4801080F07F62A1
:1072F00082F04052224301EB20559FEDB50B1192D5
:1073000053EC102B9DED100B51EC100BF1F76EF8B8
:1073100041EC180BA01CC0F313009FEDAFDB9FEDF9
:10732000B0EBB14E7E4403286CD296ED000B51ECCD
:10733000180B53EC102BF1F715FD1DD1002D01BFDB
:1073400096ED000BBDEC108B02B070BD2846F1F736
:10735000BAFA41EC180B53EC1D2BF1F74DF841EC48
:10736000190B53EC1E2B51EC180BF1F745F853ECAD
:10737000192BF0F79AFF3FE09FED9D0B51EC180B96
:1073800053EC102BF1F738F89FED9B1B53EC112BAE
:10739000F1F72FF841EC190B53EC182B51EC180BAB
:1073A000F1F72AF853EC192BF1F726F841EC190BF9
:1073B000002D04BF53EC192B51EC180B1AD02846A2
:1073C000F1F781FA41EC1A0B53EC1D2BF1F714F88D
:1073D00053EC192BF1F70DF853EC182BF1F706F8D5
:1073E00041EC180B53EC1E2B51EC1A0BF1F704F87F
:1073F00053EC182BF0F7FAFFBDEC108B02B041EC08
:10740000100B70BD9FED7E0B51EC180B53EC102B45
:10741000F0F74BFF41EC100B51EC180B53EC102B19
:10742000F1F75CF841EC190B2846F1F74CFA41EC06
:107430001B0B53EC192B51EC190BF0F7DDFF41EC52
:107440001A0B714853EC1A2B261851EC1A0BF0F753
:10745000D3FF41EC1F0B6D48C4F1510404F5D72450
:10746000B0EE4F0AF0EE6F0A0321784400F088FF77
:1074700053EC1F2B51EC100BF0F7BEFF41EC1C0B33
:107480006348B0EE4F0AF0EE6F0A0421784400F032
:1074900077FF53EC1A2B51EC100BF0F7ADFF344390
:1074A00053EC1C2BF0F701FF41EC1C0B002C4CDDC6
:1074B0009FED510B51EC180B53EC102BF0F79CFF88
:1074C00053EC182BF0F798FF41EC1A0B55B353EC23
:1074D0001D2B51EC1B0BF0F78FFF41EC1D0B53ECF8
:1074E0001C2B51EC1A0BF0F7E0FE53EC192BF0F7C4
:1074F00083FF53EC1D2BF0F7D8FE53EC1A2BF0F75B
:1075000078FF53EC182BF0F771FF41EC180B53EC9C
:107510001E2B51EC1B0BF0F76FFF53EC182BF0F701
:1075200065FF69E753EC1C2B51EC1A0BF0F7BDFE1D
:1075300053EC192BF0F760FF53EC1A2BF0F759FFBF
:1075400053EC182BF0F755FF56E735B353EC1D2BD2
:1075500051EC1B0BF0F750FF41EC1A0B53EC1C2BBA
:1075600051EC180BF0F742FF53EC192BF0F744FFE6
:1075700053EC1A2BF0F73AFF53EC182BF0F736FFC9
:1075800041EC180B53EC1E2B51EC1B0BF0F734FFA6
:1075900053EC182BF0F72AFF2EE753EC1C2B51EC81
:1075A000180BF0F723FF53EC192BF0F725FF53ECE2
:1075B000182BF0F71EFF1FE70000F07F000000000F
:1075C0000000000000005043645F0900000000005C
:1075D000000000000000F03F763C7935EF39EA3DCD
:1075E0000000E0FE422EE63FC04100000000000027
:1075F000555555555555D53F000000000000E03F5A
:10760000000000000000004086EBF9FF424000004F
:10761000384000000000000070B5414A00252DED03
:10762000020B2DED048BDDE90404944205DA24F00D
:107630000041914201D809D140B19DED040BBDEC50
:10764000048B02B0BDE8704000F02EBFB4F5801F7F
:1076500026DA08430BD0002C13DA012000F07EFF5D
:10766000BDEC048B02B0BDE8704000F031BF0220D9
:1076700000F074FF00F000FF51EC100B81F00041AE
:1076800046E09FED290B6FF0350553EC102B9DED77
:10769000040B51EC100BF0F7AFFECDE904010C46E2
:1076A00005EB2450A0F2FF30C10F40F2FF32521A16
:1076B00062F31F540844F1F706F905949DED040B9D
:1076C00041EC180B51EC100B01F0AEFA9FED181BBA
:1076D00053EC112BF0F790FE9FED170B41EC190BBB
:1076E00053EC102B51EC180BF0F786FE53EC192BD2
:1076F000F0F7DBFD9FED120B41EC190B53EC102B57
:1077000051EC180BF0F778FE53EC192BF0F7CDFD88
:10771000BDEC048B02B041EC100B70BD000000000A
:107720000000F07F00000000000000000000504357
:107730000EE526157BCBDB3F362BF111F3FE593DD1
:1077400000609F501344D33F2DE9F04D2DED040B05
:107750002DED0C8B96B0DDE92350259CDDF888A03B
:1077600025F0004624F00048BAF1000F14BF0121B3
:10777000002101EB4502FE4953184A1093422AD3D7
:10778000002814BF0123002303EB44030B44F949F1
:107790008B4220D358EA00019FEDF78B6FD0DFF8C2
:1077A000E0B35D4503D1BAF1000F05D187E0BAF12E
:1077B000000F08BF002100D0012101EB450111F5A8
:1077C000001F08D8002814BF0121002101EB44014B
:1077D00011F5001F0BD99DED241B9DED220B16B05A
:1077E000BDEC0C8B04B0BDE8F04D00F067BE002787
:1077F000002DBCBFE349884521DAE3498845A8BF8D
:1078000002271CDAC3451ADCE04901EB2851142990
:1078100008DDC1F1340220FA02F101FA02F28242DB
:107820000DD108E058B9C1F1140228FA02F101FAA9
:1078300002F2424503D101F00101C1F1020756EA0B
:107840000A011DD1002C1BDA002D18BF022F01D018
:10785000012F0AD0022000F081FE16B0BDEC0C8B87
:1078600004B0BDE8F04D00F007BE022000F076FE47
:1078700000F002FE51EC100B81F0004183E01EE0AD
:107880009FEDC39B9FEDC4AB002872D1BD488045DE
:107890002DD105F1804010F5801008BFBAF1000F1E
:1078A0000DD0B34515DC002CA1BF9DED240B16B007
:1078B000BDEC0C8B04B0A8BFBDE8F08D12E0B0EEBB
:1078C000480AF0EE680A16B0BDEC0C8B04B0BDE8B7
:1078D000F08D002C06DA9DED240B51EC100B81F09D
:1078E000004150E0AE48784490ED000BEBE7D845FE
:1078F0004FD1002C4ADA2EB186423BD1BAF1000FAB
:1079000044D126E0BAF1000F13D0022000F026FE89
:1079100000F0EEFD8DED020B9DED220B8DED000BC9
:1079200010EE900A039961F31E0003909DED020B87
:10793000C9E78DED029B9DED220B19EE901A10EE1A
:10794000900A8DED000B61F31E0003909DED020B7C
:10795000B9E78DED02AB9DED220B1AEE901A10EEF9
:10796000900A8DED000B61F31E0003909DED020B5C
:10797000A9E729E00ADA9DED220B51EC180B53EC34
:10798000102BF0F7ABFD41EC100B9CE79DED220BAB
:1079900099E7864218DAB4F1804F0DD0A4F1005077
:1079A000B0F1FF5010D1002D0EDB9DED220B51ECFC
:1079B000100B01F0C4F9E6E79DED220B53EC102B00
:1079C00051EC100B00F0AEBC9DED220B51EC100BF6
:1079D00001F01DF8BAF1000FCDE90C0134D19FED93
:1079E000720BDEB1A6F1E040B0F17F602CD1002D2A
:1079F00001DD002C0DDA002D01DD002C1FDB002D38
:107A000016DA002C14DB012F08BF9FED690B3FF441
:107A10005AAFB0EE490AF0EE690A54E7022F18BFD8
:107A2000002D0CD0012F0AD1002DFFF64CAF06E03F
:107A3000002DB8BF002C07DA012F3FF444AFB0EEA1
:107A40004A0AF0EE6A0A3EE7012000EBE57A5AEABC
:107A500007000CD05848002580457CDD5749584820
:107A6000884514DDB0420DDB002C19DB2BE0012032
:107A700000F074FD16B0BDEC0C8B04B0BDE8F04D09
:107A800000F026BDB34502DC002C09DC1BE0864279
:107A900002DA002C17DA03E05E4527DD002C12DD48
:107AA000022000F05BFD00F023FD10EE901A19EEAD
:107AB000900A8DED020B8DED009B61F31E0003908B
:107AC0009DED020BFFE6022000F048FD00F020FDD6
:107AD00010EE901A18EE900A8DED020B8DED008BD2
:107AE00061F31E0003909DED020BECE69DED220B71
:107AF00053EC182B51EC100BF0F778FC9FED320B88
:107B0000CDE90A0153EC102B9DED0A0B51EC100B43
:107B1000F0F772FC9FED2E1B53EC112BF0F769FC74
:107B20009DED0A1B53EC112BF0F766FC9FED2A1B11
:107B300053EC112BF0F75DFC9DED0A0B41EC190B9A
:107B400053EC102B51EC100BF0F756FC53EC192BA7
:107B5000F0F752FC00E07EE09FED210B41EC1A0BA8
:107B600053EC102B9DED0A0B51EC100B3CE0000088
:107B7000FFFF1F00FFFF0F00000000000000F03FAC
:107B80000000F03F0000F07F0000404301FCFFFFD9
:107B9000000000000000F07F000000000000000076
:107BA000FE3B00000000000000000000000000801C
:107BB000000000000000F0FF0000E0410000F04382
:107BC000FFFFEF3F00000000000000000000D03F7A
:107BD000555555555555D53F000000000000E03F74
:107BE000000000604715F73FF0F706FC41EC190B69
:107BF0009FEDFD0B51EC1A0B53EC102BF0F7FCFB37
:107C000041EC1A0B9FEDFA0B53EC102B9DED0A0B78
:107C100051EC100BF0F7F0FB53EC1A2BF0F7E6FBEE
:107C200041EC1A0B51EC190B53EC1A2BF0F73DFBFE
:107C30000690CDE906519DED060B53EC192B51EC46
:107C4000100BF0F7D3FB53EC1A2BF0F7D2FB41ECFF
:107C5000100B00F09FB90020B6F5801F0EDA9FEDE3
:107C6000E60B53EC102B9DED0C0B51EC100BF0F7C9
:107C7000C3FBCDE90C016FF034000E4600EB26503B
:107C8000A0F2FF38C6F31300DD4940F07F6646F0EE
:107C900040568842D8BF002409DDDA498142C8BF76
:107CA000012404DC0024A6F5801608F10108D6485A
:107CB000784400EBC4000D9690ED00BB9DED0C0BDD
:107CC00053EC1B2B51EC100BF0F790FB9DED0C0BC4
:107CD00041EC1A0B53EC1B2B51EC100BF0F7E5FAAF
:107CE00041EC100B51EC180B53EC102BF0F7F6FB9A
:107CF00041EC1C0B51EC1A0B53EC1C2BF0F77CFBEA
:107D000041EC190BC1488DED109B7844109590ED16
:107D1000000B4FF0005040EA660000EB84408DED10
:107D20000A0B00F500200B909DED0A0B53EC1B2B6A
:107D300051EC100BF0F75AFB9DED0C1B53EC112B83
:107D4000F0F757FB41EC100B53EC102B9DED100B93
:107D500051EC100BF0F750FB9DED0A0B41EC1B0BA7
:107D600053EC102B9DED100B51EC100BF0F744FB76
:107D700053EC1A2BF0F73DFB53EC1B2BF0F736FBC3
:107D800053EC1C2BF0F738FB41EC1B0B53EC192B7D
:107D900051EC190BF0F730FB41EC1A0B9C48062113
:107DA000B0EE4A0AF0EE6A0A784400F0E9FAB0EE62
:107DB00040CAF0EE60CA53EC1A2B51EC1A0BF0F7E4
:107DC0001BFB53EC1C2BF0F717FB9DED100B41EC4C
:107DD0001A0B53EC192B51EC100BF0F766FA53EC1D
:107DE0001B2BF0F709FB53EC1A2BF0F75EFA9DED15
:107DF000100B41EC1A0B53EC102B51EC100BF0F75D
:107E0000FBFA41EC1C0B9FED84DB53EC1D2BF0F7D0
:107E10004CFA53EC1A2BF0F748FA0A90CDE90A51C4
:107E20009DED0A0B53EC1D2B51EC100BF0F7DEFA15
:107E300053EC1C2BF0F7DAFA53EC1A2BF0F7D9FAC3
:107E40009DED0A0B41EC1C0B53EC102B9DED100B20
:107E500051EC100BF0F7D0FA41EC1A0B53EC192B44
:107E600051EC1C0BF0F7C8FA9DED0A0B41EC190B15
:107E700053EC102B51EC1B0BF0F7BEFA53EC192B03
:107E8000F0F713FA41EC190B51EC1A0B53EC192BC8
:107E9000F0F70BFA1090CDE910519DED100B53EC5B
:107EA0001A2B51EC100BF0F7A1FA53EC192BF0F749
:107EB000A0FA41EC190B9FED5A0B53EC102B9DEDE2
:107EC000100B51EC100BF0F797FA41EC1A0B9FEDE9
:107ED000560B51EC190B53EC102BF0F78DFA41ECCB
:107EE000190B9FED530B53EC102B9DED100B51EC28
:107EF000100BF0F781FA53EC192BF0F7D6F941EC9F
:107F0000100B4D48784400EBC40090ED001B51EC81
:107F1000100B53EC112BF0F7C8F941EC190B40464C
:107F2000F0F7D1FCCDE90A0153EC192B51EC1A0BF7
:107F3000F0F7BBF941EC100B4048784400EBC4006B
:107F400090ED00BB51EC100B53EC1B2BF0F7ADF98F
:107F50009DED0A1B53EC112BF0F7A7F90690CDE924
:107F600006519DED0A0B53EC102B9DED060B51ECC9
:107F7000100BF0F73BFA53EC1B2BF0F737FA53ECEE
:107F80001A2BF0F733FA53EC192BF0F732FA41ECD5
:107F9000100B00BF781EB0EE48AAF0EE68AA5AEAAD
:107FA000000008BF9FED268B9DED241B53EC102B8A
:107FB0008DED001B00959DED240B51EC100BF0F79F
:107FC0001BFA9DED000B41EC190B53EC102B9DEDB2
:107FD000240B51EC100BF0F709FA9DED061B53EC46
:107FE000112BF0F709FA2FE0FE822B654715F73FBA
:107FF00044DF5DF80BAE543E00000000000040433B
:108000008E9803007AB60B0074370000DA37000050
:10801000AC36000000000000000000000000084036
:10802000000000E009C7EE3FFD033ADC09C7EE3F60
:10803000F5015B14E02F3EBE40350000FA3400002D
:10804000000000000000F0BF53EC192BF0F72DF9F1
:108050009DED060B41EC190B53EC102B9DED000B25
:1080600051EC100BF0F7C8F9CDE910019DED100BA4
:1080700051EC190B53EC102BF0F717F9CDE9020175
:108080000C46AB498C422FDB611A084318D19DED99
:10809000100B53EC102B9DED020B51EC100BF0F775
:1080A000A5F941EC1B0B9FEDA40B51EC190B53EC04
:1080B000102BF0F7FAF853EC1B2BF0F715FC2DD230
:1080C000022000F04BFA00F013FA10EE901A18EEAE
:1080D000900A8DED020B8DED008B61F31E00039075
:1080E0009DED020BFFF7EFBB954A24F00041914252
:1080F00014D39449214408437FF4E5AC9DED100B63
:1081000053EC102B9DED020B51EC100BF0F76EF9B8
:1081100053EC192BF0F7E8FB7FF6D5AC24F00040C8
:1081200089498A4A002601EB205182422BDA481CF9
:108130004FF4801121FA00F02044854AC0F30A511F
:108140007A44A1F2FF3192ED000B824A8DED0A0BC9
:10815000CA4020EA0202C0F3130040F48010C1F1CB
:10816000140120FA01F60B92002CB8BF76429DED67
:108170000A0B53EC102B9DED100B51EC100BF0F78C
:1081800035F9CDE910019DED100B51EC190B53ECB5
:10819000102BF0F78AF89FED700B0A90CDE90A5189
:1081A00053EC102B9DED0A0B51EC100BF0F724F95A
:1081B00041EC1B0B9FED6A0B53EC102B9DED0A0B52
:1081C00051EC100BF0F718F99DED100B41EC1C0B66
:1081D00053EC102B9DED0A0B51EC100BF0F706F948
:1081E00053EC192BF0F705F99FED5F1B53EC112BA6
:1081F000F0F702F953EC1C2BF0F757F841EC190B90
:1082000051EC1B0B53EC192BF0F74FF8CDE90201A1
:108210009DED020B53EC1B2B51EC100BF0F7E6F825
:1082200053EC192BF0F7E5F89DED020B41EC190B1F
:1082300053EC102B51EC100BF0F7DEF8CDE90A01EE
:108240004B489DED0A0B0521784400F099F89DED0F
:108250000A1B51EC100B53EC112BF0F7CDF89DEDF0
:10826000021B53EC112BF0F7C4F8CDE906019DED8C
:10827000020B53EC192B51EC100BF0F7BDF853EC3B
:10828000192BF0F712F89FED3C0B41EC190B53EC56
:10829000102B9DED060B51EC100BF0F7A7F89DEDA0
:1082A000060B41EC1B0B53EC102B9DED020B51EC1C
:1082B000100BF0F7A1F853EC1B2BF0F70FF953EC70
:1082C000192BF0F793F89DED021B53EC112BF0F7EF
:1082D0008DF853EC1A2BF0F78CF8CDE9020101EB85
:1082E000065001150029C8BF039015DC9DED020B57
:1082F000324651EC100BF0F7CFFAFEF775FF042869
:1083000008BF00F005F932469DED020B51EC100B51
:10831000F0F7C2FACDE902019DED020B51EC180B0A
:1083200053EC102BF0F768F8FFF72DBB00000000AE
:108330000000904000000000FE822B654715973C2E
:1083400000CC904000346F3F01FCFFFF0000E03F95
:10835000A4330000FFFF0F0000000000432EE63FA3
:10836000396CA80C615C20BEEF39FAFE422EE63F64
:108370003C3200000000000000000000000000404F
:1083800070B504462DED028B4D1E00EBC500B0EE1E
:10839000408AF0EE608A90ED000B35F0060017D0B1
:1083A00053EC182B51EC100BF0F726F841EC100BA6
:1083B0006D1E04EBC50090ED001B51EC100B53EC4F
:1083C000112BEFF772FF41EC100B35F00600E7D1EF
:1083D000022D36D0042D1CD0062D1CBFBDEC028B07
:1083E00070BD53EC182B51EC100BF0F705F894ED21
:1083F0000A1B53EC112BEFF758FF53EC182BEFF738
:10840000FBFF94ED081B53EC112BEFF74EFF41ECF3
:10841000100B53EC182B51EC100BEFF7EDFF94ED14
:10842000061B53EC112BEFF740FF53EC182BEFF723
:10843000E3FF94ED040B53EC102BEFF736FF41EC08
:10844000100B53EC182B51EC100BEFF7D5FF94EDFC
:10845000021B53EC112BEFF728FF53EC182BEFF70F
:10846000CBFF94ED001B53EC112BEFF71EFFBDEC7F
:10847000028B41EC100B70BD9FED070B10B553EC58
:10848000102B9FED070B51EC100BF0F727F841EC88
:10849000100B10BD000000000000000000000000F4
:1084A000000000000000F03F10B553EC102B51EC21
:1084B000100BEFF7FAFE41EC100B10BD10B553ECAA
:1084C000112B51EC100BEFF7F0FE41EC100B10BD2F
:1084D0009FED050B10B553EC102B51EC100BEFF783
:1084E000FDFF41EC100B10BD00000000000000007B
:1084F0009FED050B10B553EC102B51EC100BEFF763
:108500007BFF41EC100B10BD00000000000000706C
:108510009FED050B10B553EC102B51EC100BEFF742
:108520006BFF41EC100B10BD0000000000000010BC
:108530000148006870470000D010002002E008C821
:10854000121F08C1002AFAD170477047002001E0CD
:1085500001C1121F002AFBD17047000001490860C9
:1085600070470000D010002030380A2801D20120C6
:1085700070470020704700002DE9FF4F8DB00F4677
:108580000546002606E025280BD0DDE90F129047AE
:108590006D1C761C28780028F5D111B03046BDE856
:1085A000F08F0024A246A1460122EC4900E00443DA
:1085B00015F8013F203B02FA03F00842F7D1287872
:1085C0002A2810D06FF02F022878A0F13001092955
:1085D00014D80AEB8A0102EB410144F0020400EBDB
:1085E000010A6D1CF0E701CF5FEA000A03D544F4ED
:1085F0000054CAF1000A44F002046D1C28782E28A9
:1086000017D115F8010F44F004042A280ED06FF09A
:108610002F022878A0F1300109290AD809EB890135
:1086200002EB410100EB01096D1CF2E757F8049BD6
:108630006D1C28786C280FD006DC4C2817D06828D1
:108640000DD06A2814D104E0742810D07A280FD1F4
:108650000DE044F400140AE044F4801401E044F412
:1086600040146978814202D104F580146D1C6D1CA0
:108670002A786E2A1FD00CDC632A31D004DC002A51
:108680008BD0582A11D1A3E0642A68D0692A0CD172
:1086900065E0732A2ED004DC6F2A73D0702A04D1CF
:1086A0009BE0752A6FD0782A6ED01046DDE90F1254
:1086B0009047761C50E1C4F30250022806D00328EC
:1086C00009D0042801CF09D0066045E101CFF11798
:1086D000C0E9006140E101CF06803DE106703BE169
:1086E00017F8040B8DF8000000208DF80100EB4610
:1086F000012003E057F804BB4FF0FF3061074FF053
:10870000000102D40DE008F10101884649450FDA65
:108710008045F8DB1BF808100029F4D108E008F1C7
:10872000010188468142FADB1BF808100029F6D1C6
:10873000DDE90F23AAEB08008146214600F036F957
:10874000304400EB080604E0DDE90F121BF8010BD2
:108750009047B8F10108F7D221464846F7E00A21D0
:10876000C4F302534FF0000B0891022B04D001CF49
:10877000C117032B09D00AE0FF1D27F00707F7E810
:10878000020108E032E01FE020E000B2C117042B34
:1087900001D140B2C117031E71F1000307DA4FF097
:1087A000000CD0EB0C006CEB01012D2302E0230543
:1087B00004D52B238DF82430012303E0E30701D0F7
:1087C0002023F7E7984658E00A2110E010210EE038
:1087D00010204FF0000B08900CE010214FF0000B20
:1087E00044F004044FF00809089103E008214FF019
:1087F000000B0891C4F30253022B04D001CF0021D7
:10880000032B06D006E0FF1D27F00707F7E802015B
:1088100003E080B2042B00D1C0B24FF00008230760
:108820002BD5702A07D0DDF820C08CF0100C5CEA44
:108830000B0C05D00EE040238DF82430012308E016
:1088400050EA010306D030238DF824308DF825201E
:1088500002239846DDF820C08CF0080C5CEA0B0C73
:108860000BD150EA010301D1630706D530238DF8FF
:1088700024304FF00108A9F10109582A04D038A288
:108880000B9208AA0A920BE03AA2F9E75B46089A13
:10889000EFF796FC0B9B9B5C0A9A521E0A92137090
:1088A00050EA0102F2D10A98ADEB000000F1200B72
:1088B000600702D524F4803401E04FF00109D94566
:1088C00002DDA9EB0B0000E0002000EB0B014144AE
:1088D0000890AAEB010AE00306D4DDE90F23214644
:1088E000504600F063F806444FF0000908E009A97B
:1088F00011F80900DDE90F12904709F10109761C12
:10890000C145F4DBE0030CD5DDE90F2321465046D9
:1089100000F04CF8064404E0DDE90F1230209047E7
:10892000761C0899481E08900029F5DC08E00A9892
:108930000A990078491C0A91DDE90F129047761CCC
:10894000BBF10001ABF1010BF1DC21465046DDE942
:108950000F2300F019F806446D1C1BE609280100DE
:1089600030313233343536373839616263646566A5
:108970000000000030313233343536373839414267
:1089800043444546000000002DE9F041044600251F
:108990001E461746880404D405E039462020B04717
:1089A0006D1C641EF9D52846BDE8F0812DE9F04123
:1089B000044600251E469046C80301D5302700E036
:1089C0002027880404D505E041463846B0476D1C91
:1089D000641EF9D52846BDE8F0810A68531C0B6077
:1089E00010707047002806D04DF6BC231946491E6A
:1089F000FDD2401EFAD17047002100EB800002E05A
:108A000000BF491CC9B2B1EB400FF9D3704782B027
:108A1000CDE9000121F0004001909DED000B02B076
:108A200051EC100B7047000010B50E4C1021204681
:108A3000F1F7ADFC206840F48060206020212046E2
:108A4000F1F7A5FC0220FFF7D7FF10212046F1F730
:108A5000A0FC0220FFF7D0FF2046BDE81040102107
:108A6000F1F795BC0014024010B50E4C10212046C1
:108A7000F1F78DFC206840F48060206020212046C2
:108A8000F1F787FC0220FFF7B7FF10212046F1F72E
:108A900080FC0220FFF7B0FF2046BDE81040102107
:108AA000F1F775BC001402402DE9F041154E074660
:108AB0000024306820F440603060254610213046A4
:108AC000F1F765FC0220FFF797FF10213046F1F720
:108AD00060FC6006040E20213046F1F751FC08B11D
:108AE00044F001040120FFF787FF6D1CEDB2082D53
:108AF000E4D317B1FFF798FF01E0FFF7B5FF204679
:108B0000BDE8F0810014024070B5164E05463046AF
:108B1000316841F4806131601021F1F738FC0024A4
:108B200028064FF02001304602D5F1F732FC01E073
:108B3000F1F72DFC6806050E0220FFF75DFF1021FE
:108B40003046F1F726FC0220FFF756FF1021304691
:108B5000F1F71DFC0220FFF74FFF641CE4B2082C64
:108B6000DED370BD0014024010B50B4C206840F4F9
:108B70008060206020212046F1F70BFC1021204668
:108B8000F1F707FC0420FFF737FF2046BDE810404F
:108B90002021F1F7FCBB00000014024010B50B4C83
:108BA000206840F48060206020212046F1F7EFFB30
:108BB0000420FFF721FF10212046F1F7EAFB2046B1
:108BC000BDE810402021F1F7E4BB00000014024092
:108BD00070B5144D0024286820F4406028602021DE
:108BE0002846F1F7D6FB0120FFF706FF10212846A3
:108BF000F1F7CFFB0120FFF7FFFE07E0641CE4B2B2
:108C0000FA2C03D9FFF7CAFF012070BD20212846A6
:108C1000F1F7B6FB0028F1D110212846F1F7B7FB98
:108C2000002070BD0014024010B541EC100BFEF79F
:108C30000FFB51EC100B10BD70B5FCF753FA06207A
:108C400000F0BEF8552000F0DBF800F0AFF8124E4F
:108C500004464FF4805529463046F1F798FB2946E3
:108C60000E48F1F796FBAA2C11D1152000F0A8F8B8
:108C7000062000F0C5F81420FFF7BEFE00F096F8BD
:108C8000044629463046F1F784FB512C01D0FA20E6
:108C900070BD142070BD000000040240000C0240B2
:108CA0004FF400410803F8F7B1FE4FF08040FDF7A4
:108CB000B9FD0F48FEF798F90E48F0F7F5FC0D489E
:108CC0003030F0F7F1FC0C48F1F79CFA0B48F1F763
:108CD00099FAF1F703FE002080F310884FF47A70C0
:108CE000FFF780FEFDF798FEFDF7CCFEFCE70000E5
:108CF000001001408864024000000240000402406D
:108D00002DE9F04104460E4600250846EFF7B7FA74
:108D100007000ED10120BDE8F0816D1C3178ADB2A5
:108D2000884205D13A4631462046EFF7AFFA20B1E6
:108D3000641C20780028F0D1EDE72846EBE700B569
:108D40002DED048B83B041EC190BEFF7B9FF41EC2B
:108D5000180B18EE100A18EE901A8DED008B0028F3
:108D600018BF0120084320F00040C0F17F6000F1EF
:108D7000E040C00F14D019EE101A19EE900A8DEDD4
:108D8000009B002918BF0121084320F00040C0F1DA
:108D90007F6000F1E040C00F04BF0120FFF7DEFB61
:108DA00051EC180B03B0BDEC048B00BD10B50120D5
:108DB000FFF722FEBDE81040FF20FCF703BA0000D9
:108DC00070B50D4E04464FF4805529463046F1F7F4
:108DD000E0FA0320FFF710FE29463046F1F7D7FAF4
:108DE00029460648F1F7D5FA2046FCF7EBF9BDE82D
:108DF00070400320FFF700BE00040240000C024058
:108E000010B5FCF7DFF9BDE810400120FFF7F4BD15
:108E10005458485F56312E322E30003880250000DD
:108E2000010000000A000000000000000000000037
:108E30000000000000000000000000000000000032
:108E40000000000000000000000000000101000020
:108E5000000000000000000000000000020300000D
:108E600000000000000000000000000003050000FA
:108E700000000000000000000000000004070000E7
:108E800000000000000000000000000005050000D8
:108E900000000000000000000000000006060000C6
:108EA00000000000000000000000000007070000B4
:108EB00000000000000000000000000008080000A2
:108EC0000000000000000000000000000909000090
:108ED0000000000000000000000000000A0A00007E
:108EE0000000000000000000000000000B0B00006C
:108EF0000000000000000000000000000C0C00005A
:108F00000000000000000000000000000D0D000047
:108F10000000000000000000000000000E0E000035
:108F20000000000000000000000000000F0F000023
:108F30000000000000000000000000001010000011
:108F400000000000000000000000000041542B530E
:108F50004F434B413D5443502C6A6F796675656CA5
:108F60002E6A6F796675656C696E672E636F6D2CFE
:108F7000373031310D0A0000000000000000000011
:108F800000000000000000000000000000000000E1
:108F900000000000000000000000000000000000D1
:108FA00000000000000000000000000000000000C1
:108FB000000000000000000000004B46422D322E51
:108FC0003447000000000000000000000000000026
:108FD0000000000000000000000000000000000091
:108FE00000004B4642313233343536000000000079
:108FF000000000000000000000000004000000006D
:10900000000000001B8E01082041002037110020C5
:10901000640000000200010000000000F88F010859
:1090200020410020301100206600000005000100F2
:10903000010000001C8E010820410020E41A0020DD
:109040006B00000031010400020000004C8F010899
:10905000204100204A1600202F050000AC0001002E
:1090600003000000F78F010820410020401A002073
:10907000DB0500000200010004000000FC8F010875
:109080002041002028110020DD050000050001001E
:109090000500000000900108204100202C11002054
:1090A000E2050000050001000600000061002B2B16
:1090B0002B000D0A000041542B530D0A0041542B84
:1090C000534F434B413D5443502C746573742E6A87
:1090D0006F796675656C696E672E636F6D2C3730BE
:1090E00031310D0A0041542B574B4D4F443D4E45F5
:1090F000540D0A0041542B55415254464C3D3430D6
:1091000039360D0A0041542B4845415254454E3DD5
:109110004F46460D0A0041542B453D4F46460D0A29
:109120000041542B454E544D0D0A0041542B4943E8
:109130004349443F0D0A0041542B494D45493F0DD9
:109140000A0041542B574946493D4B46422D322E89
:1091500034472C4B46423132333435360D0A004108
:10916000542B536F636B65743D302C302C746573D6
:10917000742E6A6F796675656C696E672E636F6DA4
:109180002C373031310D0A0000C1814001C08041CF
:1091900001C0804100C1814001C0804100C18140C7
:1091A00000C1814001C0804101C0804100C18140B7
:1091B00000C1814001C0804100C1814001C08041A7
:1091C00001C0804100C1814001C0804100C1814097
:1091D00000C1814001C0804100C1814001C0804187
:1091E00001C0804100C1814000C1814001C0804177
:1091F00001C0804100C1814001C0804100C1814067
:1092000000C1814001C0804101C0804100C1814056
:1092100000C1814001C0804100C1814001C0804146
:1092200001C0804100C1814000C1814001C0804136
:1092300001C0804100C1814001C0804100C1814026
:1092400000C1814001C0804100C1814001C0804116
:1092500001C0804100C1814001C0804100C1814006
:1092600000C1814001C0804101C0804100C18140F6
:1092700000C1814001C0804100C1814001C08041E6
:1092800001C0804100C1814000C0C101C30302C2CE
:10929000C60607C705C5C404CC0C0DCD0FCFCE0E36
:1092A0000ACACB0BC90908C8D81819D91BDBDA1AA6
:1092B0001EDEDF1FDD1D1CDC14D4D515D71716D616
:1092C000D21213D311D1D010F03031F133F3F23286
:1092D00036F6F737F53534F43CFCFD3DFF3F3EFEF6
:1092E000FA3A3BFB39F9F83828E8E929EB2B2AEA66
:1092F000EE2E2FEF2DEDEC2CE42425E527E7E626D6
:1093000022E2E323E12120E0A06061A163A3A26245
:1093100066A6A767A56564A46CACAD6DAF6F6EAEB5
:10932000AA6A6BAB69A9A86878B8B979BB7B7ABA25
:10933000BE7E7FBF7DBDBC7CB47475B577B7B67695
:1093400072B2B373B17170B0509091519353529205
:1093500096565797559594549C5C5D9D5F9F9E5E75
:109360005A9A9B5B99595898884849894B8B8A4AE5
:109370004E8E8F4F8D4D4C8C448485458747468655
:10938000824243834181804041542B41504E3D00F5
:1093900000000000000000000000000000000000CD
:1093A00000000000000000000000000000000000BD
:1093B0000000000000000000000038000000000075
:1093C000000000000000000000000000000000009D
:1093D000000000000000000000000000000000008D
:1093E000000000000000000000000000000000007D
:1093F0000000000000000000BA930108FC65002096
:1094000038110020000000000200010000000000F0
:10941000BA930108FC6500203A1100200100000009
:109420000102000801000000BB930108FC65002058
:10943000EC100020010800003C00D00702000000F2
:10944000BA930108FC6500203A110020D10F0000FA
:1094500001020010030000000000000000000000F6
:1094600000000000000000000000000000000000FC
:1094700000000000000000000000000000000000EC
:1094800000000000000000000000000000000000DC
:1094900000000000000000000000000000000000CC
:1094A00000000000000000000000000000000000BC
:1094B00000000000000000000000000000000000AC
:1094C000000000000000000000000000000000009C
:1094D000000000000000000000000000000000008C
:1094E000000000000000000000000000000000007C
:1094F000000000000000000000000000000000006C
:10950000000000000000000000000000000000005B
:10951000000000000000000000000000000000004B
:10952000000000000000000000000000000000003B
:10953000000000000000000000000000000000002B
:10954000000000000000000000000000000000001B
:10955000000000000000000000000000000000000B
:1095600000000000000000000000000000000000FB
:1095700000000000000000000000000000000000EB
:1095800000000000000000000000000000000000DB
:1095900000000000000000000000000000000000CB
:1095A00000000000000000000000000000000000BB
:1095B00000000000000000000000000000000000AB
:1095C000000000000000000000000000000000009B
:1095D000000000000000000000000000000000008B
:1095E000002F000000000700070000147F147F1404
:1095F00000242A7F2A12006264081323003649558A
:10960000225000000503000000001C224100000061
:1096100041221C000014083E08140008083E0808F7
:10962000000000A060000008080808080000606052
:109630000000002010080402003E5149453E000091
:10964000427F4000004261514946002141454B3173
:10965000001814127F10002745454539003C4A493F
:1096600049300001710905030036494949360006B1
:109670004949291E00003636000000005636000019
:109680000008142241000014141414140000412294
:10969000140800020151090600324959513E007C6C
:1096A0001211127C007F49494936003E4141412256
:1096B000007F4141221C007F49494941007F09093F
:1096C0000901003E4149497A007F0808087F0000EF
:1096D000417F4100002040413F01007F08142241AA
:1096E000007F40404040007F020C027F007F040862
:1096F000107F003E4141413E007F09090906003EBE
:109700004151215E007F09192946004649494931E6
:109710000001017F0101003F4040403F001F204009
:10972000201F003F4038403F0063140814630007C7
:109730000870080700615149454300007F4141001E
:1097400000552A552A55000041417F0000040201BE
:10975000020400404040404000000102040000209C
:1097600054545478007F48444438003844444420DA
:1097700000384444487F00385454541800087E0987
:1097800001020018A4A4A47C007F0804047800004F
:10979000447D4000004080847D00007F102844000C
:1097A0000000417F4000007C04180478007C08041D
:1097B000047800384444443800FC24242418001859
:1097C000242418FC007C0804040800485454542045
:1097D00000043F444020003C4040207C001C2040CE
:1097E000201C003C4030403C004428102844001C11
:1097F000A0A0A07C004464544C4414141414141409
:109800000000000000000000000000000000FC005C
:109810000000000002000000000C020C020000002A
:109820000000000090D0BCD0BC90000300030000FA
:109830001824FE448C000302070201001824D8B04B
:109840004C80000300010201C038E438E00001024E
:1098500002010202080600000000000000000000F3
:10986000000000F80402000000010204000204F8F5
:1098700000000004020100009060F8609000000009
:10988000010000002020FC2020000000010000005A
:10989000000000000000080600000000202020203A
:1098A0002000000000000000000000000000000296
:1098B000000000000080601C0200040300000000A3
:1098C000F8040404F8000102020201000008FC0090
:1098D0000000000203020000188444241800030260
:1098E0000202020008042424D8000102020201003E
:1098F00040B088FC80000000000302003C242424C7
:10990000C400010202020100F824242CC00001025C
:10991000020201000C04E41C04000000030000002B
:10992000D8242424D800010202020100384444440F
:10993000F800000302020100000010000000000017
:1099400002000000000020000000000006000000EF
:1099500000205088040200000000010290909090C6
:109960009000000000000000000204885020000267
:10997000010000001804C4241800000002000000C8
:10998000F804E494F80001020202020000E09CF0F6
:10999000800002030000030204FC2424D800020318
:1099A00002020100F80404040C000102020201009A
:1099B00004FC0404F80002030202010004FC247405
:1099C0000C0002030202030004FC24740C000203D6
:1099D00002000000F0080444CC4000010202010033
:1099E00004FC2020FC040203000003020404FC0425
:1099F0000400020203020200000404FC0404060442
:109A00000403000004FC24D00C040203020003023F
:109A100004FC04000000020302020203FC3CC03C00
:109A2000FC0003000300030004FC30C4FC04020338
:109A300002000300F8040404F8000102020201001D
:109A400004FC24241800020302000000F8848404AB
:109A5000F80001020207050004FC246498000203D8
:109A600002000302182424448C00030202020100B5
:109A70000C04FC040C0000020302000004FC0000C3
:109A8000FC04000102020100047C80E01C040000D0
:109A9000030000001CE03CE01C0000030003000089
:109AA000049C609C0400020300030200041CE01CF0
:109AB00004000002030200000C84641C0400020382
:109AC000020203000000FE0202000000070404007E
:109AD000000E30C00000000000010200000202FE83
:109AE000000000040407000000040204000000005D
:109AF0000000000000000000000008080808080836
:109B00000000020000000000000000000040A0A0D3
:109B1000C00000010202030204FC2020C000000378
:109B20000202010000C020206000000102020200C9
:109B300000C02024FC0000010202030200C0A0A01B
:109B4000C0000001020202000020F82424040002E8
:109B5000030202000040A0A0602000070A0A0A04D5
:109B600004FC2020C0000203020003020020E400E5
:109B70000000000203020000000020E400000808CA
:109B80000807000004FC80E020200203020003021A
:109B90000404FC000000020203020200E020E020B6
:109BA000C00003000300030020E02020C0000203E7
:109BB0000200030200C02020C000000102020100D8
:109BC00020E02020C000080F0A02010000C0202071
:109BD000E0000001020A0F0820E0402020000203FC
:109BE000020000000060A0A02000000202020300AA
:109BF0000020F820000000000102020020E0002008
